:020000040000fa
:080000000001040000000000f3
:020000040000fa
:10020000cf0b2100007922000001880000000000cf
:100210000c000700e0022800010020001100070088
:10022000000020000000e000020032000000020098
:10023000000000001a420200000000000040da0046
:100240000000fe004440a900e08721000000e0001b
:100250000300320000002000a00188004440a800f4
:100260000000060091018800800078000000eb008b
:1002700015003700e280400032a0b4009101ba00be
:10028000e280400032a0b4009102ba00e280400057
:1002900032a0b4000002eb00472bde00f507b200ed
:1002a000602ce10004003a000059eb008301e900f2
:1002b000fdff3e00040037006128e100010032002c
:1002c0000082eb00040007001101ba000200e00008
:1002d000e8ff3a00000006003159ba008301e90046
:1002e0000c0032002159ba008301e90008003200f5
:1002f0000400e00003003a00e280400032a0b400b5
:10030000f5ff370011d9ba008301e900faff3a007e
:100310008100e800e180400032a0b4000000060047
:10032000a001040000000000ca0104000000000059
:100330001c0b04000000000000000400000000008e
:10034000889fbe00800478000100780002047800d5
:10035000890178001100200025000700880f500057
:10036000010032008004eb00090078004f04be0059
:10037000000006000000fa004fb99700e88157001e
:1003800001db2000001a20006e0007000080fa0048
:1003900000000600881f7800020478002201070090
:1003a000080040004f047800000006000000fa003a
:1003b000881f7800000478003fb99700ea81570051
:1003c00080007800a01c20005e00070080007800fc
:1003d0000000e000020035000040eb0000f478006f
:1003e000010078004f0478000080fa000000060049
:1003f000889fbe008a9fbe008c9fbe008e1f780023
:100400008106780083047800000678000288b9002d
:10041000000778000000e00002003a0000017800c8
:10042000420037000d00e000400032000005780077
:10043000c900900069009000808f500004003900ce
:1004400009007800ff0007000000e00029003500e7
:10045000004020001900600003003a000a04780000
:10046000800578000b0037000a017800a100200009
:100470000c00780036010700800578000000e000dd
:1004800002003a000a047800020037000c00500015
:100490000004e800c90190006900900003005000ca
:1004a000880f500002003100000478008005eb0046
:1004b000080178008c00780003007800da0007005b
:1004c0000806460008055500490090000000440059
:1004d000c00498000b00e00004003200090078001e
:1004e000250107000000e00002003a000a00e000d9
:1004f000cfff3a00008020001900600002003200a7
:10050000090078001c01070000c0200019006000ed
:100510000200320049009000e00498000a005700f1
:10052000110009000d80d800000178000200780059
:100530004f0778004f06be004f05be004f04be00b7
:10054000000006006200fa00889fbe008a9fbe007d
:100550000004be00020578008300780060f92f00d7
:100560000f0040004101070088979f0099979f0066
:100570000000eb00a09f9f009a4578000b80fb00d5
:100580000000ea00cf04de0050c2b30080cf550067
:100590000200320009047800010037000904e90074
:1005a0000800e0000b0034001f909700080178005d
:1005b0008a0078008f9197000300010090979f00b8
:1005c0000000e000930032002f98970000004400e4
:1005d000a09f9f000905450050c2b30080cf550081
:1005e000040032000b04e000e3ff3a002f9897006c
:1005f000890037000000eb00809f9f00f0979f006c
:10060000e0979f00d0979f00c0979f00b0979f00f2
:10061000c09f9f000900370080ea20000080500042
:1006200000004000c1e92000e10078004f989700e9
:1006300001007000c09f9f000a05e8001a4478007e
:100640008800fb0080ea20000d0107008000780090
:100650000000e000f0ff3a00a0c2b300804f540059
:100660000e003a00bf8897000180e900b08f9f001c
:1006700010007800b09f9f000000e00005003d00e2
:100680000000ea00b09f9f004f9897000020a00054
:10069000c09f9f000a05e80010003700b19f9f002f
:1006a00009003700bf989700f0ff2700808f5000a7
:1006b000040032006a08b900000041000300400055
:1006c000b09f9f000a05e8001a01fb0003fd2f0000
:1006d00003004100e90f5000f2ff3600e0c2b30012
:1006e0009a4f1000040032000080eb00909f9f00a2
:1006f0008a0478001c0037008a04e800a0c2b30016
:10070000994f100007003a00bf8897000180e90068
:10071000b08f9f0010007800909f9f008a84e800af
:10072000110037000000eb00909f9f000900370088
:100730009f989700f0ff2700808f50000400320040
:100740006a08b9000000410003004000909f9f002c
:100750008904e8001901fb0003fd2f00030041009c
:10076000e90f5000f2ff3600194478008800fb00c2
:10077000e0ea2000c20007000000e00002003a00aa
:1007800000447800010037008904e800a87f9f003a
:1007900080c6b300804f540004003a00994f140003
:1007a0000a003a006640500006003700c0c6b30099
:1007b000804f540005003a00994f140003003a009e
:1007c00065404000a07f9f008904e8000905e8001b
:1007d000c8fb2f000f04440060f92f000f004000f9
:1007e0008085e80088017800194178008000780051
:1007f0000b007800ab0007000000e00005003a00a5
:10080000880078000b007800230207000000e00059
:1008100059ff3d000080eb004f05be004f04be00b5
:100820000080fa00000006008001eb0002003700a3
:1008300061f079008301e800828f5100fcff3a00eb
:1008400000000600889fbe0000047800c0019000f0
:10085000600090008000eb00808f5100390039006b
:10086000180178002000290000006100e20f50000c
:1008700007003200002020000200e00001003500e7
:1008800000202400000c71008080eb002d00370058
:100890000100260001006100810f500008003a00ad
:1008a00038009000808f5100050039000800780062
:1008b000310007008080eb000000e00021003a00da
:1008c00000c020001800600017003a00a804900043
:1008d0006002200008004000808f540012003a009f
:1008e00000202000b6020700800078002004980055
:1008f0000000e00005003a0029049800490498002f
:100900000900e80030049800060037001860a000d5
:10091000400498000020b00030049800410c98007a
:10092000510c9800f802070028009000500498002d
:10093000380090006004980000002600180c700039
:100940008000eb00010078004f04be0000000600ac
:100950008001eb00040037008301e80090cf100015
:10096000040032000000e800828f5100faff3a00d4
:100970000000eb0000000600889fbe000004780025
:100980000000e0000e003a008004780088d72000c4
:10099000180078000000e00004003200f6ff0700b5
:1009a0000000e00001003d008084eb000884e800c6
:1009b00080d82000800f540029003200f4ff370057
:1009c000000022001800600024003200a8049000fb
:1009d0000800370009015000384090000000fb007b
:1009e00089007800720907000000e000130034005d
:1009f0008084440048009000808f5400f5ff390047
:100a000028009000400498001801780000c02000e1
:100a10000000610002003200a800900001003700d1
:100a2000b800900000002400000061000a003200bd
:100a3000610498008004eb00090037002800900052
:100a40004004980060049800500c98001890a00092
:100a50008084eb0002003700510c9800800478007d
:100a6000090078004f04be00000006000200fa00f2
:100a7000f1bf9f00010878000080fa000000060026
:100a8000040037000204e00001003a000000050005
:100a90000000e80010417800814f5100f9ff3a0052
:100aa00000000600889fbe008a1f780000047800be
:100ab00001027800824478000305780070c6b30014
:100ac000804f510021003c0000c0e900804f5100e0
:100ad000de003d0072405000804f51004b0132005b
:100ae0000d003c006c405000804f51005e013c0006
:100af00000c0e900804f5100d4003d0050c2b30057
:100b0000804f5100550132007c404000804f510021
:100b100055013a00cd00370010c6b300804f510098
:100b2000ca00320004003c0069405000804f510070
:100b30004d013a007200370030c6b300804f5100bb
:100b4000180032000040e8000900370000c7b30079
:100b5000804f51001e01320008003c0000c0e90037
:100b6000804f5100e400320065003c0065405000b9
:100b700080cf54003c013a000f00370050c7b3004b
:100b8000804f51005e00320063404000804f5100b2
:100b90005b00320065405000804f510032013a0046
:100ba0001a0137009180e900010a7800780090006e
:100bb0009171780032013700a8609000c0c6b30080
:100bc00080cf50000a003a00940078006480500002
:100bd000000a78001000be004f89de00cf91de00d1
:100be0000002be0002037800820378001300370081
:100bf00010c7b30080cf500003003200a0c6b3007e
:100c000080cf500006003a009400780068805000c1
:100c1000000a78003002be002003be000700370043
:100c20001480e900000a78001000780000027800c3
:100c3000cfa2de000503780086037800049cbe0086
:100c40000694be00a860900080c6b30080cf50001c
:100c50000e00320020c6b30080cf500005003a00dd
:100c60000400fb00cf80de000101780082017800e3
:100c70000a00370040c7b30080cf500003003200a5
:100c80006640400080cf500006003a000400780023
:100c9000cf80de000101780082017800009cbe0058
:100ca0000294be003800be002801be00e00f5000d4
:100cb000e08f5800e00f5900e08f590003003d001d
:100cc00078009000d1c2b3000a00370008109000ed
:100cd0000018a3000300320078009000b1c2b300f6
:100ce000040037000008a300530032007800900091
:100cf00001c2b300017578000000e8004d00370024
:100d0000a8609000c0c6b30080cf500006003a0033
:100d10009400780064805000000a78001002be0041
:100d20006033b8001300370010c7b30080cf500005
:100d300003003200a0c6b30080cf500006003a0086
:100d40009400780068805000000a78003002be00ed
:100d50002003be00070037001480e900000a780075
:100d60001000780000027800050020000600200036
:100d700007002000049cbe000694be00a8609000fe
:100d800080c6b30080cf50000e00320020c6b300f2
:100d900080cf500005003a000480fb0001002000d5
:100da00002002000030020000a00370040c7b30003
:100db00080cf5000030032006640400080cf5000da
:100dc00006003a0004007800010020000200200024
:100dd00003002000009cbe000294be00081090009a
:100de0000038a300140032003800be002801be0005
:100df000e00f5000e08f5800e00f5900e08f5900dd
:100e00000d00320080c7b30080cf540003003200d1
:100e100080c5b30080cf540007003a0078009000ee
:100e200001c3b300017578008000e80009f578007f
:100e30000080e800700498007800900000004500f1
:100e400060049800894078006d003700a860900029
:100e5000c0c4b30080cf500006003a009400780070
:100e600068805000000a78005001be004000be00bb
:100e7000050037009400780064805000000a780074
:100e80001000be006c0a0700009cbe000294be0069
:100e9000380090000000e00003003d007800900062
:100ea000d1c2b3000a003700081090000018a30058
:100eb0000300320078009000b1c2b3000400370094
:100ec0000008a300050032007800900001c2b300c2
:100ed000017578000000e800700498007800900028
:100ee0000000450060049800894078000800780000
:100ef000dd01070064003700a8609000c0c6b300a1
:100f000080cf5000250032000a003c0064405000b1
:100f100080cf50002800320000c0e80080cf500091
:100f2000140032006840500080cf500022003a0088
:100f30000a00370040c7b30080cf50001e003200c7
:100f40006640400080cf50001b00320069405000d6
:100f500080cf500018003a00060037001480e900e6
:100f6000000a780010007800485c9000084878007b
:100f7000450037001480e900000a7800100278006c
:100f800068089000cf80de000101780082017800bf
:100f9000009abe000292be003b0037001480e900b8
:100fa000000a78001001780068089000cf80de0009
:100fb0000089be00340037001480e900000a780080
:100fc00010007800680c9000080878002e003700a8
:100fd0001180e9008008780010007800cf80de00e2
:100fe0000101780082017800009cbe000294be00de
:100ff00078009000000045006004980081c7b300ad
:1010000008007800c10307001f0037001480e900c2
:10101000000a7800100078006004980058099000d9
:101020000200e00002003d0045050700090037000e
:101030008000eb0046fe0700800078000000e00022
:10104000030032006800900000805000010037006b
:1010500058089000100c98000b00370078009000a2
:101060000275780006003700780090008000450087
:101070000904e00001003a0059c2b3008948780031
:101080000000e800700498000000eb004f057800b5
:101090004f04be00000006000400fa00889fbe0056
:1010a0008a9fbe008c1f780000047800010678003b
:1010b00070089000f800900001005000880890002f
:1010c000010050009808900001005000a80890000e
:1010d00001005000b808900001005000c8089000be
:1010e000810550000002220090bf9f0000032300f2
:1010f000a0bf9f00081090000028a30018003a002d
:101100000b00e000160034008b047800090578001d
:10111000e28f5400020036002a002000020037004f
:101120000900e0000b00340058009000c801900056
:101130000a017800ee805700030001005004980077
:101140000000e000960032006808900000004500b2
:10115000600c98008a8454004240a900ebff3c00d8
:10116000780190000200e0000b003400580090006d
:10117000c80190008c007800030001005004980022
:101180000000e0008600320068089000f80090003f
:1011900001004000600c9800880c90000900e000fd
:1011a0001500340009057800e28f54000200360073
:1011b0002a002000020037000900e0000b00340084
:1011c00058009000c80190000a017800ec80570098
:1011d00003000100500498000000e000700032009d
:1011e0006808900000004500600c98008a84540054
:1011f0004240a900ebff3c00180990000200e0000b
:101200000b003400e800900058009000c8019000e6
:1012100003000100500498000000e000600032006c
:10122000680890009808900001004000600c980049
:10123000a80c90000900e0001500340009057800b2
:10124000e28f5400020036002a002000020037001e
:101250000900e0000b00340058009000c801900025
:101260000a017800ec805700030001005004980048
:101270000000e0004a0032006808900000004500cd
:10128000600c98008a8454004240a900ebff3c00a7
:10129000380990000200e0000d003400e8009000e2
:1012a000180890008080400058009000c80190000d
:1012b00003000100500498000000e00038003200f4
:1012c00068089000b808900001004000600c980089
:1012d000c80c90000900e0001500340009057800f2
:1012e000e28f5400020036002a002000020037007e
:1012f0000900e0000b00340058009000c801900085
:101300000a017800ec8057000300010050049800a7
:101310000000e00022003200680890000000450054
:10132000600c98008a8454004240a900ebff3c0006
:10133000081090000028a3001b0032000b00e00002
:10134000190034008b04780009057800e28f5400fe
:10135000020036002a002000020037000900e000e9
:101360000b00340058009000c80190000a0178007a
:10137000ee80570003000100500498000000e000d8
:10138000070032006808900000004500600c9800db
:101390008a8454004240a90003003400eaff370069
:1013a0000080eb00010037000000eb004f067800e2
:1013b0004f05be004f04be000080fa00000006008a
:1013c000889fbe00e30440000900a100808f540004
:1013d0004a003600e38f540001003e00490020001f
:1013e000c27580000200e000020032008200780036
:1013f0000c003700a1eb200003003700908f540051
:10140000230036008080e800110078000000e00032
:10141000faff3a000f003700908f54001c0036008e
:101420008080e800110078000000e000faff3a0038
:1014300012017800a1eb200003003700908f5400c8
:10144000130036008080e80011007800820f500001
:10145000faff3a00b8758000890f5400010031008e
:1014600009047800080078003c0407000000e00050
:1014700004003a00890f5400200032000804d10013
:10148000f5ff3700081878003b040700d4ff370049
:10149000110178009201780064805100890f50009a
:1014a0000300310012009000800878000700370028
:1014b0000900410080087800920190001300980014
:1014c0001100780012881400090978009100780052
:1014d0000100e00005003200110090000000e00073
:1014e000020032000180e800010037000000eb003c
:1014f000c07588000280e800010037000000eb00a2
:101500004f04be0000000600881f7800e8eb2000b2
:101510001804e00004003a00c0b120004a040700ab
:1015200020c0b300004c78004f0478000000060093
:10153000889fbe00000478000ffd0700800478003b
:101540000004200018006000020032002800900013
:10155000090407000000eb002004980038409000c8
:101560000004e000050035000000fb00c406070091
:101570000000e000010032008084eb0018109000b1
:101580000000e00008003200c60607000000e0008e
:10159000010032008084eb0018109000f603070071
:1015a0000000eb00101498000008200018006000f4
:1015b000100032000000eb0081d72000910f1400d2
:1015c000070032000000e8008180e800e80f5000ca
:1015d000faff3a0008007800e7030700130037001d
:1015e000000140008000eb0080d72000013079002e
:1015f000f8ff3700000c780000c0eb003044980082
:101600006002200008004000200498004004980078
:1016100050049800400c980060049800500c98000a
:101620007004980076004400000c980009007800cf
:101630004f04be0000000600881f780068d8200014
:10164000180078000000e00001003200b8ff070039
:101650000884e90060d72000800f5400f8ff3a00aa
:101660004f047800000006008f04b000889fbe0081
:101670008a9fbe008c9fbe008e1f7800f0b79f002f
:1016800081f79f005001be004000be00f0979f0010
:10169000819f9f00929f9f00a39f9f0010c6b30051
:1016a0000ff19700804f51001600320010c4b300b4
:1016b000804f510013003200ffb197005308900093
:1016c0000000e00003003d0060002000d009980009
:1016d0000c0037000000e0000a003a0070c6b300ba
:1016e0000ff29700804f52000300320070c4b30025
:1016f000804f520003003a0010002000ffb2970014
:10170000d00a9800ffb09700c0fa2f000f004000e9
:10171000da03070080017800e20f500015003a005c
:1017200030002000ffb097009008980010c6b3006a
:101730000ff19700804f51000a00320064404000d2
:10174000804f5100070032000040e800804f5100f8
:101750000400320081e420000040e800804f510086
:1017600001003a00c1e42000ffb19700630090003f
:10177000160037000000e0001800340030002000a0
:101780007fb29700100a980010c6b3008ff297003e
:1017900080cf52000a0032006440400080cf5200e7
:1017a000070032000040e80080cf52000400320001
:1017b00001e520000040e80080cf520001003a001f
:1017c00041e520007fb19700620090003158780019
:1017d0003158780011487800c601370014c6b300ac
:1017e0008ff2970084cf52000300320010c4b30080
:1017f00080cf520013003a007fb097006001900044
:101800008200780000c3b30080587800ffb29700d0
:10181000e102980080c7b3008ff2970084cf520096
:101820000100320080c5b300804878000280e800e3
:10183000ffb09700e0009800710090000080e80081
:10184000f00098000300e00005003a00e3979f00d5
:1018500064fb2f000f01420003077800a00137004e
:1018600085e52000e5b79f0010c6b3008ff0970014
:1018700080cf50000500320010c4b30080cf50006c
:10188000a7003a0092e62000e2b79f00ffb1970060
:10189000530890001e0220000000e0000100350007
:1018a0000007e8000e02e800d4b79f006022b800ed
:1018b0006033b8007f9097008f9897001f9997002a
:1018c000af999700fb070700ffb097003102be00f9
:1018d0002103be000000e00004003d000400be0043
:1018e0000601be0003f0a200020037000400be00a3
:1018f0000601be00f0979f00819f9f00929f9f006e
:10190000a39f9f006f91970064015100e2979f0091
:10191000c3fa2f008f8141006a8041000048eb002c
:101920006b824100c4b79f0031003700c201200024
:1019300003002000e5fa2f000f8042007b03070020
:101940007f9497008f9c97001f9d9700af9d9700f5
:101950000800be000a01be00db0707000006be004b
:101960005fb1970067015100d2b79f004240a900c4
:101970000a003400000807000002be000203be0097
:101980000800be000a01be00fe070700f0979f0096
:10199000819f9f00929f9f00a39f9f00cfb19700c0
:1019a0006780410071002000050037006f6066000d
:1019b0004c6add004466de000c067200c4eede00f8
:1019c000e00f5600e08f5e00050034008100e90062
:1019d000e18f4000f5ff3a00010037000060eb00a6
:1019e0008100e900fdff3b0067004000c0b79f0099
:1019f000dfb297000500e000090034006022b80063
:101a00006033b8007f9097008f9897001f999700d8
:101a1000af999700dd0707000000e000c3ff3c001e
:101a200060fb2f008f0040004fb197000100510074
:101a30000000e9008e0f500001003d000007780013
:101a40000e00e00003003d0073fb2f000f814100fa
:101a50002c003700800f570005003d000e8040002d
:101a600010409000f3c0b300e74f500001003c006d
:101a70008041eb00c4fa2f000f0242000e0042002a
:101a80006a0040008e007800010037000000e90085
:101a90008100e90010417800834f5100fbff3200c4
:101aa0000107e800efcf510001003a000248e800ca
:101ab0000100e0000300350075fb2f000f8142009c
:101ac000060037000e07e8006f90970064004000a2
:101ad000e0979f0061fb2f000f8140008e004100c6
:101ae0008e017800030037001100fb006fb29700f1
:101af000e44878008301e9008100e9000300e00088
:101b0000f9ff3d00ffb29700550890000000e0008b
:101b1000f3003d000e00e900d00a9800f000370005
:101b20007f9497008f9c97001f9d9700af9d970013
:101b30006022b8006033b8000800be000a01be0091
:101b40005c0707000000e00005003d000bf0a2006c
:101b5000f8979f00899f9f009a9f9f00ab9f9f00cf
:101b60006f909700725927000280b900026a28001e
:101b70001300200040060700e4005000e1979f009a
:101b800015003b00e3801000c0ff2f0000846000c0
:101b90000800ea00e0979f007f9097008f989700d9
:101ba0001f999700af99970009e0200007003700c0
:101bb0000808a300030032003902be002903be005a
:101bc000770707000884d100e88444000800e0009b
:101bd000f7ff3c001b0037000100e0001d0034004f
:101be000c0ff2f0000806000e0979f000004780095
:101bf0006000b8000200200003ff230009e020007d
:101c0000070037000808a300030032003902be00b5
:101c10002903be00620707000884d100e88444005d
:101c20000800e000f7ff3c000002be000203be0017
:101c30007f9097008f9897001f999700af99970012
:101c4000cc070700f0979f00819f9f00929f9f0005
:101c5000a39f9f00ffb097005109900060c6b3009a
:101c60008ff1970080cf5100040032006100200006
:101c700060c4b30080cf510002003a006f92970019
:101c8000ea00420001074100f30f57000100340051
:101c90003e01200000c3b300e0779f0075fb2f00da
:101ca0008f824200b5b79f00330037000800be00a6
:101cb0000a01be00040707000006be0068075700bf
:101cc0004240a9000e0034002b0707000002be00ae
:101cd0000203be000800be000a01be00290707007b
:101ce0006022b80046782d00771924002c070700e1
:101cf000f0979f00819f9f00929f9f00a39f9f004e
:101d00003fb0970068044000890020000d003700b4
:101d1000a4002000050020000c01be00e0fd2f0003
:101d20000f004000fa0207007fa897008fb09700cd
:101d30001fb19700afb1970004c3b3000464410022
:101d40000006be00e00f5600e08f5e000600340083
:101d50008904e900e18f4400edff3a0002003700fa
:101d600000c3b300006478008904e900fcff3b0075
:101d700068044400b8b79f000e00e0000b00340078
:101d80007f9497008f9c97001f9d9700af9d9700b1
:101d90006022b8006033b8000800be000a01be002f
:101da000fa0607000000e000c0ff3c00c5fa2f0063
:101db0008f8242006a804200bfb0970000805000ce
:101dc0008001e9006f919700e70041006b814200bc
:101dd000010037000201e80000c3b300924f100079
:101de000fcff320074fb2f000f0042008080400097
:101df000828050000080410002025000e1979f0065
:101e0000ffb29700d509900060c6b3008ff297002b
:101e100080cf52000300320060c4b30080cf520074
:101e200002003a008100e8000a00370050c6b30003
:101e30008ff0970080cf5000050032008000eb004b
:101e400050c4b3008ff2970080cf520001003a00d7
:101e500011002000018741008e0f520001003d005b
:101e6000040778000e00e0001d003500840f5700c5
:101e700005003d00e2407f0095c3b30040c3b300be
:101e800080cf500001003c0005c3b3000e004100ac
:101e90008000e9008e017800010037008100e90030
:101ea0008301e90011427800854f5200fbff3200a8
:101eb0000307e80090c3b30080cf520001003a004e
:101ec0008448e8000300e00005003d000201e9004d
:101ed0000e07e8006f9097000000e800e0979f0071
:101ee0006f9297008e0178008ff097007fb0970077
:101ef000a40207004f0778004f06be004f05be0042
:101f00004f04be008f04b100000006002f03b00094
:101f1000889fbe008a9fbe008c9fbe008e1f7800e7
:101f200000077800b0e82000c0b79f0080c5b3006c
:101f300080cf500008003200a2e72000c2b79f0007
:101f40007740400080cf500003003a00830020001b
:101f5000b3b79f000a00370080c7b30080cf50009e
:101f600005003200a4002000b4b79f0080c5b30074
:101f700080cf500002003a0005012000b5b79f0055
:101f80003e04be002e05be0040c6b30080cf500008
:101f9000030032006540400080cf50000b003a0043
:101fa000e00f5400e08f5c00e00f5d00e08f5d000b
:101fb00006003d006000b8006011b8000804500041
:101fc000898458000a0559008b8559003fb1970054
:101fd000e80f510003003200f00f510045003a00b5
:101fe000020037003c002000010037004c002000b8
:101ff000e00f5400e08f5c00e00f5d00e08f5d00bb
:1020000005003a005e08900083012000a3b79f00fe
:102010000000e000080032003fb297000400e90031
:1020200008006000cfb297006540780090df9f0005
:1020300070012000a0b79f008c0078008100e900ab
:10204000050033008b05d1000a85d3008984d300b5
:102050000884d300f9ff3700089fbe000a97be002e
:102060002fb197000200e90023fc2f008f8141006f
:1020700000844100140037002fb097000000e900f1
:10208000a0b79f003fb197000200e9000400600084
:10209000cfb19700635478003e00be002e01be0011
:1020a0000c0278000402e900050033008381d100ae
:1020b0000281d3008180d3000080d300f9ff370074
:1020c000009fbe000297be003e02be002e03be006f
:1020d000e00f5200e08f5a00e00f5b00e08f5b00e2
:1020e000da0034002fb097000000e000e2ff3c006f
:1020f000d6003700ae60900080c6b30080cf50009d
:102100000b00320006003c000104e0000800320031
:102110006640500080cf500073003a000400370042
:10212000c0c6b30080cf50006f003a0031003700c6
:10213000080178000800e00005003a005e08900001
:1021400081012000a1b79f000000e00009003200db
:10215000bfb19700110009000381d8008000fd0085
:102160004fb297006440780090df9f007501200017
:10217000a5b79f003fb29700110009000481d80065
:1021800080017800afb297000500e90021fc2f0024
:102190008f804000008240000c003700bfb29700e3
:1021a000110009008501d800000178002fb09700c8
:1021b0000000e900a0b79f000590b9000080510021
:1021c000cfb0970061527800820178000300e000f0
:1021d000030034002fb197000200e000efff3c0045
:1021e00003007800cf80de000101780082017800d2
:1021f0003a0037000806be00e00f5400e08f5c0094
:1022000005003a005e08900083012000a3b79f00fc
:102210000000e000090032003fb297006121b900e0
:102220000c00be00ad060700cfb2970065407800f5
:1022300090df9f0070012000a0b79f003fb2970081
:102240006121b9000c00be00560507000006be0063
:10225000afb297000500e90021fc2f008f804000fd
:102260008080400091b79f00110037003fb1970078
:102270006114b9000801be000c00be007e04070016
:102280000005be00afb197008301e900a3b79f002e
:102290000801be00b1030700000056001fb29700fe
:1022a000cfb297006552780094b79f000a06be002f
:1022b000e00f5600e08f5e00030034002fb097005f
:1022c0000000e000e9ff3c004feade00cfa2de00a4
:1022d0000c00be000401780084017800009fbe005d
:1022e0000297be0059003700e00f5400e08f5c00f9
:1022f000e00f5d00e08f5d0005003a005e08900091
:1023000081012000a1b79f000000e0000d00320015
:102310003fb1970002027800cfa2de0005037800eb
:10232000860378000800be000a01be00ef06070021
:102330004fb297006440780090df9f007501200045
:10234000a5b79f003fb1970002027800cfa2de0040
:1023500005037800860378000800be000a01be006d
:10236000db060700009fbe000297be00afb19700da
:102370000300e90024fc2f000f0242000006420087
:1023800024003700bfb2970005047800cfc4de00f8
:10239000090578008a0578000802be000a03be001d
:1023a0005fa89700efa897007fa997008fb19700cb
:1023b000d2060700d0b79f00e1b79f00f2b79f0099
:1023c00083bf9f002fb097000000e900a0b79f00d7
:1023d0000802be000a03be005fb09700efb097008e
:1023e0007fb197008fb997004a0707005faa97004f
:1023f00000005200cfb29700655678005fb097009a
:10240000efb097007fb197008fb99700009fbe0093
:102410000297be003e00be002e01be00d0af9f005e
:10242000e1af9f00f2af9f0083b79f00e00f500025
:10243000e08f5800e00f5900e08f5900030034008e
:10244000afb097000100e000ceff3c003fb1970025
:10245000e80f510013003a000e1090000038a3005e
:1024600010003200afb19700f78f510006003e0018
:1024700024fc2f000f0242008300420000c3b3007f
:10248000914f100007003200afb297008502e900bb
:10249000a5b79f0000c3b30021fc2f008f80400030
:1024a00080f07a00afb1970078811100120f980088
:1024b0006e00900024fc2f000f02420083004200b7
:1024c000d9f807001e0990005e089000800f5100a7
:1024d00006003d0002005000000f98000e10900012
:1024e0000040a100001798000f0037000000e00036
:1024f0000d003d000e10900074006000f00f5000c1
:1025000009003a007e089000fe0090000100500093
:102510008e08900001005000020050004240a900c7
:1025200001003400000f98004f0778004f06be00ee
:102530004f05be004f04be002f03b100000006008f
:1025400080007800010037000000e8001004e0007f
:10255000fdff3a0001005000000006000000e0000e
:1025600003003400d8020700e10f400001003a00e8
:102570000000eb00000006000000e0003100320027
:102580008080e90091027800e38f52002d00360030
:102590000508a3002b003a00d27580000200e0007d
:1025a00002003200828f50000400310002087800df
:1025b000d175880016003700030178009201900061
:1025c0000300e00002003200818f5100faff390061
:1025d0001202780004004100808f50001900390079
:1025e000810f500003003a00050942008200780084
:1025f000070037000300e0000300320005804000c0
:10260000808f51000f00390093009800110198004d
:10261000110190000200e0000a0032001180400029
:10262000820f500007003a0080eb20000008eb000a
:1026300011009000110178009008410010009000f6
:1026400090009800000006000001780000002000c3
:102650000000e00008003200000080000000e00000
:10266000050032000000e900000088000000400082
:102670000100800002b0780000000600889fbe00c4
:10268000800478006684400000ff27001800600086
:102690004401de00f07f2000800f51000e003a0060
:1026a000800ceb00180478006f0064001c003a00f6
:1026b000210090000000e00019003a001100900095
:1026c0000000e00016003a00100020001100e000b9
:1026d00014003200120037000200e00005003c0048
:1026e00001007800db010700000178000000e00035
:1026f00008003c00f00028001800600001fe2300e4
:10270000010c700020c02f00800c41000080eb0005
:1027100004003700800ceb000000eb0001003700e4
:10272000200020004f04be0000000600889fbe006d
:102730008a1f78008c9fbe00000478000206be004d
:10274000e6044000190178000200d0004505de00d3
:102750008a007800f07f2000800f55000c003a00be
:102760006f00610065003a00280090000000e00062
:1027700062003a00180090000000e0005f003a009c
:10278000100020001800e0005d0032005b00370000
:102790000a00e00007003a0008007800ad010700d9
:1027a000800078000000e000020034000a00780099
:1027b000530037006108b9000c0140008d814800ca
:1027c000e07f2000800f5100e08f59000d003400a1
:1027d0001900e00004003d006000b8000200200085
:1027e00003ff2f00030037006000b8000200200044
:1027f00003ff2700009cbe000294be0010002000d2
:102800003f003700e00f5100e08f59000500340011
:10281000f000280019006000c410dd00810c700079
:10282000340037001900780001002800010360001f
:102830006f0060000040a000800c78006101510032
:10284000e0815900c0fc2f00f1ff2f00800f5100e4
:10285000818f59000d003d00860c78000000eb00d0
:102860002004980010049800000c78002400370021
:102870008880e800110c780064004400900878001b
:1028800019087800800ceb0070014100f00f410046
:10289000f7ff34008202ea00150032008881e80068
:1028a00070821200980078008508de00130078001e
:1028b0000400dd00008c7000640144009300780087
:1028c0008508de00120078000400dd0080897000b9
:1028d000920078008508de00190078000400dd0011
:1028e00000897000190078000500de00800c780077
:1028f000990c73000080eb000100370020002000dd
:102900004f06be004f0578004f04be0000000600d1
:102910000400fa00889fbe008a9fbe008c1f7800ca
:102920000006780092bf9f00a3bf9f000404be0072
:102930000401be001fb89700afb89700ce02070091
:102940000005be000001be000800be000302070033
:102950001fb99700afb9970000005100818059005e
:1029600020069800310698000a8ebe000c00780000
:102970004f0678004f05be004f04be000080fa00ed
:10298000000006000e00fa00889fbe008a9fbe006d
:102990008c9fbe0000047800014578000206780094
:1029a00083047800840678000300e00002003c0005
:1029b000190020002cec200060c6b300804f5500a9
:1029c0000e00320060c4b300804f55000b0032008f
:1029d00070c6b300804f55000300320070c4b300ce
:1029e000804f55009c003a00e48f4600800035007f
:1029f00058089000808f56007d003d008d05e8004e
:102a000060c6b300804f55001000320060c4b300b0
:102a1000804f55000d003200081090000038a300d0
:102a200004003a0058089000808f540001003d00d7
:102a3000590c9800580890000b005000500c98005a
:102a400002003b000000eb00500c98000b00e0007f
:102a500027003c00180990006800900001c3b300f3
:102a6000017079008201e800130c9800580890006a
:102a70000000e00003003c00081090000038a300b4
:102a80000500320068009000e1c2b30001f0790057
:102a90000280e800100c9800d80890000b00ea00b3
:102aa000808f500001003d008105ea000b00ea0024
:102ab000200c980001804500500c9800890f5000b0
:102ac00001003d0080047800390c980068009000f7
:102ad0009808900001004000090178008c007800ff
:102ae00051f7070058089000090050001a003700fd
:102af00098089000680090008b8f540018003d00eb
:102b000001004000090178008c00780046f70700ba
:102b10001808900000814400120c980009805500ac
:102b2000200c9800580890000000e00003003c00d2
:102b3000081090000038a30006003200e800900062
:102b4000e0c2b30080707900380890000000e8000f
:102b5000300c980058089000400c9800a6003700f0
:102b6000010040000b0178008c0078002ef7070070
:102b70001808900000814500120c98008b845400c6
:102b8000580890000000e00003003c00081090008e
:102b90000038a3000500320068009000e1c2b300d5
:102ba000017079000200e800100c980058089000ad
:102bb000890f500001003d008004780068009000fb
:102bc00098089000010040008b0046000901780041
:102bd00015f707001808900000804400100c9800ba
:102be0005808900009005000200c9800820037001f
:102bf00070c6b300804f55000300320070c4b300ac
:102c0000804f550014003a0058089000808f5400ff
:102c100004003d00081090000038a30001003a00b5
:102c2000590c9800580890000000e900500c9800da
:102c300002003b000000eb00500c980070c6b3008f
:102c4000804f550002003a005ac6b3000b0037000f
:102c50005ac4b3000900370010c6b300804f5500b6
:102c600002003a000ac7b3000400370010c4b300e2
:102c7000804f550001003a000ac5b30018099000c2
:102c8000680090003c7079008201e800130c980005
:102c90000c027800580890000000e00003003c009f
:102ca000081090000038a30017003200e8009000e0
:102cb000e0c2b30080f079008280e800110c980037
:102cc000580890000000e0000f0034008904e9007b
:102cd000890f500001003d008004780068009000da
:102ce000008040000901780084007800cef60700db
:102cf0001808900000804400100c980058089000bc
:102d000009005000200c980068009000980890007e
:102d1000010040000086e8000a5878008000780032
:102d20000d00e00004003500b0c2b3008048780018
:102d30008c04780004003700d0c2b30080487800cb
:102d40008c0478008d06ea008005eb000a0037004d
:102d5000a20020008d0078007080570089000700d5
:102d60000fb897009fb897007a81550001f17f0056
:102d70008b05e800800678000d00e000f4ff3c00c1
:102d8000e18f550009003c0050c6b300804f55004c
:102d90000300320050c4b300804f550003003a00d6
:102da00000c3b300005e78008c0478000b00e000e4
:102db000040032000b00e900fa8057000080400058
:102dc0000600370000c3b300805c780005003700c0
:102dd0008b05e90002c3b300a05c41000b00e000da
:102de000fbff3c0068009000980890000100400044
:102df00000805400300c98000810900074006000af
:102e0000f00f50000e003a007800900098089000f3
:102e100001004000a808900001004000b8089000a0
:102e200001004000c8089000810040007808900030
:102e3000808f500002003d0001005000000c9800ff
:102e40004f06be004f05be004f04be000080fa00d2
:102e50000000060000027800e6024000150078003d
:102e600001002800810360006f006000800a780084
:102e700012003a00240090000000e0000f003a0029
:102e8000140090000000e0000c003a001600200042
:102e90001400e0003800320008003700e40042006f
:102ea000910a78000480e8009008780014087800ff
:102eb000000aeb00700353000100370016002000e9
:102ec0001500e000f5ff32001300370064014200f6
:102ed00080004000120078004f00de00808a700001
:102ee0008481e8009200780081804000130078001f
:102ef0004f00de0000897000930078008180400060
:102f0000140078004f00de00808970001400780003
:102f1000000a40000603e90015007800ef0f50009a
:102f2000eaff3600100037000481e8009400d10069
:102f3000120078004f00dd00008a7000e4004200bb
:102f40009201d100110078004f00dd00008971006e
:102f50001101d100150078004f00dd0080087100dc
:102f6000950ad1000603e80015007800ff0f500015
:102f7000edff3e00ef0a6000958a730006007800be
:102f80000000060002027800809fbe0011000900c8
:102f90008200d800000178004f00be0002a2b900f4
:102fa000848050001100980002087800000006009c
:102fb0000a00fa0080017800e20f500025003e0070
:102fc000e0758000e10f500008003200e021200091
:102fd0000000e0000500320064212000852120006f
:102fe000a62120008001780004003700c4202000c2
:102ff000e5202000062120004321200014409000fd
:103000000004e000030035008009eb000000280008
:10301000140a7000154090000028a30001003a0037
:1030200015a0a0008001eb000700370015409000bc
:103030000008a300fdff320063c078000000fb0021
:10304000000b78008301e800828f5100f7ff3a00ff
:103050000800370030002000b0bf9f00c3bf9f00b2
:10306000d1bf9f00e2bf9f006a80570000c0da0016
:103070006fb99700020078000080fa000000060097
:103080000a00fa0011002000b1bf9f00c0bf9f00de
:103090006a80570000c0da004fb897000080fa003d
:1030a000000006000a00fa0051002000b1bf9f0096
:1030b000c0bf9f006a80570000c0da005fb8970069
:1030c0000080fa0000000600889fbe00800478009f
:1030d000307680000000e00003003a001000070096
:1030e0000000e0000a003500307680000900e000b2
:1030f00002003a000004780006003700000478005f
:1031000009004000060007000000e00001003d004b
:103110000084eb00080078004f04be0000000600a9
:10312000800078000000e00004003a0080ec2000fd
:103130003076880001017800060037000081eb003e
:10314000c00b2100808f500002003e0031768800c5
:103150000001eb000200780000000600020ab9003e
:10316000001bb9000200b80081004200810043004a
:103170000000060003f0a200889fbe008a9fbe00e8
:103180008c1f78002e010700350133006450e100e8
:103190004f0032006420e1005200320003826c00d4
:1031a00007003b000905d0000306d000820f540041
:1031b0000c065d000200390002003200890178002f
:1031c000030678008582550004003d000003fd00e1
:1031d0008103fd008502ea008b854200840f7200a6
:1031e00002003b0060001000e08018006011b80091
:1031f0000005eb007a28e1000a003900060078009b
:10320000c75ddd00f707b200878075002d0037002d
:10321000828171000a017800610560008180d1001f
:103220000080d3008502e900f9ff3b00060440005e
:103230008784480002003b0060041400e0841c0006
:103240000988a300070032008a8171008281710021
:10325000610164008904d1000884d3008b05e80073
:10326000170037000978a30013003a000b00e000b4
:10327000130034008b05e9000804440089844c00e5
:103280000a4474000978a3000d003a000b00e00026
:10329000070034008b05e9000804440089844c00d1
:1032a00001003a000b0020000978a300f7ff32006c
:1032b0000001eb0002003700828171000a017800f2
:1032c000f70007000cf0a70001f0a000ed003700a8
:1032d0006420e10002003a00838f6c00ed003300af
:1032e0000801be000200be00e6003700889fbe0055
:1032f0008a9fbe008c1f7800d1000700d8003300e1
:1033000003866c006450e100240032006420e10078
:10331000270032006150e100220032006120e1000c
:10332000210032008b854200eb07b1000134b80068
:10333000003ab8000804420089844a00013ab80003
:103340000030b8008880400009014a0004003300c2
:103350000000400081804800020149008b05e9001f
:10336000c909dd0083017000010032001300200054
:10337000c814de004814dd004709de001200b20068
:10338000c808de0008847000c500070001f0a10035
:103390000cf0a70001f0a000ba0037006120e100a6
:1033a000bc0032000801be000200be00f7ff37007b
:1033b0006150e100fcff3a00b6003700f4ff2f0037
:1033c000dd003700889fbe008a9fbe00010578009f
:1033d0000100e0000400350008003c000000e000af
:1033e000200032000500370060001000e080180067
:1033f00002003b0001f02c001a0037000004be0060
:103400006011b8006b0920000982cf00020039006a
:103410000882cf000441b000694252000e00320021
:1034200008003b0082817100610164008904d100c1
:103430000884d3008b05e8000442e800f9ff3a0055
:10344000050037000804440089844c008b05e9001e
:103450000442e900fbff3a00910007000af0a700d0
:1034600001f0a0004f05be004f04be0000000600a2
:1034700014002000b0003700839f68000100e000c6
:1034800002003d0060001000e08018000300e00032
:1034900002003d0060011100e0811900c100070039
:1034a0004f00e00002003b0060001000e0801800c8
:1034b00000000600889fbe008a9fbe008c1f780017
:1034c0005f0007006600330003866c006450e10073
:1034d0002e0032006420e100330032006150e10030
:1034e0002f0032006120e100310032008585550057
:1034f000eb07b00009002000080420000500370099
:103500000804440089844c000a003100060343008b
:1035100087834b000001530081815b00f8ff33007b
:103520000203be000800a0000804440089844c0087
:10353000f6ff3900c639dd00830173000100320057
:10354000130020008904d1000884d3000998a30047
:10355000050032000800a7000300a0008904d10084
:103560000884d3008b05e8008904d1000884d300c7
:103570000001eb000281d2004900070001f0a10028
:103580000cf0a70001f0a0003e0037006420e1002d
:10359000400032000801be000200be00f7ff370005
:1035a0006120e1003b0032006000b800f3ff37000b
:1035b0000000200001f82700f0ff37000001be00e6
:1035c000880007000470a70003f0a1006509b1009e
:1035d000160032000d0035006828e10006003500b5
:1035e000f0ff2f00f1ff27000300e00013003b0075
:1035f0000100280000000500000040008180480014
:103600008502e900fcff3a0008003700f88f42000d
:1036100002003c008000eb00000005008100d100aa
:103620000080d3008502e800fcff3a000300e000c0
:1036300002003b0060001000e0801800000006005f
:103640000004be00670007000003be000405be00c2
:103650000200be0063000700844f750000000600f2
:103660000200be006450e100050036006420e10065
:10367000020036000968a30001003a000800be00fd
:103680000160a0004f0678004f05be004f04be0049
:1036900000000600f0ff2f00f1ff2700f9ff3700c0
:1036a00081002000618055000b003d000b002000d0
:1036b00061fe2f000100e1001d00340082817100d5
:1036c000610164008904d1000884d3000000e8008f
:1036d000faff3a00710020006100640003007000ee
:1036e000020060000900320061044400e0844c00e4
:1036f0000988a500050032008b05e8006808e10094
:1037000002003a008904d1000884d300f20f20009f
:103710000258e10005003d00c75ddd00f907b20079
:103720008980750008007800000006000bf827006b
:103730008b00780000000500889fbe008a9fbe00b5
:10374000841f7800beff07004f007800110033008f
:10375000f0ff2f00838f6c0006003b00040565001e
:103760000a00a7000800370009f0a600100020009a
:1037700008003700820f5400838f5c00030039007b
:103780001000200001003e000000200009f0a7000a
:103790000000ea004f05be004f04be000000e0003c
:1037a000000006006022b800060220000000d000e1
:1037b0008180d2000482d2008582d2000000a00065
:1037c0000202520083825a000300310002024200ca
:1037d00083824a000000a1000603e900f3ff3a00db
:1037e00000000600c70ade00f107b200f50fb200c4
:1037f00008003200e1cf4200020032000170a00058
:1038000024000500810f700001003200040805004b
:1038100044000500810f700002003a00140005000a
:103820008502e9000000400081c04800fcff3b0029
:103830000170a0002400050081037800e9ff070063
:103840000001be006000b8000478a30013003a0035
:103850006220e10015003e000d0039008301d10017
:103860000281d3008180d3008301d1000281d30083
:103870008180d3008301d1000281d3008180d300f5
:103880000538b000c42add00f300b2008381720065
:1038900007f0a70003f0a00000000600f3ff2700d8
:1038a000f2ff2f006110b900fbff370003ff270074
:1038b000f7ff37008f1fd100440207008f87e90010
:1038c0000000e000000006001400fa00889fbe001f
:1038d0008a9fbe008c9fbe000004be000205be0091
:1038e000680047000a90be000890be006002070012
:1038f0000070a7000bf0a100304320009e02900052
:1039000080825200b0fe2f000028e10011003d002f
:10391000b0fc2f000028e100150034001e099000c3
:103920008e0890007e0090000501b0000201d100d9
:103930008180d3000080d3008502e800fbff3a00bd
:103940000b00e00085023b0060001000e0801800e2
:1039500082023700f0ff2f00f1ff27000b00e0008c
:103960007e023b0001002800000020007b0237009f
:103970006000b800790237004f89de0082017800cc
:103980007b02370007f0a200b0023700809feb00f7
:103990000e0207008f87e9000000e000000006002b
:1039a0002800fa00889fbe008a9fbe008c9fbe0040
:1039b00003866b00550207000028a30064003a004c
:1039c0000128a30067003a000008a30062003a0043
:1039d0000108a30065003a001e009000be08900098
:1039e00081064000ed3fb100f4805700ee019000e9
:1039f000111ab8008e099000311bb8009e09900082
:103a0000311cb800511db800f4855700460007006e
:103a1000fe0190003a0007008b85e8003e00070099
:103a20008e09900040000700ee019000340007006e
:103a30008b85e800380007008e09900040000700e1
:103a40009e0990001b18b800890440000a854800b0
:103a5000fe019000340007008b85e8003800070065
:103a6000ee019000300007008e0990001b18b8008e
:103a7000890440000a8548000a98a30008003a001b
:103a80000402420085824a0006034b0087834b00f4
:103a900008044c0089844c000a054d008d06e9009d
:103aa00084827200850273004c3add008502720048
:103ab0000100320015002000443ade001400b2007c
:103ac0004538de00cb45dd000b007000c540de0050
:103ad000cb4ddd008b8070004549de00cb55dd000d
:103ae0000b017100c551de000d037800d402070000
:103af00003f0a1000cf0a70003f0a00017023700ac
:103b00001b18b8008502400006834800e0834b0084
:103b100060044c00070037001b18b8000603400083
:103b200087834800faff37001b18b800870340005e
:103b300008844800e0844c0060054d000000060049
:103b40001b18b8000804400089844800faff3700b9
:103b50000108a300fe013a005800be005801be0053
:103b6000e3ff37000008a300f9013a0009047800d8
:103b7000f9ff37002800fa00889fbe008a9fbe0028
:103b80008c9fbe0003866b00e00107006400e1002b
:103b9000440032006408e1004a0032006100e100a4
:103ba000460032006108e10049003200ec0647009f
:103bb0006000b8003d02be003d03be00f486570021
:103bc0006011b8003d04be003d05be007d0320002d
:103bd0000b0037000000a0008d06e9001300320042
:103be0000402420085824a0006034b0087834b0093
:103bf00000004000818048000201490083814900a3
:103c00000802520089825a000a035b008b835b0022
:103c1000f0ff3b000802420089824a000a034b0081
:103c20008b834b008d06e900edff3a008482720021
:103c300086827200f707b2008782720001003200ac
:103c4000150020001e0490003e0b90000603540057
:103c5000e63fb0000368a300070032000000a700a1
:103c60000500a0008301d1000281d3008180d30030
:103c70000080d3000603e8008301d1000281d30055
:103c80008180d3000080d3000002eb000482d200c8
:103c90006b02070003f0a1000cf0a70003f0a000e6
:103ca000ae013700640247006408e100a801320059
:103cb0003400be003401be00f6ff37006108e100a9
:103cc000a30132006011b8006000b800f1ff3700b6
:103cd00003ff270002002000fbff3700b1fe0700b2
:103ce0000400be0000000600881f78000004780071
:103cf0005001be004000be00040040008580480026
:103d00000601490087814900009cbe000294be0064
:103d10000400e1000588e1000690e1000798e10059
:103d200002003100680044001008e8004f047800e9
:103d300000000600f4874700889fbe008a9fbe00ef
:103d40008c9fbe008e1f78000205be000004be00de
:103d5000d4b79f00e5b79f00f6b79f0087bf9f00cd
:103d60000000eb00c0b79f00b0b79f00a0b79f0056
:103d700090b79f0080b79f000d042000bfb0970050
:103d80004fb09700000140000000e0000f003d0030
:103d90004f08de0000007100c0b79f009e000700c2
:103da00001003d0012002000a100070001003d00bd
:103db00012002000a6000700b1000700b6000700af
:103dc0000f004000c8ff0700220037004f08de0048
:103dd00000067100ccb79f008f00070001003d0076
:103de000120020009200070001003d001200200098
:103df00097000700a20007000fb297009fb297003c
:103e00002fb39700bfb39700a9000700000052002e
:103e100081805a0002015b0083815b0080b79f00b4
:103e200091b79f00a2b79f00b3b79f000007eb00b8
:103e30009f0007000020e10001a8e10002b0e100be
:103e400003b8e100010031001e0020000e00560002
:103e5000c0b79f004fb297000400e0000700350094
:103e600010002000010020006011b800080470005c
:103e7000898470000a0571008b8571008d06e90048
:103e8000beff3a000400e00003003d00820007008e
:103e90000f00400094ff07004fa897000000e000cb
:103ea00004003a000fb497009fb497002fb5970015
:103eb000bfb59700940007004f0778004f06be007b
:103ec0004f05be004f04be004f01b10000000600c8
:103ed000881f780018002000881f780095ff0700d1
:103ee0008f87e9004f04780000000600801feb0078
:103ef00090ff07008f87e90000000600889fbe0042
:103f00008a9fbe008c1f78006e00070007003d00ee
:103f100073000700e00f5b00e08f5b0007003d00cf
:103f2000320007000006eb000400370034000700f1
:103f300002003d002a0007001c002000720007005c
:103f4000e3ff07000203be000002be000c00e00019
:103f500001003200220007000400be000601be007e
:103f60004f0678004f05be004f04be00000006005b
:103f7000889fbe008a9fbe008c1f780051000700fa
:103f800005003d0056000700e00f5b00e08f5b007e
:103f900006003d00040037001900070003003d0043
:103fa0006000b8006011b80010000700560007005c
:103fb000ceff07000203be000002be000c00e000be
:103fc00001003200060007000400be000601be002a
:103fd0004f0678004f05be004f04be0000000600eb
:103fe0006000b8006011b800000037000402500003
:103ff0008582580006035900878359000000060097
:104000000006eb00e00f5200e08f5a00e00f5b006b
:10401000e08f5b00000006000180400090b79f0029
:104020000001eb008fb097000100e00000000600e7
:104030000200700090b79f000180400080b79f0091
:104040000001eb00ffa897000100e000000006005f
:104050000200700080b79f00018040006faa9700a7
:10406000cf20de0001007000f0af9f00040242008c
:10407000250007004f18de00000272000000060055
:10408000e4af9f000804440089844c000a054d00f9
:104090008b854d00000006003fb29700cfb297001d
:1040a0005fb39700efb3970000fe2f0000000600fb
:1040b0003fb09700cfb097005fb19700efb1970086
:1040c000000006000205be000004be00e00f500024
:1040d000e08f5800e00f5900e08f59000000060003
:1040e0006000b8006011b8000804500089845800ce
:1040f0000a0559008b8559001c002000e00f520072
:10410000e08f5a00000006000800be000a01be0051
:1041100000000600889fbe008a9fbe008c1f7800aa
:104120000205be000004be000006eb00e00f5000d8
:10413000e08f5800e00f5900e08f590007003d0064
:104140006000b8006011b80008045000898458006d
:104150000a0559008b8559001c002000e00f520011
:10416000e08f5a00e00f5b00e08f5b0002003d0033
:104170000f0007000c00a2000800be000a01be00ec
:104180005b0107000203be000002be000c00e0005d
:1041900001003200060007000400be000601be0058
:1041a0004f0678004f05be004f04be000000060019
:1041b0006000b8006011b800040250008582580009
:1041c000060359008783590000000600889fbe003f
:1041d0008a9fbe008c9fbe000404be000605be0080
:1041e000809fbe00829fbe00630107000406780026
:1041f0000800be000a01be005f01070084067800c7
:104200004f03be004f02be008d4f76007fb0970077
:1042100013003300f0ff2f008b8f6b0006003b0074
:104220000d0666000c00a7000a00370007f0a60084
:10423000100020000a003700880f5200898f5a00b2
:104240008a0f5b008b8f5b00030039001000200099
:1042500001003e000000200007f0a7000000ea0077
:104260004f06be004f05be004f04be000000060012
:10427000800078005002be005003be004439de00ca
:10428000f700b200f37f2000030161000900320053
:104290000218e10016003a008501720083017300e4
:1042a000838173000008200015003a0040002000c0
:1042b000130037008501720083017300838173004e
:1042c00005003a0004a8be0006a8be0010002000a9
:1042d0000b0037000201e9000402420085824a0017
:1042e00006034b0087834b000748a300f9ff320009
:1042f0000740a00004a8be0006a8be0020002000c1
:1043000080009800920098000000060068044700b2
:104310000294be000094be00fc0447008694be00d8
:104320008494be0009007800d1ff070008007800df
:10433000cfff070099007800814f70000b003b0011
:104340000800be001e0107004f00b1000300370047
:10435000f3ff2700f2ff2f006110b9004f06be00e7
:104360004f05be004f04be000080fa0000000600aa
:10437000889fbe00830478000300e0002c00350015
:1043800003003c000082700004027100260032002d
:1043900036432000c50020008383cf000a00390087
:1043a0000541b1008283cf00070039000541b1000b
:1043b0008183cf00040039000541b1008083cf0024
:1043c000010039000541b10085c353006022b800e7
:1043d000120032000a003b00848272006102600019
:1043e0008301d1000281d3008180d3000080d300fb
:1043f0000603e8008743e800f7ff3a0007003700ac
:10440000000040008180480002014900838149008a
:104410000603e9008743e900f9ff3a008800070036
:1044200009f0a70003f0a0004f04be000000060042
:1044300060001000e080180060011900e0811900a0
:10444000d3ff3b00033e2c00f7ff37002800fa00a3
:10445000889fbe008a9fbe008c9fbe000706780022
:10446000878669000c003b0003047800870478000d
:1044700008f0a10009f0a100840f5000858f5800ba
:10448000860f5900890f5c00030033000cf0a20076
:1044900001003a000cf0a1009cff07006400e1005d
:1044a0005f003200780147006408e10061003200db
:1044b0006c014700748557003200be001201be0037
:1044c0003a04be001a05be001e039000be0a90000a
:1044d0008503530006003d000004fd008104fd003b
:1044e0000205fd008305fd008703ea00050378004f
:1044f0000df8a3000400320060041400e0841c00e6
:1045000060051d00e0851d006022b8007d032000cd
:104510000d38e1008006eb000b0039004433dd006c
:10452000f300b20083017300390037008482720007
:104530000d027800e10664008b85d1000a85d30066
:104540008984d3000884d3008703e900f7ff3b0088
:1045500008004000898048000a0149008b81490019
:1045600004003b0060001000e080180060011900aa
:10457000e08119000358a300090032008d82720007
:1045800084827200610260008301d1000281d30045
:104590008180d3000080d3000603e8001b003700b1
:1045a0000348a30017003a000600e000170034009b
:1045b0000603e9000d00a3000000480081804800c8
:1045c00002014900838149000348a3000f003a001b
:1045d0000600e000090034000603e9000000400086
:1045e00081804800020149008381490001003a00ae
:1045f0000003eb000348a300f5ff32006022b8007f
:104600000200370084827200618266000c0007009d
:1046100003f0a1000cf0a70003f0a0004fff37004b
:10462000640147006408e10002003a000df8a300ad
:1046300047ff3a003200be001201be0047ff3700bc
:104640001800200057002000080453000d003d0012
:104650000600200097fc2f000740e1001e003400f8
:1046600084827200610260008301d1000281d30064
:104670008180d3000080d3000804e800f8ff3a00ee
:104680004700200061046000050474000404640015
:104690000d00320061004000e080480060014900e8
:1046a000e081490003b8a500070032000603e800d6
:1046b0006538e10004003a008301d1000281d30093
:1046c0008180d3000080d300f87f20000830e10013
:1046d00003003500080378006000b8006011b800de
:1046e0004433dd00f300b2008301730000000600d4
:1046f000889fbe008a9fbe008c9fbe000404b80045
:104700000506b8008904460060854e000606b8001c
:104710000a054600e0854e000706b8008b054600f6
:10472000040eb800890446000a854e00e0854d005d
:10473000050eb8000a0546008b854e00060eb8002f
:104740008b0546000416b8000a0546008b854e000e
:104750000516b8008b054600041eb8008b05460000
:104760000800be000a01be004f06be004f05be0095
:104770004f04be000000060005ff2700058261000f
:10478000070032000428e100010032002400050087
:104790000600070001003a00440005000408050077
:1047a00002000700f9ff3a00140005006f82610063
:1047b000810270008502710085027200000006000f
:1047c000e48240001078a300070032006402400039
:1047d0001178a3003400be001401be0004003200b2
:1047e0000330a700000006003500be001501be0022
:0847f0000330a00000000600e8
:020000040000fa
:0200000401f009
:04000000e5ff000018
:020000040000fa
:0200000401f009
:04000400ff7f00007a
:020000040000fa
:0200000401f009
:04000800ffff0000f6
:020000040000fa
:0200000401f009
:04000c00ffff0000f2
:020000040000fa
:0200000401f009
:04001000ffff0000ee
:020000040000fa
:0200000401f009
:04001400ffff0000ea
:020000040000fa
:100008007c870000048600003e86000038870000d8
:10001800628700007c8700007c8700007c870000e6
:100028007c8700007c8700007c8700007c870000bc
:100038007c8700007c870000ca770000ba7800003f
:100048007c870000188400007c8700007c87000003
:100058007c8700007c8700007c8700007c8700008c
:100068007c8700007c8700007c8700007c8700007c
:100078007c8700007c8700007c8700007c8700006c
:10008800827d0000c67d00007c8700007c87000020
:100098007c8700007c8700007c8700007c8700004c
:1000a8007c8700007c8700007c8700007c8700003c
:1000b8007c8700007c8700007c8700007c8700002c
:1000c8007c8700007c8700007c8700007c8700001c
:1000d8007c8700007c8700007c8700007c8700000c
:1000e8007c8700007c8700007c8700007c870000fc
:0800f8007c8700007c870000fa
:020000040000fa
:100108007c870000048600003e86000038870000d7
:10011800628700007c8700007c8700007c870000e5
:100128007c8700007c8700007c8700007c870000bb
:100138007c8700007c870000ca770000ba7800003e
:100148007c870000188400007c8700007c87000002
:100158007c8700007c8700007c8700007c8700008b
:100168007c8700007c8700007c8700007c8700007b
:100178007c8700007c8700007c8700007c8700006b
:10018800827d0000c67d00007c8700007c8700001f
:100198007c8700007c8700007c8700007c8700004b
:1001a8007c8700007c8700007c8700007c8700003b
:1001b8007c8700007c8700007c8700007c8700002b
:1001c8007c8700007c8700007c8700007c8700001b
:1001d8007c8700007c8700007c8700007c8700000b
:1001e8007c8700007c8700007c8700007c870000fb
:0801f8007c8700007c870000f9
:020000040000fa
:1047f8000a0d00004a5500004d41000020500000fd
:1048080041310000303000003020000074650000a5
:104818007374000020260000206d0000616900000c
:104828006e740000656e0000616e00006365000034
:10483800206300006f6d00006d6100006e64000071
:10484800732d00002d2d00002d2d00002d2d0000b2
:104858002d2d00002d2d00002d2d00002d2d0000e8
:104868002d2d0000000a00000d49000020760000f0
:1048780065720000736900006f6e00002069000017
:104888006e6600006f0000000a0d00004420000062
:104898007365000074200000666100006374000006
:1048a8006f720000792000006465000066610000f6
:1048b800756c000074730000206900006e20000011
:1048c80075730000650000000a0d0000522000000a
:1048d80073650000742000006661000063740000c6
:1048e8006f72000079200000636100006c690000ad
:1048f8006272000061740000696f00006e200000a1
:10490800766100006c750000657300002069000086
:104918006e20000075730000650000000a0d00009d
:1049280046200000736500007420000063750000d5
:1049380072720000656e0000742000006361000060
:104948006c6900006272000061740000696f000009
:104958006e200000766100006c7500006573000031
:10496800207400006f20000066610000637400007e
:104978006f72000079200000636100006c6900001c
:104988006272000061740000696f00006e20000010
:10499800766100006c75000065730000000a000075
:1049a8000d430000206300006c6500006172000088
:1049b8002066000061630000746f000072790000d7
:1049c8002064000065660000617500006c740000da
:1049d80073200000736500007473000020630000fa
:1049e8006f7500006e7400006572000020260000dc
:1049f800204d00006f7200007175000065200000f6
:104a0800636c0000656100006e2000007570000096
:104a1800000a00000d410000206300006f6e0000d6
:104a280076650000727400002026000020700000e7
:104a3800726900006e7400002041000044430000c9
:104a480020760000616c00007565000073000000ae
:104a58000a0d000045200000647500006d7000001c
:104a68002045000045500000524f00004d20000036
:104a7800636f00006e740000656e00007400000033
:104a88000a0d00004d200000647500006d700000e4
:104a9800204d00006f720000717500006520000055
:104aa8006461000074610000000a00000d4a000003
:104ab800206a0000756d000070200000746f00000f
:104ac800204600006c610000736800002057000059
:104ad8007269000074650000720000000a0d000091
:104ae80053650000727600006963000065200000cd
:104af8007465000073740000732d00002d2d0000f4
:104b08002d2d00002d2d00002d2d00002d2d000035
:104b18002d2d00002d2d00002d2d00002d2d000025
:104b28002d2d00002d2d00002d2d00002d2d000015
:104b38002d2d00002d2d00002d2d00002d2d000005
:104b48002d2d00002d2d00002d2d00002d2d0000f5
:104b5800000a00000d57000020640000697300007f
:104b6800706c00006179000020740000657300001b
:104b7800742c000020770000726900007465000042
:104b8800204100005343000049490000000a00008a
:104b98000d7700002064000069730000706c00004d
:104ba800617900002074000065730000742c000017
:104bb800207700007269000074650000204800003a
:104bc80045580000000a00000d6c0000204c000051
:104bd800454400002062000061720000207400005b
:104be8006573000074200000776900007468000095
:104bf800204800004558000020760000616c000045
:104c080075650000000a00000d620000204c0000dd
:104c1800454400002062000061720000207400001a
:104c280065730000740000000a0d000042200000b7
:104c38005075000073680000204200007574000081
:104c4800746f00006e20000074650000737400002b
:104c5800000a00000d740000207300006f7500004a
:104c68006e64000020670000656e00006572000039
:104c7800617400006f72000020740000657300000a
:104c8800740000000a0d000070200000636f00002f
:104c98006f6c0000696e000067200000666100000c
:104ca8006e200000505700004d200000636f000088
:104cb8006e740000726f00006c20000074650000c4
:104cc80073740000000a00000d5a00002043000021
:104cd8005055000020650000727200006f720000dd
:104ce80020740000726100007020000074650000ec
:104cf80073740000000a00000d5300007065000086
:104d080063690000616c00002064000065620000b7
:104d180075670000206300006f6d00006d61000082
:104d28006e640000732d00002d2d00002d2d000055
:104d38002d2d00002d2d00002d2d00002d2d000003
:104d48002d2d00002d2d00002d2d00002d2d0000f3
:104d58002d2d00002d2d00002d2d00002d2d0000e3
:104d68002d2d00002d2d00002d0000000a0d000043
:104d780069200000496300006f6d0000207000008a
:104d8800726f0000746f0000636f00006c200000f9
:104d98007465000073740000730000000a0d0000c1
:104da8006b2000004b6500006e7700006f6f0000fd
:104db80064200000707200006f7400006f630000d0
:104dc8006f6c0000207400006573000074730000ad
:104dd800000a00000d3e0000000a00000d46000019
:104de800726f00006e74000020700000616e000099
:104df800656c0000207000007573000068200000da
:104e080062750000747400006f6e0000207400006a
:104e180065730000742e00002054000065720000c5
:104e28006d6900006e610000746500002074000068
:104e38006573000074200000686900007420000099
:104e4800616e0000792000006b65000079000000a9
:104e58002020000042750000747400006f6e00008e
:104e6800205400006573000074200000202000001a
:104e7800004e00006f2000005072000065730000b3
:104e8800736500006420000020200000202000003e
:104e98002000000047610000696e00002044000007
:104ea8006f7700006e200000202000002020000006
:104eb800202000000050000041470000452000006d
:104ec80020200000202000002020000020200000da
:104ed800202000002000000047610000696e0000eb
:104ee8002055000070200000202000002020000035
:104ef8002020000020200000004f00005045000046
:104f08005220000020200000202000002020000067
:104f18002020000020200000202000000042000087
:104f2800616e000064200000444f0000574e0000ee
:104f38002020000020200000202000002020000069
:104f480000410000555400004f20000020200000c0
:104f58002020000020200000202000002020000049
:104f68002020000000420000616e00006420000064
:104f780055500000202000002020000020200000c4
:104f88002020000020200000000a00000d4a000038
:104f9800756d000070200000746f00002050000044
:104fa800413100003030000030200000466c000025
:104fb800617300006865000072200000307800000e
:104fc800313700004430000036200000596f0000df
:104fd800752000006861000076650000203300003d
:104fe8003073000020740000696d00006520000027
:104ff800746f00002064000069730000636f000094
:105008006e6e000065630000740a00000d00000069
:1050180074650000726d0000696e0000616c00002c
:10502800206100006e6400002073000074610000bd
:1050380072740000206400007350000049430000af
:10504800626f00006f7400006c6f00006164000004
:10505800657200002e650000786500000a0d0000ea
:105068000057000061690000742000003330000020
:1050780073200000666f00007220000020200000ee
:1050880020000000466c00006173000068650000a5
:105098007220000073740000617200007420000028
:1050a8002020000000570000616900007420000003
:1050b8002564000073200000666f00007220000065
:1050c80020200000200000000a0d00004a550000c2
:1050d8004d4100002d5000004131000030300000eb
:1050e80030200000636f00007079000072690000d2
:1050f80067680000742000004f4800003753000024
:1051080056200000262000004f480000324e0000c4
:105118004c5400000a0d0000000a00000d53000066
:105128006f6600007477000061720000652000005f
:105138007665000072730000696f00006e20000041
:10514800002c00002064000061740000652000004d
:10515800200000002c200000636f00007079000020
:105168007269000067680000742000004a7500003a
:1051780068610000204e0000696900006e69000047
:105188006b6f0000736b0000692000004f4800003f
:10519800324e00004c5400000a0d0000000a0000c6
:1051a8000d57000072690000746500002066000059
:1051b80061630000746f00007279000020630000d2
:1051c800616c00006962000072610000746900008f
:1051d8006f6e000020760000616c000075650000ad
:1051e80073200000746f00002074000068650000e0
:1051f8002045000045500000524f00004d2e000091
:105208002050000061730000737700006f72000087
:10521800643a0000200000000a0d0000536f0000ef
:105228007272000079200000777200006f6e000033
:10523800672000005061000073730000776f000062
:10524800726400000a0d0000000a00000d52000000
:1052580065610000642000002620000075730000ce
:10526800652000002066000061630000746f000084
:105278007279000020630000616c00006962000020
:1052880072610000746900006f6e00000a0d000072
:10529800000a00000d53000065740000204600005d
:1052a800697200006d7700006172000065200000df
:1052b8006465000066610000756c0000747300008e
:1052c8000a0d0000000a00000d0a00000d41000050
:1052d800444300002028000049440000202000002a
:1052e8002920000025690000203d0000202500003d
:1052f800690000000a0d000041440000432000003e
:105308002856000044440000202900002025000001
:10531800692000003d20000025690000000a000007
:105328000d410000444300002028000042610000b5
:105338006e6400002920000025690000203d00005f
:1053480020250000690000000a0d0000414400000b
:105358004320000028520000455600002029000084
:1053680020250000692000003d200000256900007c
:10537800000a00000d4100004443000020280000fe
:10538800465700004420000029200000256900003d
:10539800203d000020250000690000000a0d0000e3
:1053a800414400004320000028540000656d0000bf
:1053b8007029000020250000692000003d20000021
:1053c80025690000000a00000d4100004443000068
:1053d80020280000415600007373000029200000b7
:1053e80025690000203d000020250000690000001c
:1053f80045450000505200004f4d0000207200004b
:105408006573000065740000206300006f7500007c
:105418006e74000065720000206300006c65000077
:10542800617200006564000020260000204d000025
:105438006f7200007175000065200000636c000049
:10544800656100006e200000757000000a0d000004
:10545800004c0000434400002077000072690000ff
:105468007465000020610000736300006969000032
:10547800200a00000d00000063680000617200004f
:10548800203d000020250000780a00000d000000e3
:105498004c4300004420000077720000697400004b
:1054a8006520000068650000780a00000d00000013
:1054b800203d000020250000630a00000d000000c8
:1054c8004c4500004420000062610000722000008a
:1054d80077720000697400006520000068650000ac
:1054e8007820000064610000746100002c20000036
:1054f8007265000076200000307800004646000003
:1055080046460000203d0000206500007869000044
:10551800740a00000d000000202000002020000078
:105528004c450000442000005465000073740000de
:105538002020000020200000000a00000d53000079
:105548006574000020460000574400002030000029
:10555800780000000a0d0000536500007420000068
:10556800524500005620000030780000004c000032
:1055780045440000206200006172000020670000be
:1055880072610000706800002074000065730000fc
:10559800742c000020730000706100006365000037
:1055a8002062000061720000203d000020650000bc
:1055b80078690000740a00000d0000000a0d000060
:1055c800536f0000756e00006420000074650000d1
:1055d800737400002c20000046430000594d000061
:1055e800487a0000202f0000207400006f6e000031
:1055f80065280000487a0000292000002a200000c1
:10560800322c000020670000697600006520000049
:10561800706900007463000068200000000a000040
:105628000d5300006f7500006e64000020740000c8
:1056380065730000742c0000206700006976000084
:105648006520000064750000726100007469000044
:105658006f6e0000286d0000732900002000000014
:105668000a0d000053650000742000004661000028
:105678006e20000028500000574d00002031000027
:1056880029200000766100006c750000652e00007e
:105698002053000074610000727400007e25000031
:1056a800642c0000204d0000617800003d250000ba
:1056b80064200000000a00000d4100006e7900001f
:1056c800206b000065790000203d00002073000079
:1056d800746f00007020000074650000737400008f
:1056e800000a00000d0000000a0d000044690000d7
:1056f8007620000062790000205a000065720000e0
:105708006f0000000a0d0000456e0000746500007f
:1057180072200000496300006f6d00002043000004
:10572800492d0000562000007465000073740000c5
:10573800206d00006f640000652c000020580000f8
:10574800203d00002065000078690000740000001a
:105758000a0d0000456e000074650000722000000c
:105768004b6500006e7700006f6f0000642000003a
:105778007465000073740000206d00006f64000001
:10578800650000000a0d00005465000073740000f5
:1057980020660000696c00006c200000636f000048
:1057a80066660000696e00002c200000766100002b
:1057b8006c7500006573000020660000726f0000c1
:1057c8006d200000616d00007020000026200000a0
:1057d800736500006e640000207400006f200000f4
:1057e8006d6f000072710000756500000000000018
:1057f800203100002e330000310000003039000055
:105808002e300000352e000032300000323000000b
:10581800003100003230000030200000200000007d
:10582800003200003430000030200000200000006a
:105838000034000038300000302000002000000054
:105848000039000036300000302000002000000041
:105858000031000039320000303000002000000024
:105868000033000038340000303000002000000011
:1058780000350000373600003030000020000000fe
:1058880000310000313500003230000030200000c7
:10589800003f00003f2000004d4800007a00000053
:1058a800312e0000384d0000487a00000033000017
:1058b8002e3500004d4800007a0000003720000017
:1058c8004d4800007a200000003100003020000020
:1058d8004d4800007a00000031340000204d0000df
:1058e800487a000000310000382000004d480000d0
:1058f8007a00000032310000204d0000487a000094
:1059080000320000342000004d4800007a000000fa
:1059180032380000204d0000487a000000350000b1
:10592800302000004d4800007a000000416c000063
:105938006c4d0000487a000000200000203500006f
:105948000020000031300000002000003235000047
:105958000020000035300000003100003030000029
:105968000032000030300000004100000056000006
:1059780000200000004a0000554d000041200000b2
:10598800504100003130000030300000002000009d
:10599800204f0000483200004e4c00005420000008
:1059a8004f48000037530000562000002000000038
:1059b8000a0d000045450000505200004f4d000000
:1059c8002063000068650000636b000073750000c9
:1059d8006d7300002c200000436100006c20000063
:1059e8003d200000255800002c20000044650000e0
:1059f8006620000043730000203d000020250000c1
:105a0800582c00002046000061630000746f0000fd
:105a1800727900002064000065660000617500006e
:105a28006c7400002072000065730000657400004b
:105a3800732000003d20000025640000000a0000db
:105a48000d45000045500000524f00004d20000059
:105a580063680000656300006b730000756d0000eb
:105a680020650000727200006f7200002c20000098
:105a7800726500006c6f0000616400002066000021
:105a880061630000746f00007279000020640000f8
:105a980065660000617500006c740000730000000a
:105aa80046610000637400006f72000079200000f6
:105ab8007365000074750000702000006f6b0000b3
:105ac8000050000075730000682000004155000078
:105ad800544f0000206600006f7200002020000074
:105ae8002000000066610000637400006f7200000f
:105af800792000006465000066610000756c000094
:105b08007473000000200000202000002020000006
:105b1800202000002020000020200000000a0000b3
:105b28000d0a00000d4a0000554d0000412d0000ef
:105b3800504100003130000030300000202f0000bc
:105b480020760000002000002f200000000a00003e
:105b58000d4300006f700000797200006967000053
:105b680068740000204a0000756800006120000089
:105b78004e690000696e0000696b00006f730000d9
:105b88006b6900002c2000004f480000324e0000d6
:105b98004c54000020260000204f00004837000029
:105ba800535600000a0d00000a0d0000000a00000c
:105bb8000d5300006574000020550000415200009c
:105bc8005420000075730000657200002062000018
:105bd80061750000642000007261000074650000b7
:105be800207400006f20000023250000692c0000ad
:105bf8002020000025730000626400000a0d0000e8
:105c080000530000657200007669000063650000bb
:105c1800207000006167000065730000202000000c
:105c2800200000004d610000696e00002070000037
:105c3800616700006573000020200000202000003c
:105c48002020000000730000656c00006563000000
:105c5800746500006420000020200000202000005f
:105c6800202000002000000046610000637400004e
:105c78006f72000079200000646500006661000012
:105c8800756c0000747300000073000065740000f8
:105c98002f730000746f000072650000642000001c
:105ca80020200000202000002000000020530000d9
:105cb80057520000002d00002e2d0000004f00005c
:105cc80056450000524c00004f410000442000009f
:105cd800505200004f54000045430000540000009b
:105ce8004c43000044200000425200004947000095
:105cf800485400004e450000535300002020000087
:105d08000025000069200000252500002020000053
:105d1800202000002020000020200000202000007b
:105d280020200000200000004c4300004420000018
:105d3800434f00004e5400005241000053540000ed
:105d4800202000002020000000420000414e0000fa
:105d5800442000004441000054410000202000007d
:105d68002020000020200000200000004243000006
:105d780044200000646100007461000020200000dd
:105d8800202000002020000020200000004a000001
:105d9800554d000041200000536500007269000065
:105da800616c00002020000020200000200000007e
:105db800496300006f6d000020430000492d00007a
:105dc8005620000020200000202000002020000095
:105dd800004b0000656e0000776f00006f640000e4
:105de8002054000053340000383000002020000008
:105df800200000004b6500006e7700006f6f000008
:105e0800642000005453000032300000303000009d
:105e180020200000004500006c650000637200004f
:105e2800616600007420000053650000726900007c
:105e3800616c0000200000005961000065730000db
:105e480075200000566f00006c7400006167000048
:105e580065200000202000002000000049630000a9
:105e68006f6d0000205600006f6c00007461000028
:105e7800676500002020000020200000004300008b
:105e88004f4d00002031000020200000202000009d
:105e9800202000002020000020200000200000001a
:105ea8004261000075640000205200006174000027
:105eb800652000002573000020200000004300003a
:105ec8004f4d00002032000020200000202000005c
:105ed80020200000202000002020000020000000da
:105ee800464100004e2000004d41000058200000af
:105ef800525000004d20000020200000202000000b
:105f08000041000054200000256900002004000022
:105f18004320000020200000202000002020000056
:105f28002000000045580000434900005445000087
:105f38005220000020200000202000002020000027
:105f480020200000004d00004158000020500000b3
:105f580057520000200000005720000020200000b9
:105f68002000000050410000205600004f4c000067
:105f78005441000047450000202000002020000078
:105f880020200000004c00006f7700002020000057
:105f980020200000202000002020000000480000f1
:105fa8006967000068200000202000002020000011
:105fb800202000000052000061640000696f0000aa
:105fc800205000006f6c00006c20000020200000b2
:105fd80020200000200000005261000074650000cd
:105fe800203d0000204f00006666000020200000d1
:105ff8002020000020200000202000000052000087
:1060080061740000652000003d200000256c000040
:10601800692000006d73000020200000202000008f
:1060280020000000434900002d56000020520000c7
:1060380061640000696f00002c3000003d4f0000d3
:10604800666600000041000064640000726500009c
:10605800737300002025000030320000584800000b
:10606800202000002020000020000000434f0000f6
:106078004d200000322000004d6f000064650000d4
:1060880020200000202000002020000000530000f5
:10609800657200007669000063650000202000003a
:1060a8002020000020200000202000002000000008
:1060b8005041000031300000303000002052000014
:1060c800656d00006f74000065200000202000004e
:1060d8000042000065650000702000006c6500004b
:1060e8006e2c0000203000003d4f000046460000a6
:1060f800200000004265000065700000203d00009f
:1061080020250000692000006d7300002020000099
:1061180020200000005600006f6c00007461000031
:1061280067650000202000002020000000430000d8
:10613800616c0000206d0000756c00007420000088
:106148003d200000256c00006920000020000000b0
:106158004375000072720000656e00007420000034
:10616800202000000050000077720000203c000052
:10617800333000004d4800007a0000002020000065
:106188002d2d00002d2d00000020000057000000dc
:10619800436100006c2000006d7500006c74000005
:1061a800203d000020250000332e0000326600004c
:1061b800202000002020000000500000777200001e
:1061c80020350000304d0000487a00002000000013
:1061d8004c4500004420000042610000722000008d
:1061e800486f00006c6400002020000020200000a0
:1061f80000250000692000006d73000020200000c9
:106208002020000020200000202000002020000086
:1062180020200000004c00004544000020420000ff
:10622800617200002044000065630000617900008d
:1062380020200000200000002569000020570000f1
:106248002f310000303000006d7300002020000066
:106258002020000020200000200000004b650000e6
:1062680065700000204f00005045000052200000db
:10627800737400006174000065200000004e000087
:106288006f200000202000002020000020200000b7
:106298002020000020200000202000002000000016
:1062a8005965000073200000202000002020000015
:1062b80020200000202000002020000020200000d6
:1062c8000020000046570000442000002020000065
:1062d80052450000562000002020000053570000bf
:1062e80052000000202000000020000020200000b4
:1062f800004200004344000020620000616e00007c
:1063080064200000444300004241000020200000b7
:106318002000000062690000747300002000000083
:10632800496e000020200000004f00007574000036
:1063380020000000434f00004d31000020520000b3
:1063480058200000256c0000692000002020000073
:106358002020000020200000004300004f4d0000d6
:106368003220000052580000202500006c6900000f
:106378002020000020200000202000002000000035
:1063880046610000637400006f720000792000000d
:10639800636100006c200000202000002020000025
:1063a8000046000061630000746f0000727900000d
:1063b80020630000616c00002d3e00007573000032
:1063c8006500000053650000743d0000392000009e
:1063d800436f0000756e0000743d000025690000e1
:1063e80020200000200000004465000066610000d5
:1063f800756c0000747300002d3e000045450000d8
:10640800505200004f4d0000000000000a0d00002f
:106418005458000073740000617400006520000087
:10642800576f000072640000732000003d200000d8
:10643800256400002c2000005375000063650000ef
:1064480073730000203d000020250000642c00002c
:10645800200000000a0d0000576f00007264000061
:10646800732000003d200000256400002c2000005f
:10647800537500006365000073730000203d000041
:1064880020250000642c00002043000068650000ff
:10649800636b0000737500006d2000003d20000054
:1064a80025580000000a00000d5700006f72000018
:1064b80064730000203d000020250000642c0000cb
:1064c80020530000756300006365000073730000cb
:1064d800203d000020250000642c0000204300001f
:1064e80068650000636b0000737500006d20000094
:1064f8003d20000025580000000a00000d4600005d
:1065080061630000746f000072790000204300008e
:10651800616c00006962000072610000746900002b
:106528006f6e0000204400006174000061200000cc
:10653800696e000020750000736500000a0d0000f8
:10654800000a00000d63000068650000636b00002e
:10655800737500006d20000066610000696c000022
:10656800656400002c2000005573000065200000c1
:1065780046690000726d00007761000072650000d6
:106588002064000065660000617500006c740000fe
:10659800730a00000d000000447500006d700000d3
:1065a8002045000045500000524f00004d200000db
:1065b800636f00006e740000656e00007473000065
:1065c8000a0d0000000a00000d250000352e00000d
:1065d8003458000000200000253400005800000056
:1065e8000a0d00004c610000737400002073000065
:1065f800756300006365000073730000206300008a
:106608006f640000652000003d2000002558000050
:10661800200000000a0d00004661000074610000bf
:106628006c20000045520000524f0000522000002c
:10663800577200006f6e000067200000636f000053
:1066480066660000696e0000206100006464000056
:1066580072650000737300002025000058000000d8
:106668000a0d0000537900007350000057520000d3
:106678002046000020250000642000005220000071
:10668800256400002c2000004c6100007374000099
:1066980020730000616d0000706c000065730000dd
:1066a8002c20000074680000697300002069000055
:1066b800732000006c6f00006767000065640000cd
:1066c8002046000020250000642000005220000021
:1066d800256400002028000057290000000a000057
:1066e8000d530000797300004944000063750000f1
:1066f80072200000253300002e310000662c0000b7
:10670800204c0000617300007420000073610000d9
:106718006d7000006c6500006420000025330000e7
:106728002e3100006620000028410000292c0000be
:10673800206c00006172000067650000737400003f
:1067480020760000616c000075650000206900007b
:10675800732000006c6f000067670000656400002c
:10676800000a00000d4300006f6600006669000023
:106778006e200000706c000061630000656400001a
:10678800207400006f200000255800002c20000015
:10679800646500006174000068200000636f0000f9
:1067a800756e00007420000025640000200a0000b7
:1067b8000d0000000a0d0000436f0000666600002f
:1067c800696e00002025000058200000636f00005b
:1067d8006e740000656e0000740000000a0d000071
:1067e8004657000044200000706f000077650000e5
:1067f80072200000202000002564000020570000bf
:10680800000a00000d5200004556000020700000ec
:106818006f7700006572000020200000202500002e
:1068280064200000570000000a0d000042610000cb
:106838006e640000200000002d2d00002d000000d7
:106848003f3f000020000000312e0000380000000b
:10685800332e000035000000372000002000000023
:10686800313000002000000031340000200000001a
:106878003138000020000000323100002000000004
:1068880032340000200000003238000020000000f0
:106898003530000020000000416c00006c00000052
:1068a800204d0000487a00002c20000047610000bd
:1068b800696e00002025000064200000000a000026
:1068c8000d50000041200000766f00006c7400003d
:1068d800726100006765000020250000332e00006b
:1068e8003166000020560000000a00000d5000002c
:1068f800412000006375000072720000656e0000a0
:106908007420000020250000332e000031660000ae
:1069180020410000000a00000d5000004120000046
:10692800746500006d700000202000002020000029
:106938002025000064200000430000000a0d00002c
:106948004465000061740000682000006361000075
:10695800757300006520000030780000255800009d
:10696800203d000000200000485700002070000073
:10697800726f00007465000063740000696f0000a6
:106988006e000000205200006576000020500000d4
:1069980057520000002000004355000052520000ea
:1069a800454e00005400000020530000572000000e
:1069b8006f760000657200006c6f00006164000073
:1069c80020700000726f000074650000637400009e
:1069d800696f00006e0000002c2000004155000087
:1069e800544f0000424100004e4400002077000050
:1069f80061730000204f00006e0000002c20000092
:106a0800556e00006b6e00006f7700006e2000006e
:106a18003f3f00003f0000000a0d00000a0d000083
:106a28004d6f000072710000756500002064000061
:106a3800617400006120000053740000617200005e
:106a4800742000005f5f00005f5f00005f5f000070
:106a58005f5f00005f5f00005f5f00005f5f000036
:106a68005f5f00005f5f00005f5f00005f5f000026
:106a7800000a00000d0a00000d45000076650000c0
:106a88006e74000020230000202500006420000010
:106a98002d2d00002d2d00002d2d00002d2d000086
:106aa8002d2d00002d2d00002d2d00002d000000a3
:106ab800204f00006c640000657300007420000023
:106ac80065760000656e000074000000204e00002e
:106ad800657700006573000074200000657600008b
:106ae800656e0000740000000a0d00000a0d000029
:106af8004d6f000072710000756500002064000091
:106b08006174000061200000456e000064200000f0
:106b18005f5f00005f5f00005f5f00005f5f000075
:106b28005f5f00005f5f00005f5f00005f5f000065
:106b38005f5f00005f5f00005f0a00000d0000005b
:106b4800446500006174000068200000636f000065
:106b5800756e000074200000256400002c200000e1
:106b68004e65000078740000206600007265000021
:106b780065200000636f000066660000696e000013
:106b880020250000580a00000d0000000000000049
:106b980000000000a0f00000190000008084000040
:106ba8001e000000000900003d00000020b30000a6
:106bb80081000000001b0000b70000000024000056
:106bc800f4000000e08b000029010000a052000042
:106bd8005701000080ba00008c01000080c300004b
:106be800c9010000c03b0000470300002530000039
:106bf80032580000200000000a0d00002d2d000072
:106c08002d2d00002d2d00002d2d00002d2d000014
:106c18002d2d00002d2d00002d2d00002d2d000004
:106c28002d2d00002d2d00002d2d00002d2d0000f4
:106c38002d2d00002d2d00002d2d00002d2d0000e4
:106c48002d2d00002d2d00002d2d00002d2d0000d4
:106c58002d2d00002d2d00002d2d00002d2d0000c4
:106c68002d2d00002d2d00002d2d00002d2d0000b4
:106c78002d2d00002d2d00002d2d00000a0d0000e7
:106c8800000a00000d54000058200000256900008b
:106c98002c200000412000004672000065710000b1
:106ca800202500006c6900002c2000004220000014
:106cb8004672000065710000202500006c69000024
:106cc8000a0d0000002d00002d2d00002d2d0000c4
:106cd8002d2d00002d2d00002d2d00002d2d000044
:106ce8002d2d00002d2d00002d2d00002d2d000034
:106cf8002d2d00002d2d00002d2d00002d2d000024
:106d08002d2d00002d2d00002d2d00002d2d000013
:106d18002d2d00002d2d00002d2d00002d2d000003
:106d28002d2d00002d2d00002d2d00002d2d0000f3
:106d38002d2d00002d2d00002d2d00002d2d0000e3
:106d48002d2d00002d0a00000d0000000a0d000086
:106d58004578000069740000204b0000656e000053
:106d6800776f00006f6400002074000065730000f6
:106d7800742000006d6f0000646500000a0d0000bb
:106d8800000a00000d4b0000656e0000776f0000e0
:106d98006f64000020560000464f000020410000ac
:106da8002066000072650000712000000a0d0000d6
:106db800000a00000d4b0000656e0000776f0000b0
:106dc8006f64000020560000464f0000204200007b
:106dd8002066000072650000712000000a0d0000a6
:106de800000a00000d4b0000656e0000776f000080
:106df8006f64000020520000582000005646000032
:106e08004f2000006d6f000064650000200a00003c
:106e18000d0000000a0d00004b6500006e770000b1
:106e28006f6f0000642000005458000020560000d6
:106e3800464f0000206d00006f64000065200000d0
:106e48000a0d0000000a00000d4b0000656e0000ee
:106e5800776f00006f640000205400005820000085
:106e680066720000657100002c2000006d6f000044
:106e7800646500002c2000006d7500006c74000033
:106e8800692000000a0d0000000a00000d4b0000f8
:106e9800656e0000776f00006f64000020580000e6
:106ea800492000000a0d0000000a00000d4b0000f8
:106eb800656e0000776f00006f640000204d0000d1
:106ec800656d00006f72000079200000303000000e
:106ed800206d00006f640000652000000a0d0000ae
:106ee800000a00000d4b0000656e0000776f00007f
:106ef8006f640000205000006f770000657200008a
:106f0800204f00006e2f00004f6600006620000032
:106f18006d6f000064650000200a00000d0000008d
:106f28000a0d00004b6500006e7700006f6f0000cf
:106f380064200000506f0000776500007220000098
:106f48004f660000662000000a0d0000000a0000dd
:106f58000d4b0000656e0000776f00006f64000045
:106f6800205000006f77000065720000204f00007d
:106f78006e2000000a0d0000000a00000d4b000002
:106f8800656e0000776f00006f64000020500000fd
:106f98006f77000065720000205300006c650000e8
:106fa80065700000200a00000d00000000000000cd
:106fb80000000000a0f0000019000000808400001c
:106fc8001e000000000900003d00000020b3000082
:106fd80081000000001b0000b70000000024000032
:106fe800f4000000e08b000029010000a05200001e
:106ff8005701000080ba00008c01000080c3000027
:10700800c9010000c03b0000470300000a0d000052
:1070180052610000646900006f2000006164000094
:10702800647200006573000073200000736500003f
:1070380074200000746f00002030000078250000e4
:1070480030320000580a00000d0000002530000012
:1070580032580000200000000a0d0000000a00005d
:107068000d4600007265000071200000256c0000cc
:10707800692c000020420000616e000064200000be
:10708800256900002c20000052610000646900009e
:107098006f200000307800002530000032580000d2
:1070a8002c200000446500007374000020300000ac
:1070b8007825000030320000582c000020630000c2
:1070c8006e74000020250000690a00000d00000011
:1070d8002d2d00002d2d00002d2d00002d2d000040
:1070e8002d2d00002d2d00002d2d00002d2d000030
:1070f8002d2d00002d2d00002d2d00002d2d000020
:107108002d2d00002d2d00002d2d00002d2d00000f
:107118002d2d00002d2d00002d2d00002d2d0000ff
:107128002d2d00002d2d00002d2d00002d2d0000ef
:107138002d2d00002d2d00002d2d00002d2d0000df
:107148002d2d00002d2d00002d2d00002d2d0000cf
:107158000a0d0000000a00000d45000078690000d3
:1071680074200000496300006f6d00002043000098
:10717800492d00005620000074650000737400005b
:10718800206d00006f640000650a00000d0000001b
:107198000a0d0000536500006e64000020430000e3
:1071a800492d000056200000436f00006d6d00005f
:1071b800616e0000642000003033000048200000a9
:1071c800746f00002052000061640000696f0000c5
:1071d800203000007825000030320000580a0000f6
:1071e8000d0000000a0d0000536500006e640000e9
:1071f80020200000434900002d56000020430000d5
:107208006f6d00006d6100006e64000020300000aa
:10721800354800002c200000663d0000332e000099
:1072280036390000394d0000487a0000200a000075
:107238000d0000000a0d0000536500006e64000098
:1072480020200000434900002d5600002043000084
:107258006f6d00006d6100006e640000203000005a
:10726800354800002c200000663d00003134000045
:10727800352e000032370000354d0000487a0000f6
:10728800200a00000d0000000a0d000053650000f0
:107298006e64000020430000492d000056200000c5
:1072a800436f00006d6d0000616e000064200000f7
:1072b8004a6100006d6d00006572000020630000e7
:1072c8006f640000652000000a0d00000000000047
:1072d800202000002020000045720000726f00008e
:1072e8007220000021200000200000000a0d00008c
:1072f80054520000415000003a2000004f73000033
:10730800636900006c610000746f00007220000067
:1073180045720000726f0000720a00000d00000044
:107328004f530000434300004f4e00002030000040
:1073380078250000580a00000d0000000a0d000022
:1073480054520000415000003a20000041640000ff
:10735800647200006573000073200000457200002d
:10736800726f0000720a00000d0000005730000024
:107378002030000078250000580a00000d000000a9
:10738800573100002030000078250000580a00001e
:107398000d00000057320000203000007825000062
:1073a800580a00000d00000057330000203000008c
:1073b80078250000580a00000d000000573400002e
:1073c8002030000078250000580a00000d00000059
:1073d800573500002030000078250000580a0000ca
:1073e8000d0000005736000020300000782500000e
:1073f800580a00000d000000573700002030000038
:1074080078250000580a00000d00000057380000d9
:107418002030000078250000580a00000d00000008
:10742800573900002030000078250000580a000075
:107438000d000000573100003020000030780000b7
:10744800255800000a0d00000057000031310000e7
:107458002030000078250000580a00000d000000c8
:107468005731000032200000307800002558000015
:107478000a0d0000005700003133000020300000e2
:1074880078250000580a00000d0000005731000060
:107498003420000030780000255800000a0d000054
:1074a800005700003135000020300000782500002a
:1074b800580a00000d0000000a0d00005452000098
:1074c800415000003a20000053740000616300003e
:1074d8006b20000045720000726f0000720a000005
:1074e8000d0000000a0d0000545200004150000039
:1074f8003a2000004d61000074680000204500003b
:10750800727200006f7200000a0d0000000a00008d
:107518000d53000070750000726900006f7500005f
:1075280073200000496e000074650000727200004c
:10753800757000007420000045720000726f000032
:10754800720a00000d0000000a0d00000a0d00007c
:10755800504100003130000030300000205200005f
:10756800656d00006f74000065200000436f000027
:107578006e740000726f00006c20000070610000e3
:10758800636b000065740000203000007830000054
:10759800310a00000d00000052610000773a000037
:1075a8002020000053540000582c00002000000048
:1075b80025300000325800002c2000000045000053
:1075c80054580000000a00000d4300006f640000da
:1075d800656400003a200000000a00000d0a00005f
:1075e8000d480000444c000043200000706b000070
:1075f800742000006c6500006e2000002564000007
:107608002c2000004461000074610000200000008c
:107618002530000032580000200000002043000000
:1076280052430000203d0000204f00006b2e000058
:107638000a0d00000a0d000000200000435200005f
:107648004320000046610000696c0000656400008a
:107658002025000030320000580a00000d0a000002
:107668000d00000053740000756300006b200000db
:1076780042750000747400006f6e00000053000033
:107688005731000020410000444a000055530000d3
:1076980054200000446f0000776e00000053000083
:1076a800573200002050000041470000450000000c
:1076b8005357000033200000414400004a550000a1
:1076c800535400002055000070000000535700007c
:1076d800342000004f5000004552000000530000c5
:1076e8005735000020420000414e000044200000b1
:1076f800446f0000776e000000530000573600000a
:1077080020410000555400004f000000535700006e
:1077180037200000424100004e4400002055000080
:1077280070000000000000004a000000f2000000a5
:107738009401000035020000dc0200007b03000019
:107748001f040000c50400006505000009060000cc
:10775800ac06000050070000550000004802000079
:107768000400000049020000d30300000a000000e2
:10777800d4030000c304000009000000b3050000a2
:10778800b006000007000000a407000096080000eb
:10779800050000008d090000800a000003000000b9
:1077a800750b00006b0c000002000000550d000076
:1077b800620f00000100000000000000000000004f
:1077c800a0f0000019000000808400001e000000e6
:1077d800000900003d00000020b300008100000007
:1077e800001b0000b700000000240000f4000000a7
:1077f800e08b000029010000a052000057010000a2
:1078080080ba00008c01000080c30000c90100009c
:10781800c03b0000470300002000000000010000fa
:10782800010200002003000003040000040200001d
:10783800060600000606000005070000070700000e
:1078480047310000004700003200000047330000c5
:1078580000470000340000004735000000470000e2
:1078680036000000473700000047000038000000dd
:10787800ffff0000feff0000fcff0000f8ff000013
:10788800f0ff0000e0ff0000c0ff000080ff0000e4
:1078980000ff000000fe000000fc000000f80000ef
:1078a80000f0000000e0000000c0000086010000b9
:1078b800c200000061000000300000001700000056
:1078c8000b00000007000000030000007f0100001b
:1078d800bf0000005f0000002f000000170000003c
:0c78e8000b00000007000000030000007f
:020000040000fa
:1078f4000400fa00100798009e0090004006200043
:10790400808f5000020036004006200010079800c7
:107914009e009000800220000088b900800078005a
:1079240000fa2000010f50001e007800921d07008d
:107934000080fa00000006000200fa00000f780040
:10794400400620009e0f1000020036004006200072
:10795400000f78001e0078006a00b900000f78005c
:107964001e0078007e1d07000080fa00000006005b
:107974000000fa00889fbe00506980000000e80003
:1079840050698800a15a8000f0578000808f500011
:1079940002003400a05a8000f0578800516980002a
:1079a400600a2000808f500012003a00f0578000d7
:1079b4006103b900c25d8000d35d80000234b80069
:1079c40003b0b90009027800000242000790b90030
:1079d400000242008404780040c8de00cf80de004c
:1079e400705a88000000eb00f05788000000eb009c
:1079f40050698800705a80006213070090cb2a00f7
:107a0400f41107004f04be000080fa0000000600d5
:107a14000400fa00889fbe00a00020002629070069
:107a24006101b900505a8000615a80000200400090
:107a340083804800505a8800615a88004069800059
:107a44000000e8004069880040698000ef0f5000a2
:107a54001a0034000000eb0040698800505a80008e
:107a6400615a8000c40cde004c09dd004404de00d1
:107a740008047100e05d8000f15d80000001be003b
:107a84000243b80003c0b9000702780000024200b4
:107a94000990b9000002420084037800068fbe00fa
:107aa4006000b800505a8800615a88001e00be0069
:107ab4004008de000100200000588800b06a800001
:107ac4000000e00004003a00401f2000b06a880073
:107ad40000588000405a8800405a8000291307004b
:107ae400b0cb2a00bb110700d0cb2a00b911070084
:107af4004f04be000080fa00000006000000fa00f7
:107b0400f05a800041072000b212070040c0b300c1
:107b14008311070030c4b300811107000080fa000c
:107b2400000006000000fa00e7c2bf0001c8b3006d
:107b3400014060000004e00010003200ca82a90085
:107b4400c682a900105c80000000e00006003a0034
:107b540000c8b300290e07000000eb00105a88008b
:107b64000000eb00205a88000040eb00a5ebb700b2
:107b7400105c80000010a000105c88000080fa00f7
:107b8400000006000000fa000000eb00105c880012
:107b9400caa2a80020002000ab280700caa2a9009e
:107ba4000000eb00806988000080fa0000000600f5
:107bb4000200fa00100020004d280700005c80003d
:107bc4000000e00018003a0073280700004f780016
:107bd40042cdbf009e4f50000f003a00206a800043
:107be4000000e00010003200206a80000000e9007c
:107bf400206a8800206a80000000e0000a003a0041
:107c040042cdbf000080fb00105d880060092000a9
:107c1400206a8800040037001e40780042edb70057
:107c240060092000206a88000080fa000000060035
:107c34000200fa00004f78001e4078003c2807003c
:107c4400b3cbbf000004e000020032000000eb00f0
:107c5400272807000080fa00000006000200fa004e
:107c6400a4cbbf000004e00093003200b3cbbf00fc
:107c74000000fb00000f78001e007800e40f5000a5
:107c84000d003c001e007800e30f500048003d004a
:107c94001e007800e10f5000130032001e0078002f
:107ca400e10f50002a003c001e0078000000e000b4
:107cb4000b003200800037001e007800e60f5000f1
:107cc400720032001e007800e60f500057003500a5
:107cd4001e007800e70f5000720032007600370073
:107ce400b3ff07007400370064260700f0648000c7
:107cf4000000e00005003a00806b80000000e00016
:107d040002003a000000eb00105d8800e06480008f
:107d14000000e00068003a00505e80000000e000cf
:107d240065003200505e8000e06488001f26070072
:107d3400f06480000000e0005f003a00007d200055
:107d4400f06488000000eb00806b88005a00370064
:107d5400931e0700505e80000000e00056003200d1
:107d6400a06b8000e10f500005003a00505e8000d7
:107d7400e0648800505e80006300b900f06488000d
:107d8400f06480000000e00002003a000000eb0014
:107d9400105d8800e06480000000e00046003a00c6
:107da400505e8000e0648800f11d07004200370047
:107db400061b0700e06480000000e0003e003a007b
:107dc400505e80000000e0003b003200505e800006
:107dd400e0648800206b80000000e00003003200b3
:107de400505e80006300b900f0648800f064800095
:107df4000000e00002003a000000eb00105d880083
:107e0400b3cbbf00e44f500002003a00061a07004b
:107e140001003700271a07000000eb00206b8800e0
:107e24000000eb00306b880023003700ab2507000f
:107e3400e06480000000e0001f003a00505e800013
:107e44000000e0001c003200505e8000e064880006
:107e5400b06b80000000e00003003200505e800040
:107e64006300b900f0648800f06480000000e00062
:107e740002003a000000eb00105d880013250700a3
:107e84000000eb00b06b88000b003700005c800042
:107e94000000e00008003a004b270700105d88004e
:107ea40005003700005c80000000e00002003a009a
:107eb40064270700105d8800805e80000000e000f9
:107ec40014003a00305c80000000e0000f00320033
:107ed400115d8000305c8000808f50000b00320008
:107ee400a5cbbf000004e00008003200415e800022
:107ef400c0f620008f1c07000040eb00a5ebb70084
:107f0400e862a800ca82a900c682a900105d8000a8
:107f1400305c88000080fa00000006000000fa00cf
:107f2400a06a80000000e00015003a00401f200015
:107f3400a06a8800e0002000df270700cf80de0071
:107f4400d05a8800e15a8800d25a8000e35a80004f
:107f540000fa20000012b8006010b9000503780090
:107f64000003430000fa20000098b9000003430016
:107f7400860278004028de0001002000f05a8800c4
:107f8400f0002000cc270700c0002000ca2707000b
:107f9400c05a8800d0002000c7270700b05a8800c4
:107fa40090002000c4270700a05a8800b05a80001f
:107fb4002d210700b05b8800c15b8800c05a800097
:107fc40029210700d05b8800e15b8800a05880006d
:107fd4000000e800a0588800705880008158800094
:107fe400b25b8000c35b800062ec070070588800bd
:107ff400815888005058800061588000d25b80000e
:10800400e35b80005bec07005058880061588800ef
:10801400a1588000800c2000808f500016003a0088
:108024007058800081588000a2702d0033ba23005c
:10803400adec070030588800415888005058800043
:1080440061588000a2702d0033ba2300a6ec07000b
:1080540010588800215888006000b80070588800c3
:10806400815888006000b800505888006158880022
:108074000000eb00a0588800305880004158800070
:108084000200200003222400cbec07000000e000e3
:1080940001003c000700370012588000235880007c
:1080a40030588000415880006e210700a05b880092
:1080b400020037000000eb00a05b8800a05b80009a
:1080c4000000e00004003200a05b8000905b8800a8
:1080d400c012200090588800905880000000e000f2
:1080e40003003200905880000000e9009058880096
:1080f400905880000000e00002003a000000eb000d
:10810400905b88000080fa00000006000000fa007e
:10811400c6c2bf00704060000004e00048003200a6
:10812400c8c2bf00684060000004e00044003200a0
:10813400105d8000ea0f500003003a00b01f2000d9
:108144009069880002003700603b20009069880035
:10815400a05a80006101b900b0588000c158800065
:108164000200400083804800b0588800c15888004d
:10817400b05a800080007800d0588000808f500072
:1081840002003600b05a8000d058880000598000a0
:108194000000e8000059880000598000e30f5000f7
:1081a4002e003400b0588000c1588000f058880078
:1081b400d0588000e05888000000eb000059880087
:1081c4000000eb00d05888006000b800b058880068
:1081d400c1588800f158800000f72000808f5000bb
:1081e4001e003600e158800090698000808f5000a6
:1081f4001a003100ca82a900c682a900e862a80058
:1082040000c4b3007d0c07000040eb00a5ebb700f1
:10821400405e80006300b90080007800c0f6200052
:10822400c41b070080382100906a880010002000d9
:10823400806988000000eb00205a8800070037009e
:108244000000eb00005988000000eb00d0588800c3
:108254006000b800b0588800c15888000080fa0057
:10826400000006000200fa00f05a8000fe0f5000e1
:1082740003003c000000eb00331b07000e00370036
:10828400f15b8000f05a80000088b900000f78008c
:108294001e0078004300de00000f7800c0a8200014
:1082a4009e0f100002003600c0a82000000f7800c6
:1082b4001e007800241b07000080fa00000006005e
:1082c4000000fa00825d80000046250011000900cc
:1082d4000200d800f05b88000080fa00000006006d
:1082e4000000fa00b4cbbf000004e0000300320039
:1082f400005c8000e10f500002003a00d682a80022
:1083040001003700d682a9000080fa0000000600b0
:108314000000fa00b4cbbf000004e00002003a0001
:10832400d682a80001003700d682a9000080fa0096
:10833400000006000000fa00115d800060b9200012
:1083440000804000104078000004e00005003d007b
:10835400115d800060b92000808040000040eb0087
:1083640080487800115d800060b9200000804000e2
:10837400104078008000fb00c0698000808f5000ae
:1083840006003400125d8000c069800080407800df
:1083940060b9200000004100014878000080fa0024
:1083a400000006000200fa00b2cbbf000000fb0090
:1083b400000f78001e007800e30f50001100320017
:1083c4001e007800e30f500004003c001e007800fb
:1083d4000000e00013003500070037001e0078009d
:1083e400e40f50000a0032001e007800e50f500030
:1083f4000a0032000b00370070002000c0698800ba
:108404000800370060002000c069880005003700bc
:1084140030002000c0698800020037000000eb0033
:10842400c0698800c3ff07000080fa00000006004e
:108434001200fa00889fbe00f0f32e000016880098
:108444000000eb0010168800b0e02700301688000a
:108454000002200040168800e00024006016880016
:1084640000002200701688000000eb0090168800bf
:1084740000012000a0168800c0c72f00f016880055
:108484000000eb0000178800000028002017880077
:108494008000200030178800bafd0700ca82a900b6
:1084a400c682a900a222070040442500a004880037
:1084b400841a0700c0cc210010598800c524070085
:1084c4000000eb00f52407000000eb00072507007f
:1084d4002003200006fd07002003200016fd0700ee
:1084e400910d0700d70d0700870d0700f0cb2a0078
:1084f400380f0700c0bf2a00360f070000c4b300be
:10850400770d0700b0cc2a00320f0700415e8000cf
:10851400c0f62000071b07000000eb00400798008e
:10852400090037004e009000dc2407004e00900044
:10853400ee24070020032000432607004e0090008d
:108544000000e800400798004e009000ee0f500035
:10855400f4ff3600e862a900d1a2a900007d200042
:10856400392607000000eb00cc2407000000eb00d4
:10857400de240700e862a800d1a2a800cf200700eb
:10858400e222a900c81d070020002000e075880031
:108594003a2607002209070040079800b708070099
:1085a4003007980059080700405c8000801f78005d
:1085b4003e009000801f7800ce009000811f78005c
:1085c400c0cd2a00801f780069df0700e8875700c4
:1085d4004e0090000000e00003003a003e009000ce
:1085e4000000e00013003200d909070030d22a004d
:1085f400801f78005edf07008f87e900bf07070050
:1086040014080700c50807005b080700405e8000e7
:108614006a00b90080007800c0f62000c51a07007f
:10862400390d070040d52a00ea0e0700007d20001e
:1086340005260700305d8000adfc0700405d80002a
:10864400bdfc0700105d8000eb0f500002003400f9
:10865400b0002000105d8800805e80000000e00013
:1086640002003a000040eb00a5ebb700405e80003a
:108674000000400080007800f0a42000ad1a07003c
:10868400caa2a800200d0700caa2a9001b00370037
:108694000040eb00120d070050d62a00cd0e070053
:1086a40000c4b3000e0d070060d72a00c90e0700ee
:1086b400c3c2bf000044b2000004e0000f003a004f
:1086c400110d070040d52a00c20e07008b070700d2
:1086d4009208070028080700de070700405e8000b4
:1086e4006a00b90080007800c0f62000911a0700e3
:1086f400007d2000d425070004003700cec2bf004f
:10870400684060000004e000e1ff3200b3cbbf002a
:108714000004e00002003a00100020007425070065
:10872400605d800072200700705d80006c1d070092
:10873400b3cbbf00e24f500002003a00821b070097
:1087440001003700851b070070d82a00801f7800bd
:1087540007df07008f87e90030d92a00801f7800df
:1087640003df07008f87e900c0bf2a00801f78005d
:10877400ffde07008f87e90070da2a00801f780087
:10878400fbde07008f87e90020c02a00801f7800e5
:10879400f7de07008f87e900b0da2a00801f78002f
:1087a400f3de07008f87e900705d8000e30f50005f
:1087b4000c003200705d80004300dd008000780012
:1087c400d0c02a0000804000715d8000801f7800c6
:1087d400811f7800b0dd2a00801f7800e4de0700e6
:1087e400e68757000000eb00205a88000000eb00e9
:1087f400305a88000000eb00105a8800b0fe0700d1
:10880400b0002000205c8800a4cbbf00e14f5000e2
:1088140004003a000000eb00105d88001000200006
:10882400a0698800bafe0700defe07000040eb00e6
:1088340096ebb7004124070000003700c5c2bf0013
:108844000080fb004400de000004a20061406000e0
:108854006140600061406000614060004401dd00ef
:10886400512c200091407800f0ceb30000c060008d
:1088740002407000c5e2b700a5cbbf000004e000d1
:1088840002003200e862a90001003700e862a80093
:10889400a2fd07001dfe070072fe0700a1fc0700f1
:1088a400a5cbbf00e14f50000f003a00105c8000e0
:1088b4000000e00007003a00105d80000000e000c6
:1088c40004003200c682a8000000eb00a069880002
:1088d40009003700ca82a900c682a900100020003e
:1088e400a069880004003700ca82a900c682a900d2
:1088f4000000eb00a0698800c6c2bf0070406000a1
:108904000004e00003003a00305a8000e80f5000f1
:108914006b003a00d05b8000e15b8000991f070088
:1089240050079800205b80000000e0000300320044
:10893400205b80000000e900205b8800205b800051
:108944000000e0000c003a00305b80000000e00012
:1089540009003200315b8000705e800000805000ae
:10896400305b8800305b80000000e00002003d00c6
:108974000000eb00305b8800315b80005e009000fb
:10898400810f5000040034005e019000325b8800c7
:10899400605e8000205b8800335b80005307980092
:1089a4005e00900079004000500798005e0090003f
:1089b40022032000110009000200d800505b880047
:1089c400b05b8000c15b80006e1f070050079800f9
:1089d4005e009000605b8800005b80000000e000a7
:1089e40003003200005b80000000e900005b8800a7
:1089f400005b80000000e0000c003a00105b800087
:108a04000000e00009003200115b8000705e80000d
:108a140000805000105b8800105b80000000e000c4
:108a240002003d000000eb00105b8800115b800039
:108a34005e009000810f500004003400de009000be
:108a4400115b8800605e8000005b8800125b800020
:108a540052079800de009000700c2000808f5000b8
:108a64000a0034005e0090002003b0005007980014
:108a74005e00900042062000110009000200d800a8
:108a84000080e800405b8800080037005e0090002a
:108a940079004000500798005e00900022032000f7
:108aa400110009000200d800405b8800405b800090
:108ab4007a230700505b80008c23070012003700e4
:108ac4000000eb00105b88000000eb00305b8800c6
:108ad4000000eb0085230700c6c2bf0070406000a1
:108ae4000004e00006003a00005c8000e10f500042
:108af40003003a00f0ff2d00402307000200370076
:108b04000000eb0065230700105d800048fc0700af
:108b1400115d800060b920000080400010407800a2
:108b24000b210700005c80000000e00002003a0016
:108b3400105d800059210700f5fd0700cec2bf007b
:108b4400624060000004e0008a003a0080bb20001c
:108b540010658800105a80000000e0000d003a0003
:108b6400205a8000e80f50000a003a00415e80005d
:108b7400c0f620006f190700f06980000000e000d3
:108b84001b0032000000eb00f0698800fa060700c1
:108b940017003700105a8000e10f500007003a0018
:108ba400305a8000ef0f500004003a00415e80000c
:108bb400c0f620005f1907000d003700415e8000f9
:108bc40020c420005b1907000900370010658000ed
:108bd4000000e00006003a00405e80006a00b90030
:108be40080007800c0f62000521907000400370006
:108bf400cec2bf00624060000004e000f3ff320018
:108c0400106580000000e00043003a00105a800024
:108c14000000e800105a8800105a8000e10f50004c
:108c24000e0034000000eb00105a8800006a800037
:108c34000000e000030032000000eb00006a88003e
:108c440036070700f06980000000e00003003200ee
:108c54000000eb00f0698800c70607000000eb0085
:108c6400205a88000000eb00305a880000e22400fb
:108c7400106588000040eb00990b0700105a800033
:108c8400e10f500003003a0050e02a00510d0700a4
:108c94000200370060e12a004e0d070000c4b30053
:108ca4008f0b070070e22a004a0d070015003700f9
:108cb400106580000000e00012003a000040eb0064
:108cc400870b070080e32a00420d070000c4b300ad
:108cd400830b070090e42a003e0d0700d707070026
:108ce400405e80006a00b90080007800f0a4200093
:108cf40010190700cec2bf00624060000004e0000b
:108d0400fcff3200cec2bf00624060000004e000fd
:108d1400e7ff320014003700105a80000000e00022
:108d240009003a00205a80000000e800205a880018
:108d3400205a8000e80f50000b0034000000eb00c4
:108d4400205a880008003700305a80000000e800ec
:108d5400305a8800305a8000ef0f5000020034006f
:108d64000000eb00305a88004e180700400620002f
:108d740035240700cec2bf00684060000004e00054
:108d840021003a007ffb0700a5cbbf000004e000f0
:108d940009003200415e8000c0f62000e51807009b
:108da4000040eb00a5ebb700e862a800ca82a90066
:108db400c682a9000d003700415e800020c4200057
:108dc400dc18070010c0b300a5ebb700e862a900e7
:108dd4000000eb00906a8800105a80000000e00058
:108de40002003a000000eb00205a88001906070030
:108df4004006200014240700cec2bf006840600073
:108e04000004e000fcff3200005c80000000e00091
:108e140085003a00c3c2bf000044b2000004e00071
:108e24002d003a00a4cbbf000004e00013003a0078
:108e340010c0b300a4ebb7000000eb00e0648800ae
:108e4400505e800000004000f0648800105d8000e7
:108e5400205c88000000eb00105d88000000eb003f
:108e6400305c8800415e800020c42000b1180700f7
:108e7400d31e0700d1a2a900100037000040eb0068
:108e8400a4ebb700b0002000105d8800115d8000e5
:108e940060b92000808040000040eb0080487800ea
:108ea4000040eb00a5ebb700e862a800415e80003b
:108eb400c0f620009f180700d1a2a800e50507000e
:108ec40040062000e0230700c3c2bf000044b200f4
:108ed4000004e000fcff3200c3c2bf0001c8b300bd
:108ee400014060000004e00026003a00a4cbbf006b
:108ef4000004e00023003a00805e80000000e000ef
:108f040006003a00a5cbbf000004e00003003200d5
:108f14000040eb00a5ebb700e862a800105d8000fc
:108f24000000e800105d8800105d8000eb0f500029
:108f340002003400b0002000105d8800105d800045
:108f4400eb0f500004003a00415e8000f0a42000c2
:108f54007818070003003700415e800020c4200019
:108f640074180700bb05070040062000b62307005d
:108f7400c3c2bf0001c8b300014060000004e000a8
:108f8400fbff3200c3c2bf000042b2000004e00095
:108f940025003a00a4cbbf000004e00022003a0000
:108fa400805e80000000e00006003a00a5cbbf0010
:108fb4000004e000030032000040eb00a5ebb70022
:108fc400e862a800105d80000000e900105d8800e0
:108fd400105d80000000e00002003c001000200052
:108fe400105d8800105d8000e10f500004003a001d
:108ff400415e8000c0f620004e18070003003700d1
:10900400415e800020c420004a1807009105070033
:10901400400620008c230700c3c2bf000042b200f8
:109024000004e000fcff3200a4cbbf000004e00019
:109034000100320009fb0700a4cbbf000004e000dc
:109044000c003200a06980000000e00002003a0039
:10905400d1a2a90008003700006580000000e000ec
:1090640002003200d1a2a90003003700d1a2a80057
:1090740001003700d1a2a800b5cbbf000004e00076
:1090840002003a000d13070001003700e311070046
:109094000040eb00920a0700105a8000e10f5000d4
:1090a400f3013200235a8000630798006e00900099
:1090b400e40f500014013200ee009000e48f5000e1
:1090c4000a003c006e019000e20f5100850032005e
:1090d400ee019000e28f5100ab003c006e00900066
:1090e400e10f5000560032000c003700ee009000f3
:1090f400e68f5000620132006e019000e60f5100cd
:1091040030013500ee019000e78f510086013200f6
:109114006e009000e80f5000ad01320061170700a7
:1091240050079800105d80000000e000210032002c
:109134005e0090000000e0000b003400125d80002f
:1091440060b9200000004100104078008040e80031
:1091540060b920000000410001487800415e8000b1
:1091640020c42000f31707005e0090000000e00018
:109174000b003d00125d800060b92000000041003a
:10918400104078008040e90060b9200000004100f0
:1091940001487800415e800020c42000e5170700e4
:1091a40064fc07005e0090000000e0000100320053
:1091b40028050700105d80006700b9008000780072
:1091c400d0c42a0000804000020c070000c2b30093
:1091d400d30b0700115d800060b9200000804000bf
:1091e40010407800be0d0700a0e52a00f90b070027
:1091f400905b80000000e00003003a00f0e52a00e4
:10920400f40b070002003700905b80008e0d07000e
:1092140000c4b300320a0700806980000000e00047
:109224000300320030e62a00ea0b0700a6043700e8
:10923400f7f90700cef9070030fa0700a204370057
:1092440040e72a00e30b070000c4b300240a070028
:1092540014170700500798005e0090000000e0001b
:1092640009003200415e800020c42000b1170700cd
:10927400415d80005e00900000804000405d8800f9
:1092840010002000f0698800415d80004006200045
:10929400808f50000200340040062000405d8800aa
:1092a400405d80000000e00002003d000000eb0093
:1092b400405d8800405d8000801f780050e82a00ef
:1092c400801f780040b2200037dc0700e487570095
:1092d40040b22000bf0b0700405d800096f90700f4
:1092e4007904370080e92a00ba0b070000c4b300f0
:1092f400fb090700eb160700500798005e0090007a
:109304000000e00009003200415e800020c420001b
:1093140088170700315d80005e00900000804000e7
:10932400305d880010002000f0698800315d800005
:1093340040062000808f50000200340040062000c8
:10934400305d8800305d80000000e00002003d00d8
:109354000000eb00305d8800305d8000801f7800e5
:1093640050e82a00801f780040b220000edc07007d
:10937400e487570040b22000960b0700305d800060
:109384005bf907005004370090ea2a00910b0700ac
:1093940000c4b300d2090700c216070050079800a2
:1093a4005e0090000000e000240032001000200065
:1093b400f0698800415e800020c420005d1707002a
:1093c40031bb2000914078005e00900000c0400056
:1093d400b3ebb700b3cbbf00e14f50000c00320039
:1093e400b3cbbf00e24f500009003200b3cbbf0043
:1093f400e34f500006003200b3cbbf00e44f5000ef
:1094040003003200b3cbbf00e54f500005003a0023
:109414000000eb00105d880010002000e06488006c
:10942400671d0700b3cbbf00e24f500002003a00b3
:10943400451807000100370048180700b3cbbf00e8
:109444000004e00002003d000040eb00b3ebb70075
:10945400b3cbbf00e74f50000200340070c0b3002c
:10946400b3ebb700b3cbbf000004e00002003a0046
:10947400a0eb2a00570b0700b3cbbf00e14f50000d
:1094840002003a00b0ec2a00520b0700b3cbbf0035
:10949400e24f500002003a00c0ed2a004d0b0700d5
:1094a400b3cbbf00e34f500002003a00d0ee2a00d5
:1094b400480b0700b3cbbf00e44f500002003a0052
:1094c400e0ef2a00430b0700b3cbbf00e54f500089
:1094d40002003a00f0f02a003e0b0700b3cbbf00b5
:1094e400e64f500002003a0000f22a00390b070050
:1094f400b3cbbf00e74f5000f3033a0020f32a0038
:10950400340b0700f00337000040eb007409070038
:1095140030f42a002f0b070000c4b30070090700c1
:1095240060160700200798002e0090000000e0005d
:1095340016003200415e800020c42000fd160700a2
:10954400605d8000800078002e0090000080400064
:10955400605d880010002000f0698800605d800074
:109564000000e00002003d000000eb00605d8800a8
:10957400605d8000e70f500002003400700020009e
:10958400605d8800605d8000d91c0700605d80001c
:109594004300dd0080007800d0c02a000080400035
:1095a400801f780040f52a00801f780040b2200018
:1095b4007ddb0700e487570040b22000050b07005d
:1095c400c10337000040eb004509070030f62a00cc
:1095d400000b070000c4b30041090700311607005f
:1095e400200798002e0090000000e00016003200d2
:1095f400415e800020c42000ce160700705d80000c
:10960400800078002e00900000804000705d88008b
:1096140010002000f0698800705d80000000e00008
:1096240002003d000000eb00705d8800705d80006a
:10963400e70f50000200340070002000705d8800c5
:10964400705d8000a6190700705d80004300dd0096
:1096540080007800d0c02a0000804000801f78007d
:1096640040f52a00801f780040b220004edb07003e
:10967400e487570040b22000d60a0700920337005f
:1096840040f72a00d30a070000c4b30014090700f6
:10969400041607006500b900500798005e009000aa
:1096a4000000e00009003200415e800020c4200078
:1096b400a0160700815d80005e00900000804000dd
:1096c400805d880010002000f0698800815d8000c2
:1096d40040062000808f5000020034004006200025
:1096e400805d8800815d800010032000808f500021
:1096f40002003c0020032000805d8800805d800023
:10970400801f780050f82a00801f780040b22000a3
:1097140025db0700e487570040b22000ad0a0700ac
:10972400e7fa07006803370060f92a00a90a07006e
:1097340000c4b300ea080700da15070050079800d0
:109744005e0090000000e0000a003200415e8000ec
:1097540020c420007716070021bb20009140780028
:109764005e00900000c04000b2ebb7001000200083
:10977400f0698800b2cbbf00e54f5000020034000e
:1097840050c0b300b2ebb700b2cbbf000004e0009e
:1097940002003d000040eb00b2ebb70070fa2a0073
:1097a4008c0a0700b2cbbf000000fb004200dd00c2
:1097b4008000780010ca2a0000804000850a070053
:1097c40000fb2a00830a0700f6fa07003e0337006d
:1097d40060fb2a007f0a070000c4b300c00807002a
:1097e400b0150700500798005e0090000000e000ec
:1097f4000a003200415e800020c420004d1607009c
:1098040041bb2000914078005e00900000c0400001
:10981400b4ebb70010002000f0698800b4cbbf009f
:10982400e14f5000020034000040eb00b4ebb700fd
:10983400b4cbbf000004e00002003d0010c0b30040
:10984400b4ebb700b4cbbf000004e0000300320067
:1098540070fc2a005f0a07000200370030fd2a006e
:109864005c0a0700aafa070069f807001603370024
:109874000040eb009a080700305a80006101b900eb
:109884000080eb008080eb000201400083814800ef
:1098940072079800030f9800e000200001002000e8
:1098a4007e0190008e099000800f5100818f590035
:1098b40012003e007e0090008e08900000600100bf
:1098c4005300370076003700a1003700c800370086
:1098d400fe003700370137008101370038023700b6
:1098e400ca013700ee013700130237005302370074
:1098f4007a02370090023700c0023700f0fd2a00d8
:10990400340a070000c4b300750807006515070092
:1099140080007800400620000088b90050079800b5
:109924005e0090000000e0002600320010002000dd
:10993400006a8800505e80000000e00006003a00e3
:109944005e0090000000e00003003400800c200062
:10995400505e880015003700515e8000800c2000a6
:10996400808f500006003a005e0090000000e00086
:1099740003003d000000eb00505e88000b00370040
:10998400505e80000000e00004003a005e00900099
:109994000000e00001003d0004003700505e80003c
:1099a400de00900001004000505e8800515e80009f
:1099b40000712200808f50000200360000712200e6
:1099c400505e8800505e80000000e00005003a0010
:1099d40041b2200002ff2a0012000900b2587800a8
:1099e40008003700505e800001002000809fbe0008
:1099f40030002b00801f780040b220006ada070094
:109a0400e687570040b22000f2090700ae02370093
:109a140060012b00ef09070000c4b3003008070001
:109a240020150700500798005e0090000000e00039
:109a34001100320010002000006a8800915e80004e
:109a44005e00900000804000905e8800915e80007f
:109a5400f00d2000808f500002003400f00d200033
:109a6400905e8800905e80000000e00002003d00ef
:109a74000000eb00905e8800905e8000801f7800fc
:109a840070022b00801f780040b2200046da0700e5
:109a9400e487570040b22000ce0907008a0237004d
:109aa4000040eb000e080700a0032b00c9090700c3
:109ab40000c4b3000a080700fa140700200798003e
:109ac4002e0090000000e00016003200415e80008d
:109ad40020c4200097150700b5cbbf008040780054
:109ae4002e00900000c04000b5ebb700100020002d
:109af400f0698800b5cbbf000004e00002003d001f
:109b04000040eb00b5ebb700b5cbbf00e14f500010
:109b14000200340010c0b300b5ebb7001000200001
:109b2400f0698800b5cbbf000004e00002003a00f1
:109b3400b0042b00a7090700b5cbbf00e14f5000cc
:109b440061023a00c0052b00a20907005e0237003b
:109b540043b22000d0062b0010000900b059780051
:109b640040b220009b09070000c4b300dc070700d3
:109b7400cc140700500798005e0090000000e0003d
:109b84001100320010002000006a8800415e80004d
:109b94005e00900000804000405e8800405e8000cf
:109ba4000000e00002003d000000eb00405e880081
:109bb400415e800040062000808f50000200340087
:109bc40040062000405e8800405e8000801f7800d0
:109bd400e0072b00801f780040b22000f2d9070074
:109be400e487570040b220007a09070036023700a4
:109bf400f0082b007709070085f7070000c4b300bd
:109c0400b7070700a7140700500798005e009000ec
:109c14000000e0002200320010002000006a8800ea
:109c2400e25d8000f35d80005e009000cf80de0086
:109c34000200400083804800e05d8800f15d8800f8
:109c4400e05d8000f15d80000001be00f0f32100c2
:109c540001002000800f5100818f590004003e0054
:109c640000f4210001002000e05d8800f15d88001f
:109c7400e05d8000f15d80000001be00802c2300c7
:109c840001002000800f5100818f5900040036002c
:109c9400802c230001002000e05d8800f15d880035
:109ca400e05d8000f15d8000809fbe00b0092b0064
:109cb400801f780040b22000bbd90700e687570018
:109cc40040b2200043090700ff013700c00a2b00ff
:109cd4004009070026f70700d0cb2a003d090700fa
:109ce40000c4b3007e0707006e1407006a00b900c1
:109cf400500798005e0090000000e000220032004f
:109d040010002000006a8800c25d8000d35d8000de
:109d14005e009000cf80de00020040008380480097
:109d2400c05d8800d15d8800c05d8000d15d800089
:109d34000001be00f076210001002000800f5100d8
:109d4400818f590004003e000077210001002000ab
:109d5400c05d8800d15d8800c05d8000d15d800059
:109d64000001be000071220001002000800f51009c
:109d7400818f590004003600007122000100200088
:109d8400c05d8800d15d8800c05d8000d15d800029
:109d9400809fbe00b0092b00801f780040b22000d5
:109da40081d90700e687570040b22000090907005f
:109db400c5013700700b2b0006090700105d8000f9
:109dc400ea0f500003003a00200c2b0001090700a1
:109dd40009003700b05b8000c15b8000691a07008e
:109de40050079800710720005e009000f9090700f1
:109df400900c2b00f708070000c4b30038070700d5
:109e040028140700500798005e0090000000e0004e
:109e14002800320010002000006a8800005e8000e4
:109e2400115e80000004be005e009000cf80de0062
:109e340063e50700a2702d0033c223002ae5070062
:109e44000001be000800be00cae40700005e8800ee
:109e5400115e8800005e8000115e80000200200018
:109e640003f0230081e507000000e0000100350055
:109e7400040037000000200001f02300005e880089
:109e8400115e8800005e8000115e800002002000e8
:109e940003fc230048e507000000e00001003c004b
:109ea400040037000000200001fc2300005e88004d
:109eb400115e8800005e8000115e8000809fbe00fd
:109ec400c00c2b00801f780040b2200036d9070058
:109ed400e687570040b22000be0807007a01370029
:109ee400100e2b00bb080700105d8000ea0f500025
:109ef4000a003a00b05b8000c15b8000211a0700b1
:109f040050079800710720005e009000b109070017
:109f1400900c2b00af08070002003700200c2b0028
:109f2400ac08070000c4b300ed060700dd1307000a
:109f3400500798005e0090000000e0002800320006
:109f440010002000006a8800205e8000315e8000de
:109f54000004be005e009000cf80de0018e507001c
:109f6400a2702d0033c22300dfe407000001be000d
:109f74000800be007fe40700205e8800315e880090
:109f8400205e8000315e80000200200003f0230088
:109f940036e507000000e00001003500040037004a
:109fa4000000200001f02300205e8800315e88005c
:109fb400205e8000315e80006266260063fe23001e
:109fc400fde407000000e00001003c00040037004d
:109fd4006066260061fe2300205e8800315e8800f2
:109fe400205e8000315e8000809fbe00c00c2b008c
:109ff400801f780040b22000ebd80700e6875700a6
:10a0040040b22000730807002f013700c00e2b0058
:10a014007008070000c4b300b1060700a1130700cd
:10a02400500798005e0090000000e000110032002c
:10a0340010002000006a8800615e80005e009000cd
:10a0440000804000605e8800605e80000000e000e8
:10a0540002003d000000eb00605e8800615e80004d
:10a06400803e2000808f500002003400803e20009b
:10a07400605e8800605e800000004000801f780001
:10a08400d00f2b00801f780040b22000c6d80700f4
:10a09400e487570040b220004e0807000a01370049
:10a0a400f0102b004b08070000c4b3008c06070017
:10a0b4007c130700500798005e0090000000e00049
:10a0c4001100320010002000006a8800715e8000d8
:10a0d4005e00900000804000705e8800705e80002a
:10a0e4000000e00002003c0010002000705e8800c8
:10a0f400715e8000803e2000808f5000020034009a
:10a10400803e2000705e8800715e80002003200085
:10a114000088b900801f780000122b00801f78008f
:10a1240040b22000a0d80700e487570040b22000c6
:10a1340028080700e400370020132b002508070037
:10a1440000c4b300660607005613070050079800c2
:10a154005e0090000000e0001000320010002000bb
:10a16400006a8800815e80005e00900000804000ec
:10a17400805e8800805e80000000e00002003d00f8
:10a184000000eb00805e8800805e8000e10f5000dc
:10a194000200340010002000805e8800805e800091
:10a1a4000000e00003003a0030142b000908070007
:10a1b400c500370040152b0006080700c200370011
:10a1c40050162b000308070000c4b3004406070020
:10a1d400b05b8000c15b80006a19070050079800db
:10a1e400710720005e009000fa08070060172b003a
:10a1f400f8070700d05b8000e15b8000611907006d
:10a2040050079800710720005e009000f1080700d5
:10a2140090172b00ef070700a05b80000000e00010
:10a2240003003a00f0e52a00ea070700a600370019
:10a23400a05b800084090700a3003700d0172b001f
:10a24400e407070000c4b30025060700e0182b004c
:10a25400e0070700b3cbbf000004e00003003a00ae
:10a2640040192b00db0707000200370090192b0070
:10a27400d8070700d91e0700204798000000eb000c
:10a28400000f78000f0037002e4090000080fb0084
:10a294004300de00610060000004e00003003200bf
:10a2a40010c3b3009e0707000200370000c3b300c9
:10a2b4009b0707002e409000004040002047980074
:10a2c4001e0fe800310020009e8f1000eeff3400c6
:10a2d40090172b00bf0707007b003700006b80003e
:10a2e40001002000809fbe00e0192b00801f780031
:10a2f40040b220002cd80700e687570040b2200067
:10a30400b407070000c4b300f5050700d06a800055
:10a3140001002000809fbe00101b2b00801f7800ce
:10a3240040b2200020d80700e687570040b2200042
:10a33400a807070064003700401c2b00a50707008e
:10a34400d812070080007800e06980000080400097
:10a35400e069880000c4b300e1050700e0698000fb
:10a36400e80f50001b00340042b22000531d2b00a4
:10a37400100009003359780040b220009507070007
:10a384000000eb00e0698800405e80006a00b900cc
:10a3940080007800c0f62000661307003b02070027
:10a3a4000000eb00f06988000000eb00006a880000
:10a3b4000000eb00205a88000000eb00305a8800af
:10a3c4000000eb00105a8800007d20009e1e07004c
:10a3d4003d003700e0698000801f7800601e2b007c
:10a3e400801f780040b22000efd70700e4875700b1
:10a3f40040b22000770707003300370080e32a00cb
:10a4040074070700a712070080007800d069800055
:10a4140000804000d069880000c4b300b005070084
:10a42400d0698000e80f50001e00340040b22000c4
:10a43400811f2b00100009003158780040b2200021
:10a44400640707000000eb00d0698800405e8000cc
:10a454006a00b90080007800c0f6200035130700b8
:10a46400260007007b0007002c010700c20007003c
:10a474000000eb00f06988000000eb00006a88002f
:10a484000000eb00205a88000000eb00305a8800de
:10a494000000eb00105a8800007d20006a1e0700af
:10a4a40009003700d0698000801f7800601e2b00ef
:10a4b400801f780040b22000bbd70700e487570014
:10a4c40040b2200043070700c8c2bf0068406000d4
:10a4d4000004e00006003200a5cbbf000004e00049
:10a4e4000300320010002000005c8800d3f837001d
:10a4f4000000eb00005c8800d0f837000200fa008e
:10a504000000eb00000f7800060037009e00780082
:10a5140060b92000808040000040eb008048780053
:10a524001e0fe800b00020009e0f1000f7ff34005b
:10a53400b0002000105d88000040eb00a4ebb700e1
:10a544000040eb00a5ebb70020032000305d88003d
:10a5540020032000405d880010002000505d88002a
:10a5640030002000605d880030002000705d8800ad
:10a574000040eb00b3ebb700a0052000805d88002d
:10a5840040c0b300b2ebb7000040eb00b4ebb7003f
:10a5940010c0b300b5ebb70000f4210001002000a7
:10a5a400c05d8800d15d8800b097220001002000c2
:10a5b400e05d8800f15d88000000200001f82300c0
:10a5c400005e8800115e88000000200001fa23006c
:10a5d400205e8800315e880020032000405e8800f1
:10a5e400803e2000505e880020032000605e8800ca
:10a5f40040002000705e88000000eb00805e880050
:10a604000000eb00905e88001300200082b8200058
:10a61400010f2f00f00720001a1d0700405c800086
:10a624000000e800405c880012002000010f2f00a9
:10a63400f0072000201d070013002000020f2f0048
:10a64400f107200080b820003c1d07000080fa00bc
:10a65400000006000400fa000000eb001007980058
:10a664001a0037001e0090000000400080007800af
:10a6740000002f008080400012002000f00720001e
:10a684000d1d0700000f78001e0090000000400020
:10a694008000780000002f00008140001e00900020
:10a6a400000040008000780060b920000080400075
:10a6b40013002000f1072000201d0700000f780080
:10a6c4001e0090000000e800100798001e00900093
:10a6d400e70f5000e3ff3600b5cbbf000004e000f5
:10a6e40008003a001e007800801f78001e009000c9
:10a6f400801f7800a0202b00801f78001cd7070043
:10a70400e68757000080fa00000006000400fa0003
:10a714000000eb0010079800110037001e009000a5
:10a72400000040008000780060b9200000814000f3
:10a734001e009000000040008000780000002f0000
:10a744008080400013002000f0072000cd1c07008b
:10a75400000f78001e0090000000e8001007980029
:10a764001e009000e70f5000ecff36000000eb00e5
:10a774000080fa00000006000400fa000000eb006c
:10a78400b05d88000000eb00100798002900370036
:10a794001e009000e70f500009003e00b25d8000eb
:10a7a4001e0090008000400060ba2000008040003d
:10a7b4001000780000004100b05d880003003700fd
:10a7c400b05d80000000ea00b05d88001e009000cb
:10a7d400000040008000780000022f0080804000cc
:10a7e40012002000f0072000b31c0700000f7800bf
:10a7f4001e009000000040008000780000022f003e
:10a80400008140001e00900000004000800078009d
:10a8140060ba20000080400013002000f1072000ef
:10a82400c61c0700000f78001e0090000000e8001e
:10a83400100798001e009000e80f5000d4ff360067
:10a84400b5cbbf000004e0000a003a00b05d800010
:10a85400801f78001e007800801f78001e00900082
:10a86400801f7800e0222b00801f7800c0d60700ec
:10a87400e88757000080fa00000006000600fa008e
:10a884000000eb00000f78000000eb0020079800a8
:10a89400170037002e009000000040008000780070
:10a8a40060ba2000008140002e00900000004000ab
:10a8b4008000780000022f008080400013002000f8
:10a8c400f00720006f1c0700100798002e0090006e
:10a8d4008000400060ba2000008040001000780032
:10a8e4001e0f40002e0090000000e8002007980092
:10a8f4002e009000e80f5000e6ff36001300200001
:10a9040082b82000010f2f00f00720005d1c070013
:10a914001e0078000080fa00000006000400fa001f
:10a924000000eb00a05e88000000eb001007980018
:10a93400290037001e009000ed0f500009003e0072
:10a94400a25e80001e0090008000400080bb2000ba
:10a95400008040001000780000004100a05e8800e4
:10a9640003003700a05e80000000ea00a05e8800bb
:10a974001e009000000040008000780000042f00ba
:10a984008080400012002000f00720004a1c0700cd
:10a99400000f78001e009000000040008000780046
:10a9a40000042f00008140001e00900000004000c1
:10a9b4008000780080bb200000804000130020004d
:10a9c400f10720005d1c0700000f78001e009000b6
:10a9d4000000e800100798001e009000ee0f5000e1
:10a9e400d4ff3600b5cbbf000004e0000a003a00f3
:10a9f400a05e8000801f78001e007800801f780011
:10aa04001e009000801f780070252b00801f7800a6
:10aa140057d60700e88757000080fa0000000600b8
:10aa24000600fa000000eb00000f78000000eb00c5
:10aa340020079800170037002e0090000000400007
:10aa44008000780080bb2000008140002e00900030
:10aa5400000040008000780000042f008080400047
:10aa640013002000f0072000061c070010079800c0
:10aa74002e0090008000400080bb20000080400039
:10aa8400100078001e0f40002e0090000000e80027
:10aa9400200798002e009000ee0f5000e6ff3600cd
:10aaa4001e0078000080fa00000006000400fa008e
:10aab4000000eb00305f88000000eb0010079800f6
:10aac400290037001e009000e70f500009003e00e7
:10aad400325f80001e0090008000400060bd2000b6
:10aae400008040001000780000004100305f8800c2
:10aaf40003003700305f80000000ea00305f880008
:10ab04001e009000000040008000780000082f0024
:10ab14008080400012002000f0072000e61b0700a0
:10ab2400000f78001e0090000000400080007800b4
:10ab340000082f00008140001e009000000040002b
:10ab44008000780060bd20000080400013002000d9
:10ab5400f1072000f91b0700000f78001e00900089
:10ab64000000e800100798001e009000e80f500055
:10ab7400d4ff3600b5cbbf000004e0000a003a0061
:10ab8400305f8000801f78001e007800801f7800ee
:10ab94001e009000801f780070252b00801f780015
:10aba400f3d50700e88757000080fa00000006008c
:10abb4000600fa000000eb00000f78000000eb0034
:10abc40020079800170037002e0090000000400076
:10abd4008000780060bd2000008140002e009000bd
:10abe400000040008000780000082f0080804000b2
:10abf40013002000f0072000a21b07001007980094
:10ac04002e0090008000400060bd200000804000c5
:10ac1400100078001e0f40002e0090000000e80095
:10ac2400200798002e009000e80f5000e6ff360041
:10ac34001e0078000080fa00000006000000fa0000
:10ac4400c05d8000d15d8000b05e8800c15e880078
:10ac5400e05d8000f15d8000d05e8800e15e8800e8
:10ac6400005e8000115e8000f05e8800015f880055
:10ac7400205e8000315e8000105f8800215f8800c4
:10ac84008aff07000080fa00000006000200fa00b4
:10ac9400c7ff0700000f78001e00e00015003a000f
:10aca40010282b00801f7800b1d507008f87e9009a
:10acb400b05e8000c15e8000c05d8800d15d880008
:10acc400d05e8000e15e8000e05d8800f15d880078
:10acd400f05e8000015f8000005e8800115e8800e5
:10ace400105f8000215f8000205e8800315e880054
:10acf40014003700502a2b00801f78009cd50700d1
:10ad04008f87e90000f4210001002000c05d880065
:10ad1400d15d8800b097220001002000e05d88002a
:10ad2400f15d88000000200001f82300005e880027
:10ad3400115e88000000200001fa2300205e8800d4
:10ad4400315e8800f5fe07000080fa00000006006e
:10ad54000600fa00002d2b00801f780084d5070020
:10ad64008f87e9000000eb00100798001b003700f4
:10ad74009e00900000002f00808040006401470086
:10ad840013002000f00720003e1b0700000f78008e
:10ad94001e0090006f0060000000e00006003a0012
:10ada4001e009000801f7800702e2b00801f7800fa
:10adb4006fd50700e48757002e009000801f7800ad
:10adc400f02e2b00801f780069d50700e487570018
:10add4001e0090000080e800100798009e0090007c
:10ade400f00f2000808f5000e1ff34001e00780037
:10adf400801f7800402f2b00801f78005cd507004f
:10ae0400e48757000080fa00000006000000fa0002
:10ae14001300200082be2000810f2f00f0072000c5
:10ae2400181b070013002000a2be2000a10f2f0052
:10ae3400f0072000131b0700415f8000f0092f007a
:10ae4400808f500004003600415f8000800e2f0088
:10ae5400808f500002003600000a2f00405f8800f7
:10ae64000080fa00000006000200fa001200200030
:10ae7400810f2f00f00720000f1b0700000f780040
:10ae840013002000820f2f00f107200080be200055
:10ae94002a1b0700000f780012002000a10f2f00ca
:10aea400f0072000041b0700000f780013002000a7
:10aeb400a20f2f00f1072000a0be20001f1b0700d7
:10aec400000f78000080fa00000006000600fa0077
:10aed400200798000000eb001007980011003700cd
:10aee4001e0090000000400080007800c0be2000da
:10aef400008140001e0090000000400080007800a7
:10af04002e0090008080400013002000f0072000f5
:10af1400dc1a0700000f78001e0090000000e80013
:10af2400100798001e009000e30f5000ecff36005d
:10af34000080fa00000006000800fa0030079800bc
:10af44000000eb00200798000000eb0010079800b9
:10af5400160037001e0090000000400080007800ba
:10af64003e0090008080400012002000f007200086
:10af7400d11a0700000f78001e0090000000400066
:10af8400800078003e00900000814000640047008b
:10af940013002000f1072000e81a0700000f7800d2
:10afa4001e0090000000e800100798001e009000aa
:10afb400e30f5000e7ff36000080fa0000000600af
:10afc4000200fa000000eb00000f780012002000dd
:10afd400a10f2f00f0072000b71a0700130020006c
:10afe400a20f2f00f10720000e007800d31a0700eb
:10aff400000a2f00000f780012002000810f2f009c
:10b00400f0072000ac1a070013002000820f2f0065
:10b01400f10720000e007800c81a0700000a2f006c
:10b02400000f7800050037001e007800c2ff0700fb
:10b034001e00780068004000000f78009e00780031
:10b04400f00e2f00808f5000f7ff36000080fa00ca
:10b05400000006000600fa0020079800ae009000e9
:10b06400f0092f00808f500004003600ae009000dd
:10b07400800e2f00808f5000070036002e009000b5
:10b08400801f7800e0302b00801f7800b8d40700c0
:10b09400e4875700200037000000eb0010079800f9
:10b0a4001a0037001e009000000040008000780065
:10b0b4002e0090008080400012002000f007200045
:10b0c4007d1a0700000f78001e0090000000400069
:10b0d400800078002e009000008140001e00900047
:10b0e4000000400080007800c0be200000804000c6
:10b0f40013002000f1072000901a0700000f7800c9
:10b104001e0090000000e800100798001e00900048
:10b11400e30f5000e3ff36000080fa000000060051
:10b124000a00fa00889fbe00004f9800b5cbbf000c
:10b134000004e0001f003a00905c8000815c800005
:10b14400325b8000135b8000801f7800811f7800d1
:10b15400821f7800831f780040332b00801f780003
:10b1640083d40700ea875700a05c8000cf80de000c
:10b1740093e007000200200003122400cce0070043
:10b184000004be00705a8000cf80de008ce007000f
:10b194000200200003122400c5e00700889fbe00bf
:10b1a400809fbe0030372b00801f780070d40700ca
:10b1b400ea875700815c8000c07f2000808f5000a8
:10b1c40003003600f01f200020079800030037001a
:10b1d400805c80004200de0020079800915c8000c3
:10b1e400e00f2000808f500003003600f00720009d
:10b1f4001007980003003700905c80000000d10025
:10b20400100798001e009000c900dd002e00900079
:10b2140080804000c0be200001087800115d8000dd
:10b2240060b9200000804000104078000040e80031
:10b234004400dd0060479800105d8000ef4060002e
:10b244006e40900000c0700060479800c0be2000af
:10b25400ee40900031409800405a80004200de00e9
:10b2640080407800c0be200021409800715a8000c0
:10b27400a05c8000808f500003003400705a80006e
:10b28400000f780002003700a15c8000010f7800f5
:10b29400f01f20009e0f100004003400c1be2000e7
:10b2a40000c0eb00d0409800050037001e00780075
:10b2b4000080d10080407800c0be2000514098003a
:10b2c400f05a800080407800c0be200041409800c1
:10b2d400c0be20008e48900071409800a4cbbf00ef
:10b2e400e14f500006003a00c0be200070409000bc
:10b2f400804078000104a000c0be20007140980086
:10b30400c8c2bf00614060000004e00006003200d3
:10b31400c0be200070409000804078000144a0002e
:10b32400c0be200071409800c8c2bf0062406000e7
:10b334000004e00006003200c0be2000f04090008f
:10b3440000c2b30080c07000c0be200071409800ed
:10b354004f04be000080fa00000006000400fa005a
:10b36400889fbe00d0002000d31a0700505c8800dc
:10b37400c0002000d01a0700605c88009000200004
:10b38400cd1a0700705c8800505c800036140700fa
:10b39400008fbe001e00be00fa140700805c880007
:10b3a400605c800030140700008fbe001e00be00e9
:10b3b400f4140700905c8800705c80006103b8009e
:10b3c400c25d8000d35d80000234b80003b0b900d0
:10b3d40009027800000242000790b900000242000e
:10b3e4008404780040c8de00cf80de00a05c8800c2
:10b3f4004f04be000080fa00000006000200fa00bc
:10b40400004f7800d5ff070080fe07001e4078003b
:10b4140043ff0700405f80000eff0700b5cbbf006d
:10b424000004e00009003a00505f80000000e800da
:10b43400415f8000801f7800811f7800503b2b0003
:10b44400801f7800cad30700e6875700405f80005a
:10b4540068004000405f8800415f8000800e2f003c
:10b46400808f500002003600000a2f00405f8800e1
:10b47400505f80000000e800505f88007afe0700fb
:10b484000080fa00000006001a00fa00881f780005
:10b4940060079800c0be200090007800f01f2000d4
:10b4a400008060004200dd0050079800c0be20000c
:10b4b400100078004900de000000400040079800ba
:10b4c400c0be2000204490000800fb00cf80de00b6
:10b4d400bbdf070070079800010f98000804e00024
:10b4e40007003d0002002000033824007e00900085
:10b4f4008e0890001fdf070070079800010f980066
:10b504007e0090008e089000200798003107980074
:10b51400d2cc2c00c3ec23002e009000be0090007f
:10b5240071df07002007980031079800c0be200093
:10b53400504490000800fb00cf80de00a0df07002d
:10b54400100f9800210f98000804e00007003d0048
:10b5540002002000033824001e089000ae0890006a
:10b5640004df0700100f9800210f98001e099000b7
:10b57400ae099000028fbe00d2cc2c00c3e423009d
:10b584001e00be0058df0700008fbe00ee019000d1
:10b59400831f7800e03d2b00801f780074d30700e0
:10b5a400e48757005e009000801f7800203f2b0046
:10b5b400801f78006ed30700e4875700ce00900008
:10b5c400811f780050402b00801f780068d307004b
:10b5d400e487570080412b00801f780064d3070064
:10b5e4008f87e900c0be2000304090000080fb003f
:10b5f4006f0060006101b900320f9800430f98009a
:10b60400b0002000010020003e099000ce09900007
:10b61400800f5100818f59000f003e003e089000ba
:10b62400ce089000006001001000370014003700bd
:10b63400180037001c0037002000370024003700b2
:10b64400280037002c003700300037003400370062
:10b65400380037003c00370000422b00801f780080
:10b6640043d307008f87e9003b00370040422b009b
:10b67400801f78003ed307008f87e900360037002b
:10b6840080422b00801f780039d307008f87e900a0
:10b6940031003700c0422b00801f780034d30700ec
:10b6a4008f87e9002c00370000432b00801f7800af
:10b6b4002fd307008f87e9002700370040432b0072
:10b6c400801f78002ad307008f87e9002200370003
:10b6d40080432b00801f780025d307008f87e90063
:10b6e4001d003700c0432b00801f780020d30700c3
:10b6f4008f87e9001800370000442b00801f780072
:10b704001bd307008f87e9001300370040442b0048
:10b71400801f780016d307008f87e9000e003700da
:10b7240080442b00801f780011d307008f87e90025
:10b7340009003700c0442b00801f78000cd3070099
:10b744008f87e9000400370000452b00801f780034
:10b7540007d307008f87e900c0be20003040900067
:10b764000080fb004400de000080fb00801f7800a6
:10b7740040452b00801f7800fdd20700e487570066
:10b784002e019000be019000829fbe0030462b0027
:10b79400801f7800f6d20700e68757001e00be001f
:10b7a400809fbe0090472b00801f7800f0d20700d6
:10b7b400e6875700c0be2000404090000080fb0098
:10b7c400801f7800f0482b00801f7800e8d2070023
:10b7d400e4875700c0be2000704090000080fb004a
:10b7e400801f7800204a2b00801f7800e0d20700d9
:10b7f400e4875700c0be2000704090000004e000c1
:10b8040004003d00704b2b00801f7800d8d2070045
:10b814008f87e900c0be2000704090000080fb00cc
:10b824004400de00610060000004e0000400320017
:10b83400604c2b00801f7800cdd207008f87e90071
:10b84400c0be2000704090000080fb004500de0078
:10b85400610060000004e00004003200f04c2b00a2
:10b86400801f7800c2d207008f87e900c0be200085
:10b87400704090000080fb004600de006100600024
:10b884000004e00004003200804d2b00801f78008b
:10b89400b7d207008f87e900c0be20007040900037
:10b8a4000080fb00610060000004e000040032003e
:10b8b400004f2b00801f7800add207008f87e9006e
:10b8c400c0be2000704090000004e000040032007c
:10b8d400c0be200070409000e14f400004003a00d8
:10b8e40020502b00801f7800a1d207008f87e90029
:10b8f4004f0478000080fa00000006000600fa00f9
:10b9040042fd0700405f80002007980060ff2f0081
:10b91400000f780000512b00801f780094d207009c
:10b924008f87e9001e007800100798002400370074
:10b934001e009000801f7800d0532b00801f7800d9
:10b944008bd20700e48757001e0090009e0f500022
:10b9540004003a00c0552b00801f780084d20700f1
:10b964008f87e9001e009000e10f400004003a00b8
:10b97400a0562b00801f78007dd207008f87e90036
:10b984002e00900051fd07002e009000befe07001f
:10b994002e0090006800400020079800ae00900040
:10b9a400800e2f00808f500002003600000a2f0006
:10b9b400200798001e0090000000e800100798007f
:10b9c4001e0090000000e000d9ff350080572b00d6
:10b9d400801f780066d207008f87e900405f8000ef
:10b9e400515f8000801f7800811f7800405a2b002f
:10b9f400801f78005ed20700e68757000080fa00b7
:10ba0400000006000200fa00004f78000900fc0064
:10ba1400b1168000f00f2000008160001e80fb0042
:10ba24004800dd008000780000f02f0000806000f6
:10ba340000007100b016880010002000ee18070006
:10ba4400d6a2a80010002000eb180700d6a2a90077
:10ba540010002000e81807000080fa00000006002b
:10ba64000200fa0000002800000f78000400fc0027
:10ba74009116800000f02f0000807000901688005e
:10ba8400d6c2a800d6e2a9000900370010002000a1
:10ba9400d9180700d6a2a80020002000d618070055
:10baa400a116800000f02f00008f6000d6a2a9002c
:10bab4001e0078000000e000f4ff3500d6c2a900a3
:10bac400d6e2a8000400fc0090168000f10f2000cc
:10bad40001006000901688000080fa000000060053
:10bae4000200fa00004f7800ddff0700d6e2a9004b
:10baf40000c8b3001e407000c2ff0700d6e2a800d1
:10bb04000080fa00000006000000fa00d4ff0700dd
:10bb1400d6e2a90010c0b300baff0700d6e2a8001d
:10bb24000080fa00000006000000fa00d6e2a90036
:10bb3400d6c2a900f0002000c318070080c3b300d8
:10bb4400b0ff070050002000bf18070080c3b300f7
:10bb5400acff070010002000bb18070080c3b3002f
:10bb6400a8ff070010002000b7180700c0c0b300ea
:10bb7400a4ff070010002000b318070010c0b30092
:10bb8400a0ff070020002000af18070060c0b3002a
:10bb94009cff070010002000ab180700d6e2a800a5
:10bba4000080fa00000006000200fa00004f78004e
:10bbb400abff07001e40780092ff07000080fa00e8
:10bbc400000006000200fa00004f780011479800b8
:10bbd400a3ff0700d6e2a900f0c3b3001e4f600024
:10bbe40000c4b3001e40700086ff0700d6e2a80020
:10bbf4009bff07001e40900082ff0700c2ff070062
:10bc04000080fa00000006000400fa0020479800b3
:10bc1400314798000040eb00004f780004003700e3
:10bc24008fff07002e40900076ff07001e4fe800ac
:10bc34003e4090009e4f1000f9ff35000080fa004e
:10bc4400000006000000fa0085ff0700d6e2a90004
:10bc540000c4b3006bff0700d6e2a80011c0b30014
:10bc64000040eb00e8ff070051c0b30000c1b3007f
:10bc7400e5ff070021c0b3000040eb00e2ff07002e
:10bc840011c0b3000040eb00dfff070051c0b30058
:10bc940040c1b300dcff070021c0b3000040eb004b
:10bca400d9ff070011c0b3000040eb00d6ff070026
:10bcb40051c0b30050c1b300d3ff070021c0b3008b
:10bcc4000040eb00d0ff070011c0b3000040eb00c0
:10bcd400cdff070051c0b30010c0b300caff070076
:10bce40021c0b3000040eb00c7ff070011c0b30040
:10bcf40080c0b300c4ff070011c0b30040c1b3004b
:10bd0400c1ff070011c0b30080c0b300beff07002d
:10bd140051c0b3000040eb00bbff070021c0b300db
:10bd24000040eb00b8ff070011c0b30000c1b3002e
:10bd3400b5ff070011c0b3000040eb00b2ff0700dd
:10bd440011c0b30000c1b300afff070031c0b3009e
:10bd54000040eb00acff070031c0b3000040eb0033
:10bd6400a9ff070011c0b30000c1b300a6ff07007c
:10bd740041c0b3000040eb00a3ff070021c0b300a3
:10bd84000040eb00a0ff070031c0b30000c1b300c6
:10bd94009dff070031c0b3000040eb009aff07008d
:10bda40059ff07000080fa00000006001200fa00a4
:10bdb400000f98008e08900000032000808f500030
:10bdc4000200340000032000000f98000e089000c9
:10bdd40062002000110009000200d800200798002a
:10bde4000e08900062002000110009000200d80033
:10bdf4008000fd00100798000000eb00000f7800a1
:10be04000000eb00300798000c0037001e0178009a
:10be1400be009000c0c12b0000804000904078001c
:10be24006800470000004100014878001e0fe80048
:10be34003e0090000000e800300798003e009000ab
:10be4400e70f5000f1ff34000000eb00000f780012
:10be5400090037009e007800680047008080400099
:10be640020c0b300804878001e0fe8002e00900028
:10be74000000e900200798002e0090000000e00078
:10be8400f4ff3c001e0090000000e00008003400b5
:10be94001e0178009e00900000c12b00008040002d
:10bea4009040780068004700000041000148780095
:10beb4000000eb003007980008003700be00900037
:10bec40068004700008040001040780036ff0700fb
:10bed4003e0090000000e800300798003e0090000b
:10bee400e70f5000f5ff34000080fa000000060060
:10bef4001600fa00100f9800210f98009e08900079
:10bf040000032000808f5000020034000003200052
:10bf1400100f980080002000100798001e08900061
:10bf240062002000110009000200d80030079800c8
:10bf34001e08900062002000110009000200d800d1
:10bf44008000fd00200798002e0890000000e0000b
:10bf540032003a000000eb00000f78000c003700bc
:10bf64009e0078006a0047008080400020c0b30033
:10bf7400804878001e0fe8003e0090000000e900b1
:10bf8400300798001e0090000000e9001007980098
:10bf94003e0090000000e000f1ff3c002e00900005
:10bfa4000000e0000c0034001e017800ae00900098
:10bfb40000c12b0000804000904078006a004700d8
:10bfc40000004100014878001e0fe8001e009000a8
:10bfd4000000e900100798000000eb0040079800fb
:10bfe400090037009e0078006a0047008080400006
:10bff40000c2b300804878001e0fe8004e00900095
:10c004000000e80040079800ce0090001e00900059
:10c01400808f5000f3ff350031003700700020009e
:10c02400000f78000c0037009e0078006a0047007b
:10c034008080400020c0b300804878001e0fe900d3
:10c044003e0090000000e900300798001e009000b8
:10c054000000e900100798003e0090000000e00096
:10c06400f1ff3c002e0090000000e0000c003400c2
:10c074001e017800ae00900060c12b0000804000db
:10c08400904078006a0047000000410001487800b1
:10c094001e0fe9001e0090000000e9001007980040
:10c0a4000000eb0040079800090037009e0078006c
:10c0b4006a0047008080400000c2b30080487800d6
:10c0c4001e0fe9004e0090000000e80040079800b1
:10c0d400ce0090001e009000808f5000f3ff3500ca
:10c0e4000000eb004007980008003700ce009000e5
:10c0f4006a0047000080400010407800aafe070054
:10c104004e0090000000e800400798004e009000a8
:10c11400e70f5000f5ff34000080fa00000006002d
:10c124000200fa00004f78001e4078009efe0700cf
:10c134000080fa00000006000400fa00204798007e
:10c144002e409000004f78002e4090000080fb00ad
:10c154004400de00204798002e409000e94f500034
:10c1640004003e002e4090000043b0002047980099
:10c17400030037002e4090007043b0002047980021
:10c184002e40900088fe07001e407800204798004b
:10c194002e4090006f406000204798002e40900091
:10c1a400e94f500004003e002e4090000043b000d0
:10c1b40020479800030037002e4090007043b000e1
:10c1c400204798002e40900077fe07000080fa0078
:10c1d400000006000200fa008e0078008008780053
:10c1e400080037000e007800100078001040780036
:10c1f4006dfe07008e0078000e00780010017800b4
:10c20400e10841000e00780010007800104078002a
:10c214000004e000f3ff3a000080fa00000006008a
:10c224000600fa00008fbe00424798004e4090007e
:10c234000004e00030003a001e00be0002a02c0002
:10c24400a3b923008bdc07000043b00056fe0700af
:10c254001e00be0002a02c00a3b9230085dc070049
:10c264000003be0000a02c000032b800a0b92300d7
:10c2740000b0b900050178000001410000a02c00c5
:10c2840000b8b90000014100820278001e1f1200ac
:10c294001e971a00e0c2b30043fe07001e00be0052
:10c2a40002102e00535f200072dc07000043b00030
:10c2b4003dfe07001e00be0002102e00535f20004a
:10c2c4006cdc07000003be0000102e000032b80032
:10c2d400505f200000b0b900050178000001410062
:10c2e40000102e0000b8b90000014100820278005d
:10c2f4001e1f12001e971a004e4090000004e0001a
:10c304000e003200f0672900810920003e01400040
:10c31400ae8148000200be000001be00e0cf220052
:10c3240011132000800f5100818f590003003e003b
:10c3340000c2b3001cfe0700060037001e00be004a
:10c3440002682900830920004adc07000043b0008a
:10c3540015fe07001e00be000268290083092000a4
:10c3640044dc07000003be00006829000032b80066
:10c374008009200000b0b9000501780000014100e7
:10c384000068290000b8b900000141008202780069
:10c394001e1f12001e971a001e00be000224240055
:10c3a400f300200033dc07000043b000fefd07006b
:10c3b4001e00be0002242400f30020002ddc070030
:10c3c4000001be00002424000012b8006f10b90060
:10c3d4000503780000034300002424000098b900fa
:10c3e40000034300860278001e1f12001e971a00e5
:10c3f400e0c2b300ecfd07001e00be00026a280084
:10c40400130020001bdc07000043b000e6fd07001a
:10c414001e00be00026a28001300200015dc07007d
:10c424000001be00006a28000012b8006110b900c3
:10c434000503780000034300006a28000098b9004f
:10c4440000034300860278001e1f12001e971a0084
:10c454001e00be00027122000300200005dc07005c
:10c464000043b000d0fd07001e00be000271220090
:10c4740003002000ffdb07000001be000071220062
:10c484000012b8006010b9000503780000034300ef
:10c49400007122000098b90000034300860278006e
:10c4a4001e1f12001e971a001e00be00823e2000ae
:10c4b40003002000efdb07000043b000bafd0700d3
:10c4c4001e00be00823e200003002000e9db0700be
:10c4d4000001be00803e20000012b8006010b900c8
:10c4e4000503780000034300803e20000098b90053
:10c4f40000034300860278001e1f12001e971a00d4
:10c50400e0c2b300a8fd07001e00be0042062000e2
:10c5140003002000d7db07000043b000a2fd0700a2
:10c524001e00be004206200003002000d1db0700ed
:10c534000001be00400620000012b8006010b900df
:10c544000503780000034300400620000098b9006a
:10c5540000034300860278001e1f12001e971a0073
:10c564001e00be00a200200003002000c1db070063
:10c574000043b0008cfd07001e00be00a200200096
:10c5840003002000bbdb07000002be00a000200067
:10c594000023b8006020b9000701780000014100c1
:10c5a4006a28b90000014100820378001e1f1300ad
:10c5b4001e971b004e4090000004e00003003a0068
:10c5c4001e0078000043b00077fd07000080fa00e9
:10c5d400000006000600fa001007980021079800e2
:10c5e4000000eb00000f78009e009000f070220025
:10c5f400808f500002003400f07022001007980071
:10c60400ae00900040072000808f500012003200de
:10c614001e009000703eb00080007800e07c200096
:10c62400808f500005003e0000c2b3005efd07008d
:10c6340010002000000f7800090037001e00900051
:10c64400823e2000110009000200d8000043b0001f
:10c6540055fd07000200370010002000000f78008d
:10c664001e009000823e2000110009000200d80044
:10c6740080007800803e20000088b90080007800a7
:10c684001e009000010050001007980010002000c8
:10c694009e0f10000c003a001e0090003006b000ff
:10c6a40080007800600c2000808f500006003e005f
:10c6b4002e009000e20f50000300320000c2b300cd
:10c6c40039fd0700060037001e00900042062000d6
:10c6d400110009000200d8000043b00032fd070039
:10c6e4001e00900042062000110009000200d8003c
:10c6f40080007800400620000088b900800078009f
:10c704001e00900001005000100798002e009000b9
:10c71400e20f500002003a00e0c2b30022fd07001d
:10c724001e009000a2002000110009000200d800a1
:10c734000043b0001cfd07001e009000a200200072
:10c74400110009000200d8006a00b90080007800d6
:10c754001e00900001005000100798002e00900069
:10c76400e10f500002003a00e0c2b3000efd0700e2
:10c774001e0090000043b0000bfd07000080fa008b
:10c78400000006000200fa00000f7800703e20004e
:10c794009e0f100002003400703e2000000f78004d
:10c7a400310620001e80400080007800600c2000cc
:10c7b400808f500003003e0000c2b300fafc070063
:10c7c400060037001e007800420620001100090010
:10c7d4000200d8000043b000f3fc07001e007800fc
:10c7e40042062000110009000200d80080007800f1
:10c7f400400620000088b9001e0f10001e007800bb
:10c80400a2002000110009000200d8000043b0007b
:10c81400e5fc07001e007800a200200011000900ba
:10c824000200d8006a00b9001e0f1000e0c2b30075
:10c83400ddfc07001e0078000043b000dafc0700ae
:10c844000080fa00000006000200fa00000f7800e1
:10c85400300620009e0f1000020034003006200035
:10c86400000f78001e007800a200200011000900cb
:10c874000200d8000043b000cbfc07001e00780083
:10c88400a2002000110009000200d8006a00b900cb
:10c894001e0f1000e0c2b300c3fc07001e007800a6
:10c8a4000043b000c0fc07000080fa00000006004e
:10c8b4000200fa00004f780090c0b3009e4f1000b1
:10c8c4000200340090c0b300004f780001c3b300ed
:10c8d4001ec04000b4fc07000080fa0000000600ff
:10c8e4000400fa00004f78001e00fb0010079800b7
:10c8f4001e009000e30f5000230032001e00900041
:10c90400e30f50000a003c001e009000e10f5000ad
:10c91400170032001e009000e10f500017003c0089
:10c924001e0090000000e0000e00320024003700da
:10c934001e009000e50f5000190032001e00900008
:10c94400e50f5000130035001e009000e60f500064
:10c95400160032001e009000e70f5000160032004f
:10c964001700370040c22b001afe070014003700de
:10c9740070c22b0017fe070011003700a0c22b0065
:10c9840014fe07000e003700d0c22b0011fe070072
:10c994000b00370000c32b000efe07000800370011
:10c9a40030c32b000bfe07000500370060c32b00cb
:10c9b40008fe07000200370090c32b0005fe0700a5
:10c9c4000080fa00000006000600fa002007980024
:10c9d400b0cfb3004aeab7001000200050548800da
:10c9e4000000eb0010079800260037001e0090009e
:10c9f400a1a0200001004000104f7800b0cfb30088
:10ca04009e4f100006003200e0cfb3009e4f10008e
:10ca14000300320000c0eb009e4f100010003a00eb
:10ca240052548000a0a420008000410000c0eb000c
:10ca3400804878000200e800505488005154800077
:10ca44001e4178000244a200a0a4200000804000ff
:10ca5400024878000100e8005054880006003700be
:10ca640051548000a0a42000008040001e4878009b
:10ca74000100e800505488001e0090000000e80007
:10ca8400100798009e0090002e009000808f5000a8
:10ca9400d6ff350052548000a0a42000800041003d
:10caa400e0cfb300804878000200e80050548800ca
:10cab4000080fa00000006000400fa000000eb0009
:10cac400000f78000b0037001e0178001e0078006c
:10cad4008000400060ba200000804000900178008f
:10cae40082004100c0a820000080400003087800b4
:10caf4001e0fe8001e007800e80f5000f2ff360019
:10cb04000040eb002047980040c0b3000aeab70099
:10cb1400a1a02000914078002e40900001404000e8
:10cb2400204798000000eb00000f78001000370049
:10cb34009e007800c0a8200000804000904078004b
:10cb44002e40900001404000204798001e01e8005c
:10cb54009e007800c0a8200000804000904078002b
:10cb6400a0a0200000004100014878001e0fe8004a
:10cb74001e007800f10f5000edff36001e00e800a3
:10cb8400a1a0200001004000ae40900001487800c0
:10cb94000080fa00000006000400fa000040eb00e8
:10cba4002047980050c0b3000aeab700a1a02000b3
:10cbb400914078002e4090000140400020479800aa
:10cbc4000000eb00000f7800110037009e00780091
:10cbd400c0bf2a0000804000904078002e409000a2
:10cbe40000c04000204798001e01e8009e00780025
:10cbf400c0bf2a00008040001040780080407800c8
:10cc0400a0a0200000004100014878001e0fe800a9
:10cc1400400020009e0f1000ecff34001e00e800ce
:10cc2400a1a0200001004000ae409000014878001f
:10cc34000080fa00000006000200fa000040eb0049
:10cc4400004f780010c0b3000aeab700712e20002c
:10cc54009140780000c8b30000c060000004e00008
:10cc6400040032000acabf0001c8b30001407000ca
:10cc74000aeab700806980000000e0000400320086
:10cc84000acabf0001c8b300014070000aeab70035
:10cc9400a5cbbf000004e000040032000acabf00b4
:10cca40001c4b300014070000aeab700a4cbbf007e
:10ccb400e14f500004003a000acabf0001c2b300a9
:10ccc400014070000aeab700c8c2bf0070406000ab
:10ccd4000004e000030032000acabf000044a000c0
:10cce4000aeab7000acabf001e4f4000115d800067
:10ccf40060b9200000804000104078000040e80047
:10cd04004400dd0010479800105d8000ef40600093
:10cd14001e40900000c07000104798001e40900014
:10cd24000beab7000bcabf001e4f40000040eb00e7
:10cd340010479800c6c2bf00704060000004e000c5
:10cd440006003a00005c8000e10f500003003a0046
:10cd5400f0c0b300104798001f003700c6c2bf00e0
:10cd6400704060000004e00016003200405b800068
:10cd7400ee0f500003003400e0c0b30010479800e9
:10cd840002003700405b800010479800505b800031
:10cd9400ee0f5000050034001e40900001ceb30099
:10cda40001407000104798000b003700505b800072
:10cdb400c400dd001e409000014070001047980040
:10cdc40005003700806980000000e00002003200a6
:10cdd40000c5b300104798001e4090000ceab7004d
:10cde4000ccabf001e4f40000040eb0010479800e3
:10cdf400915b8000f00f2000808f5000030034000e
:10ce040000c0eb001047980002003700905b8000e0
:10ce1400104798001e4090000deab7000dcabf00ed
:10ce24001e4f4000405a80004200de000eeab70068
:10ce34000ecabf001e4f4000715a8000f01f200030
:10ce4400808f50000300340000c0eb000feab700ed
:10ce540003003700705a80000080d1000feab70049
:10ce64000fcabf001e4f4000f05a800010eab700fe
:10ce740010cabf001e4f40001e40780011eab700e0
:10ce84000080fa00000006000200fa0080aa2b00cd
:10ce9400801f780036cd07008f87e90000ad2b0096
:10cea400801f780032cd07008f87e9000000eb0077
:10ceb400000f78000b0037009e007800a0a020002f
:10cec40000804000104078000080fb00801f780044
:10ced400c0ad2b00801f780025cd0700e4875700e4
:10cee4001e0fe800600020009e0f1000f2ff3400c7
:10cef40030ae2b00801f78001dcd07008f87e9001e
:10cf040070002000b0fe070070ae2b00801f780078
:10cf140017cd07008f87e9000000eb00000f7800b1
:10cf24000b0037009e007800a0a420000080400081
:10cf3400104078000080fb00801f7800c0ad2b00fb
:10cf4400801f78000acd0700e48757001e0fe80011
:10cf5400505480009e0f1000f2ff35000080fa004c
:10cf6400000006000200fa00000f78001e0078009e
:10cf740095fe070051548000a0a420001f0b070059
:10cf84000080fa00000006000200fa00004f78005a
:10cf94000000eb00205a8800105d80000000e000d3
:10cfa4001c003200b0c2b3009e4f10000b003a00c8
:10cfb400125d800060b9200000004100104078003c
:10cfc4008040e80060b9200000004100014878007a
:10cfd400415e800020c4200056080700d0c2b30080
:10cfe4009e4f10000b003a00125d800060b92000d3
:10cff40000004100104078008040e90060b9200042
:10d004000000410001487800415e800020c42000f7
:10d0140048080700c7ec07000080fa00000006007b
:10d024000000fa00d7ea0700a5cbbf000004e00027
:10d0340007003200415e8000c0f620003d08070072
:10d044000040eb00a5ebb700e862a800060037003b
:10d05400415e800020c420003608070010c0b300e1
:10d06400a5ebb700e862a9000080fa000000060002
:10d074000400fa00000f7800c2ea07001e007800de
:10d08400100798001e009000e10f500010003200bd
:10d094001e009000e10f500004003c001e009000b0
:10d0a4000000e00008003200180037001e00900065
:10d0b400e20f50000d0032001e009000e90f5000f6
:10d0c4001100320011003700d5ff07000f003700b0
:10d0d400415e800020c420001608070010c0b30081
:10d0e400a5ebb700e862a90008003700415e8000a4
:10d0f400c0f620000f0807000040eb00a5ebb700c6
:10d10400e862a80001003700a40207000080fa00ca
:10d11400000006000400fa00000f78001e007800ea
:10d12400100798001e009000e10f50001600320016
:10d134001e009000e20f5000190032001e00900003
:10d144000000e000010032001a003700b4cbbf0039
:10d154000004e000060032000040eb00b4ebb7002e
:10d16400415e800020c42000f20707001100370050
:10d1740010c0b300b4ebb700415e8000c0f62000dd
:10d18400ec0707000b00370010c0b300b4ebb70086
:10d19400415e8000c0f62000e60707000500370066
:10d1a4000040eb00b4ebb700415e800020c42000d7
:10d1b400e007070056ec07000080fa0000000600b4
:10d1c4000000fa00005c80000000e00021003a004a
:10d1d400a4cbbf000004e0000e003a0010c0b3006e
:10d1e400a4ebb7000000eb00e0648800105d800051
:10d1f400205c88000000eb00105d8800415e800028
:10d2040020c42000cb070700ed0d0700d1a2a90020
:10d21400100037000040eb00a4ebb700b000200082
:10d22400105d8800115d800060b92000808040009e
:10d234000040eb00804878000040eb00a5ebb7000d
:10d24400e862a800415e8000c0f62000b90707002c
:10d25400d1a2a8000080fa00000006000200fa0033
:10d26400004f7800005c80000000e00038003a00c5
:10d27400a4cbbf000004e00035003a00805e8000cb
:10d284000000e00006003a00a5cbbf000004e00067
:10d29400030032000040eb00a5ebb700e862a800f1
:10d2a400e0c3b3009e4f100012003a00105d8000ee
:10d2b4000000e800105d8800105d8000eb0f500056
:10d2c40002003400b0002000105d8800105d800072
:10d2d400eb0f500004003a00415e8000f0a42000ef
:10d2e4009407070003003700415e800020c420003b
:10d2f40090070700c0c3b3009e4f100014003a000b
:10d304000040eb00a4ebb700105d80000000e900d2
:10d31400105d8800105d80000000e00002003c0009
:10d3240010002000105d8800105d8000e10f5000a7
:10d3340004003a00415e8000c0f620007d0707002b
:10d3440003003700415e800020c4200079070700f5
:10d354000080fa00000006000000fa000000eb0064
:10d36400e0668800d0ab2000f06688000000eb0087
:10d37400106788000000eb00206788000080fa0036
:10d38400000006000400fa00004f7800b0cfb3009c
:10d394009e4f100006003a00efff07001000200027
:10d3a400206788000000eb00100798002f0037006a
:10d3b400206780000000e00003003a000000eb005a
:10d3c4001007980029003700e0cfb3009e4f1000eb
:10d3d40006003a00e0668000bceab700deff070002
:10d3e400c0ab2000100798002000370000c0eb00fd
:10d3f4009e4f100005003a001000200010678800be
:10d404000000eb0010079800180037001067800038
:10d41400e10f500003003a001e44a2000000eb009c
:10d4240010678800e166800000042000808f5000af
:10d4340004003a00c8ff07000000eb001007980042
:10d444000a003700e06680000000e800e06688001b
:10d45400f06680001e487800f06680000000e80056
:10d46400f06688000000eb00100798001e00900092
:10d474000080fa00000006000600fa00bccabf00e3
:10d484000080fb00100798001e009000fe0f500063
:10d4940002003400e0012000100798000040eb0077
:10d4a400004f78001e0090000000e00015003400da
:10d4b400100020002007980008003700ae009000fc
:10d4c400c0ab200000804000104078001e4f400098
:10d4d4002e0090000000e80020079800ae009000a5
:10d4e4001e009000808f5000f4ff3500ae009000c5
:10d4f400c0ab200000804000904078001e407800bf
:10d50400014f50001e009000801f780010af2b00c8
:10d51400801f7800e0a92000a3cb0700e487570010
:10d52400e0a92000100d070010002000200798003b
:10d5340010003700ae009000c0ab20000080400017
:10d54400104078000080fb00801f7800c0b02b00e2
:10d55400801f7800e0a9200093cb0700e4875700e0
:10d56400e0a92000000d07002e0090000000e80054
:10d57400200798001e0090008000e8002e00900014
:10d58400808f5000ebff3c001e04e00005003a00d1
:10d59400e1a9200020b12b000e000900b05878004a
:10d5a400070037001e80fb00801f780010b22b009c
:10d5b400801f7800e0a920007bcb0700e487570098
:10d5c400e0a92000e80c07000080fa000000060033
:10d5d4000e00fa000040eb0060479800bccabf0090
:10d5e4000080fb00100798001e009000e10f50001f
:10d5f40003003c001000200040079800840037001e
:10d604009e009000e0032000808f5000030034004f
:10d6140021002000410798007d0037001000200001
:10d62400200798000a003700ae009000c0ab20002d
:10d6340000804000904078006e409000014040001f
:10d64400604798002e0090000000e8002007980032
:10d65400ae0090001e009000808f5000f2ff350055
:10d66400ae009000c0ab20000080400090407800e5
:10d674006e40900001405000604798006e4090005a
:10d684000004e0000300320032002000420798004a
:10d694005f003700bdcabf000080fb006101b90014
:10d6a4000080eb008080eb00020140008381480091
:10d6b4005207980063079800d00020000100200062
:10d6c4005e019000ee019000800f5100818f59009f
:10d6d4004d003e005e009000ee00900000600100ee
:10d6e40029003700440037002a0037001e003700a5
:10d6f400210037002c0037002e003700310037009e
:10d7040041003700160037000f00370002003700d1
:10d71400070037002f003700d082a80046fd07001d
:10d72400800020000ffe0700d082a90036003700d9
:10d73400d082a80018fd07007000200009fe070031
:10d74400d082a90030003700d082a800dafc07009c
:10d754004001200003fe0700d082a9002a00370000
:10d76400bcf3070028003700b0c2b30006fe070070
:10d77400b8f3070024003700d0c2b30002fe07004c
:10d78400b4f307002000370025fe0700b1f30700bb
:10d794001d003700becabf000080fb0034fe070036
:10d7a400acf307001800370085fe0700a9f3070053
:10d7b40015003700e0c3b300a8fe0700a5f3070077
:10d7c40011003700c0c3b300a4fe0700a1f3070093
:10d7d4000d003700becabf000080fb006a00b9001c
:10d7e400000f78009e007800d16688001e01780042
:10d7f400826a880004003700becabf000080fb00b4
:10d8040044fe0700dcf307008001eb0043079800a7
:10d814004e0090000080fa00000006000400fa00a8
:10d82400d06680000000e00008003200806a8000ba
:10d834000000e00005003a00d0668000806a88009d
:10d84400fdfc070080002000c6fd0700f00907006a
:10d854000004e00008003200e709070020479800b0
:10d864002e409000c7fe07000000e00002003200d6
:10d8740057ff0700000f78000080fa000000060040
:10d884000000fa00c03f2a00801f7800b8ca0700d1
:10d894008f87e90070432a00801f7800b4ca07000c
:10d8a4008f87e90080442a00801f7800b0ca0700ef
:10d8b4008f87e90080462a00801f7800acca0700e1
:10d8c4008f87e90020492a00801f7800a8ca070032
:10d8d4008f87e900304d2a00801f7800a4ca070012
:10d8e4008f87e900d0502a00801f7800a0ca070063
:10d8f4008f87e900c0522a00801f78009cca070065
:10d904008f87e90040542a00801f780098ca0700d6
:10d914008f87e90090552a00801f780094ca070079
:10d924008f87e90020572a00801f780090ca0700db
:10d934008f87e900d05a2a00801f78008cca07001c
:10d944008f87e900b05c2a00801f780088ca07002e
:10d954008f87e900705e2a00801f780084ca070060
:10d964008f87e90070602a00801f780080ca070052
:10d974008f87e90080612a00801f78007cca070035
:10d984008f87e900d0622a00801f780078ca0700d8
:10d994008f87e90060642a00801f780074ca07003a
:10d9a4008f87e90070662a00801f780070ca07001c
:10d9b4008f87e900f0672a00801f78006cca07008f
:10d9c4008f87e900a06b2a00801f780068ca0700cf
:10d9d4008f87e900206d2a00801f780064ca070041
:10d9e4008f87e900d06e2a00801f780060ca070084
:10d9f4008f87e9000080fa00000006000000fa00aa
:10da0400106f2a00801f780059ca07008f87e90029
:10da14003df80700c0722a00eef9070053003700f2
:10da240000c4b3002ef80700d0732a00e9f90700f8
:10da3400cfc2bf000044b2000004e00006003a0078
:10da440000c4b30026f80700e0742a00e1f90700d7
:10da5400401f2000fc100700cec2bf0062406000df
:10da64000004e00006003a0000c4b3001cf80700fc
:10da7400f0752a00d7f90700401f2000f2100700b4
:10da8400cec2bf00644060000004e00006003a001b
:10da940000c4b30012f8070000772a00cdf907008c
:10daa400401f2000e8100700cec2bf00684060009d
:10dab4000004e00008003a0000c4b30008f80700be
:10dac40010782a00c3f90700e862a900401f20006b
:10dad400dd10070001003700e862a800c3c2bf00e0
:10dae4000042b2000004e00006003a0000c4b300a3
:10daf400fbf7070030792a00b6f90700401f200021
:10db0400d1100700c3c2bf000044b2000004e0000b
:10db140008003a0000c4b300f1f70700507a2a0065
:10db2400acf90700d1a2a900401f2000c6100700cd
:10db340001003700d1a2a800c3c2bf0001c8b300ce
:10db4400014060000004e00006003a0000c4b30095
:10db5400e3f70700707b2a009ef90700401f2000ae
:10db6400b9100700401f2000b7100700280907005c
:10db74000004e000aaff3200ca040700a4cbbf00df
:10db84000004e00002003a00d1a2a800010037001e
:10db9400d1a2a9000080fa00000006001600fa00d5
:10dba400ca82a900c682a900e862a800d1a2a8007e
:10dbb400907c2a00801f7800edc907008f87e90058
:10dbc400c0802a00801f7800e9c907008f87e90018
:10dbd4000040eb00c2f707000e80e80051832a00e2
:10dbe40010000900315878001001b1000e80e800df
:10dbf40078f9070000c4b300b9f707000e80e80005
:10dc040061842a0010000900315878001001b10025
:10dc14000e80e8006ff907008d20a9000de2a9002d
:10dc24000f42a9008f00a90017e2a90019e2a90078
:10dc34001942a900e0012000000f78000f0037000e
:10dc44000040eb00a6f707008e80e8001e00780075
:10dc5400801f780070852a00801f780001007800fa
:10dc6400d1c90700e48757000e80e80059f907007e
:10dc7400803e2000741007001e0fe9001e00e00023
:10dc8400efff3d008ce0a9000000eb00800c880051
:10dc94000000eb00b00c88000000eb00200c8800b2
:10dca40013e1a8008cc0a90011e1a900067d0400bd
:10dcb400010000000080fa00000006001000fa00d5
:10dcc400d30807000004e0001e023200ca0807005f
:10dcd400004f78001e80fb006101b900f0fb2f00ab
:10dce400f1ff2f0002014000838148005207980091
:10dcf4006307980060032000010020005e0190008b
:10dd0400ee019000800f5100818f59000c023e00fb
:10dd14005e009000ee009000006001006f0037008c
:10dd2400ba013700da00370063003700d600370045
:10dd34004a00370002023700010237002e00370084
:10dd4400f4013700fe013700fd013700f30137000d
:10dd5400fb013700fa013700f9013700f8013700f9
:10dd64004f003700f6013700f5013700f4013700a2
:10dd7400f3013700d8003700f1013700f001370014
:10dd8400cb013700ee013700ed013700ec0137001d
:10dd9400eb013700ea013700e9013700e8013700f9
:10dda4005c013700e6013700de013700e40137008b
:10ddb400e3013700e2013700e1013700c801370011
:10ddc400df013700cd013700f6003700dc013700f2
:10ddd400db013700da0137009e013700d801370034
:10dde400d7013700d60137008a013700d401370044
:10ddf400d3013700d300370080862a00801f7800c3
:10de04005bc907008f87e90010892a00801f78000a
:10de140057c907008f87e900c0bf2a00801f780018
:10de240053c907008f87e900508a2a00801f7800b1
:10de34004fc907008f87e90020c02a00801f78009f
:10de44004bc907008f87e900e08a2a00801f780009
:10de540047c907008f87e900ba013700308d2a00cf
:10de6400801f780042c907008f87e9006e08070009
:10de740040079800ce009000204d2000808f500075
:10de840002003a006df30700ae01370000912a004a
:10de9400801f780036c907008f87e900a901370081
:10dea40090922a00801f780031c907008f87e9000b
:10deb40076f30700a3013700d0942a00801f78006e
:10dec4002bc907008f87e9008cf10700e1f10700f7
:10ded40092f2070028f207009a0137009000200010
:10dee4003007980064003700be0090007107980066
:10def4007e019000ec0f510035003200fe019000cd
:10df0400ec8f51000a003c007e009000ea0f5000a4
:10df14001b003200fe009000ea8f500022003c00fb
:10df24007e019000e90f51000b0032004f003700d2
:10df3400fe019000ee8f5100390032007e00900007
:10df4400ee0f50002c003500fe009000ef8f5000c3
:10df54003d003200450037003e009000d60f070018
:10df6400801f78003e019000821f780070962a007e
:10df7400801f7800fec80700e68757003b00370083
:10df84003e009000cc0f0700801f7800be01900077
:10df9400831f7800e0972a00801f7800f4c80700e8
:10dfa400e6875700310037003e009000c20f07009b
:10dfb400801f78003e009000801f780030992a006e
:10dfc400801f7800eac80700e6875700270037005b
:10dfd4003e009000b80f0700801f7800be0090003c
:10dfe400811f7800809a2a00801f7800e0c807000b
:10dff400e68757001d0037003e009000ae0f070073
:10e00400801f78003e019000821f7800d09b2a0078
:10e01400801f7800d6c80700e68757001300370032
:10e024003e009000a40f0700801f7800be019000fe
:10e03400831f7800209d2a00801f7800ccc8070029
:10e04400e6875700090037003e0090009a0f07004a
:10e05400801f78003e009000801f7800709e2a0088
:10e06400801f7800c2c80700e68757003e00900072
:10e074000000e800300798003e009000ef0f5000c9
:10e0840099ff34002f01370031f307002d013700c9
:10e09400c09f2a00801f7800b5c807008f87e90059
:10e0a4000000eb004007980012002000010f2f0031
:10e0b400f0072000800e07006800470013002000ce
:10e0c400020f2f00f10720009c0e0700bcf307008d
:10e0d4001ff307001b013700d0a22a00801f78001d
:10e0e400a3c807008f87e90087f6070011003700ef
:10e0f400c70707000004e000fdff3200be07070069
:10e10400004f7800d1c0b3009ecf100001003a0048
:10e114007df607001e80fb00801f780000a42a0003
:10e12400801f780092c80700e48757001e407800db
:10e13400fbf70700b2c1b3009e4f1100ecff3a0099
:10e1440000013700c0a42a00801f780088c8070097
:10e154008f87e9006cf607000e003700b807070048
:10e16400004f7800d3c0b3009ecf110001003a00e5
:10e1740065f607001e80fb00801f7800c0a52a00fa
:10e18400801f78007ac80700e48757001e40780093
:10e19400e3f70700b0c1b3009e4f1000efff3a0051
:10e1a400e800370040a62a00801f780070c80700e6
:10e1b4008f87e90054f6070000a92a0005f8070034
:10e1c4000000eb00400798004600370010aa2a0020
:10e1d400801f780066c807008f87e900980707004a
:10e1e400004f78001e80fb0040079800940707004a
:10e1f400004f78004e009000c800dd001e80fb0038
:10e2040000804000400798004e0190000200780012
:10e214000080ea008180ea00780d0700e8c2bf00b0
:10e224000080fb004300de000004a20061406000a7
:10e234006140600061406000614060004301dd00b6
:10e24400812e20009140780070cfb30000c06000a0
:10e2540002407000e8e2b700e0aa2a00801f7800bc
:10e2640043c807008f87e90075070700004f78004f
:10e274001e80fb004007980071070700004f7800dc
:10e284004e009000c800dd001e80fb0000804000ae
:10e29400400798004e019000020078000080ea00d8
:10e2a4008180ea00690d0700d1c2bf000080fb0035
:10e2b4004500de000004a20061406000614060008f
:10e2c40061406000614060004501dd00112d2000c7
:10e2d40091407800f0cdb30000c0600002407000af
:10e2e400d1e2b7004e009000e10f4000b7ff3a00c2
:10e2f4000080eb00410d07000080eb00530d070088
:10e304000000eb00650d07000000eb00770d07002f
:10e314008c003700b0ab2a00801f780014c80700b7
:10e324008f87e900f8f5070000a92a00a9f707007c
:10e334000000eb0030079800180037003e00900002
:10e34400560d07003e009000680d0700d1c2bf00c3
:10e354000080fb004500de000004a2006140600074
:10e364006140600061406000614060004501dd0083
:10e37400112d200091407800f0cdb30000c0600062
:10e3840002407000d1e2b70020032000ae0e070067
:10e394003e0090000000e800300798003e00900026
:10e3a400ee0f5000e5ff34000000eb003b0d0700ca
:10e3b4000000eb004d0d0700e8c2bf000080fb0029
:10e3c4004300de000004a200614060006140600080
:10e3d40061406000614060004301dd00812e200047
:10e3e4009140780070cfb30000c06000024070001c
:10e3f400e8e2b70020032000930e0700040707009b
:10e404000004e0004f003a00c9ff37007bfd07001d
:10e414004c00370020ae2a00801f7800d4c70700c4
:10e424008f87e900000707003007980030b12a0001
:10e43400801f7800cec707008f87e900fa0607001f
:10e4440020079800ae0090003e00900039030700ba
:10e454003c003700c0a82000801f7800e042200064
:10e46400801f780040b32a00801f7800c0c70700cf
:10e47400e6875700ec060700300798003e0090003e
:10e48400b1020700f0b52a00801f7800b8c7070062
:10e494008f87e900d8060700004f780050b72a009c
:10e4a400801f7800b2c707008f87e9002500370076
:10e4b40080b72a00801f7800adc707008f87e90066
:10e4c4000000eb00300798001e0090003e01900011
:10e4d400110009000200d800100798001900370045
:10e4e40060b82a00801f7800a1c707008f87e90061
:10e4f40015040700c404070012003700c0ba2a003c
:10e50400801f78009ac707008f87e9007e01070003
:10e514000c003700a1fd07000a003700f7f40700dc
:10e524000800370060bc2a00801f780090c70700ed
:10e534008f87e90000c4b300b0f30700010037007f
:10e54400cffc07000080fa00000006000600fa0075
:10e554001007980021079800b0002000000f7800f1
:10e564000c0037001e007800c200dd00a05c2b0008
:10e57400008040001000be000001be001e0090009c
:10e58400ae009000800f5100818f590003003900c4
:10e594001e0fe9001e00e000f2ff3c00b000200066
:10e5a4009e0f100002003a000000eb00000f7800fc
:10e5b4001e0078000080fa00000006000000fa0047
:10e5c40060c4b300d908070010c4b300d70807001b
:10e5d400b0c3b300d50807000080fa0000000600ad
:10e5e4000000fa0060c4b300d008070020c4b300e0
:10e5f400ce080700b0c3b300cc0807000080fa00bf
:10e60400000006000000fa0060c4b300c708070059
:10e6140020c5b300c5080700b0c3b300c308070092
:10e624000080fa00000006000000fa0060c4b30095
:10e63400be08070040c5b300bc080700b0c3b30060
:10e64400ba0807000080fa00000006000000fa0083
:10e65400d0c4b300b508070020c5b300b308070051
:10e6640010c3b300b108070000c3b300af0807002c
:10e6740000c3b300ad08070000c3b300ab08070034
:10e68400b0c3b300a90807000080fa000000060028
:10e694000000fa0080c5b300a408070040c5b30019
:10e6a400a2080700b0c3b300a00807000080fa0066
:10e6b400000006000000fa0080c5b3009b080700b4
:10e6c40090c4b30099080700b0c3b30097080700cb
:10e6d4000080fa00000006000000fa0000c5b30044
:10e6e4009208070030c5b30090080700b0c3b30018
:10e6f4008e0807000080fa00000006000200fa00fd
:10e70400004f780000c5b3008808070030c5b30087
:10e71400860807001e40780084080700b0c3b300d1
:10e72400820807000080fa00000006000a00fa00d0
:10e734006000b800100798002107980061c020000d
:10e744009140780000c3b30080cf500005003a0028
:10e7540071c020009140780000c3b30080cf500006
:10e76400050032001e009000ae00900030079800b3
:10e77400410798002900370040002000000f78006e
:10e784001f0037009e009000a0002000000ab8007f
:10e794001e0090006000b9000501780000014100ee
:10e7a4002e0090006a00b900000141008202780046
:10e7b40014079800250798009e00780040c02000a8
:10e7c40000804000104078000080fb000100200021
:10e7d4006f0160006000b8000300200002007000b8
:10e7e400838070001e019000ae0190000200400082
:10e7f4008380480010079800210798001e0fe80046
:10e80400c10020009e8f1000deff34001e00900027
:10e81400ae00900030079800410798003e00900039
:10e82400ce0090000080fa00000006000400fa0008
:10e834000000eb00000f780041c0200091407800f8
:10e8440060c4b30080cf500028003a0005ccbf005c
:10e854000080fb0010079800200420009e00900018
:10e86400808f50000f003200400520009e00900071
:10e87400808f500011003200100420009e00900090
:10e88400808f50000100320016003700a7ff0700f8
:10e89400b05f8800c15f880010002000000f78007e
:10e8a40012003700a1ff0700d05f8800e15f8800f5
:10e8b40020002000000f78000c003700a05f8000cb
:10e8c400e30f500004003a0006ccbf000080fb00b8
:10e8d4006f006000406b880030002000000f78005b
:10e8e400020037000000eb00000f780041c0200058
:10e8f4009140780080c5b30080cf50000e003a00ec
:10e9040005ccbf008080fb0090042000808f500065
:10e91400010032000600370084ff0700f05f880022
:10e924000160880040002000000f780002003700da
:10e934000000eb00000f78001e0078000080fa0051
:10e94400000006000600fa00204798000000eb00d3
:10e95400000f7800ae409000b0c3b30080cf5000e9
:10e964000a003a00a05f8000e10f5000020034006a
:10e97400aeff0700000f78000000eb00a05f8800e6
:10e984001e007800200798000d003700a15f80006a
:10e9940090032000808f500007003c00a15f80009e
:10e9a40040c02000008040002e41900002487800c2
:10e9b4000100e800a05f88001e007800200798008e
:10e9c4002e0090000080fa00000006000600fa0005
:10e9d4004800370001080700204798002e409000a7
:10e9e400d8ff0700000f7800400020009e0f1000a1
:10e9f4000e003a00b3cbbf00e34f50000b003a00c7
:10ea0400f05f800001608000d0fe07001060880085
:10ea1400005c80000000e00002003a00106080000a
:10ea2400105d880010002000206b8800b3cbbf006d
:10ea3400e44f50002f003a00300020009e0f1000d9
:10ea440010003a00406b8000200798002e009000d0
:10ea54000000e000040032002e009000e10f50009e
:10ea64000500320007003700d4fe07001000200024
:10ea7400306b880003003700d9fe07001000200027
:10ea8400306b8800306b8000e10f500019003a00b1
:10ea9400100020009e0f1000030032002000200010
:10eaa4009e0f100013003a00406b80000000e0004d
:10eab40005003a00b05f8000c15f8000a3fe07003c
:10eac4001060880004003700d05f8000e15f8000a0
:10ead4009efe070010608800005c80000000e000db
:10eae40002003a0010608000105d880010002000d1
:10eaf400206b8800a90707000004e000b5ff3a0076
:10eb04000080fa00000006000c00fa000000eb0090
:10eb1400000f7800e222a900a9070700dd003700f2
:10eb24009e0707000080fb00300798003e0090001d
:10eb34000000e0002b003200a807070040479800bf
:10eb44004e4090000000fb00100798009e009000cb
:10eb5400f00f200000806000100798001e00900055
:10eb6400801f7800a05f2b00801f780000c607007c
:10eb7400e48757009e009000b0032000808f50006f
:10eb840004003a0000602b00801f7800f8c50700dd
:10eb94008f87e9004e4090006aff07000000e00004
:10eba40010003200d05f8000e15f8000b25f80001f
:10ebb400c35f8000446b8000809fbe00829fbe00c4
:10ebc400841f780050642b00801f7800e8c507007c
:10ebd400ec87570070662b00801f7800e4c507009f
:10ebe4008f87e9000a0507000004e000a90032004d
:10ebf40001050700404798004e4090000000fb00cc
:10ec04006101b90000fd2f00f1ff2f000201400057
:10ec1400838148004207980053079800800420002d
:10ec2400010020004e019000de019000800f510091
:10ec3400818f590097003e004e009000de00900046
:10ec4400006001007f003700850037009100370025
:10ec5400900037008f0037008e0037008d0037009a
:10ec64008c0037008b0037008400370089003700a0
:10ec7400880037008700370086003700850037009a
:10ec8400840037008300370082003700810037009a
:10ec9400800037007f0037007e0037007d0037009a
:10eca4007c0037007b0037007a003700790037009a
:10ecb400780037007700370076003700750037009a
:10ecc400740037007300370072003700710037009a
:10ecd400700037006f0037006e0037006d0037009a
:10ece4006c003700200037006a00370069003700e5
:10ecf400680037006700370066003700650037009a
:10ed040064003700630037001e003700230037001b
:10ed1400600037005f0037005e0037005d00370099
:10ed24005c0037005b0037003400370059003700bf
:10ed340058003700570037003600370055003700b9
:10ed440054003700390037005200370019003700eb
:10ed5400500037001d0037004e0037004d003700cb
:10ed64004c0037001f003700a06a2b00801f78007a
:10ed74007fc507008f87e90010002000000f78008e
:10ed840044003700506c2b00801f780078c50700c2
:10ed94008f87e90009fe07003e003700d06d2b0085
:10eda400801f780072c507008f87e9000cfe0700fa
:10edb40038003700506f2b00801f78006cc50700a7
:10edc4008f87e9000ffe070032003700e0702b0048
:10edd400801f780066c507008f87e90012fe0700d0
:10ede4002c00370070722b00801f780060c507006c
:10edf4008f87e90026fe07002600370090742b0059
:10ee0400801f78005ac507008f87e90029fe070094
:10ee14002000370090752b00801f780054c5070030
:10ee24008f87e90009fe07001a00370050772b008e
:10ee3400801f78004ec507008f87e90026fe070073
:10ee44001400370040792b00801f780048c5070064
:10ee54008f87e90000c3b30028fe07000d003700c8
:10ee6400b07a2b00801f780041c507008f87e90026
:10ee740010c3b30021fe070006003700107c2b00ee
:10ee8400801f78003ac507008f87e90090c3b3005c
:10ee94001afe07001e00e00021ff32000080fa0085
:10eea400000006000200fa0030658000000f7800c0
:10eeb4000000eb00306588001e0078000080fa0036
:10eec400000006000000fa000000eb00800c88003f
:10eed4000000eb00b00c880040062000600c8800a5
:10eee40040062000700c8800e0002000800c8800a0
:10eef400007d2000900c8800007d2000a00c88007c
:10ef0400e0002000b00c88000000eb00000c88003a
:10ef14000000eb00100c8800e0002000200c8800aa
:10ef2400b0cc21007008880013e1a8008ce0a80090
:10ef34000000eb00e0648800800c2000206488005e
:10ef44000080fa00000006000200fa00000f7800ba
:10ef54001e007800000c88000080fa000000060003
:10ef64000200fa00000f78001e007800600c880090
:10ef74000080fa00000006000200fa00000f78008a
:10ef84001e007800900c88000080fa000000060043
:10ef9400809fbe00821f78003400f800000020002b
:10efa400a00188000200fa0050648000000f78007d
:10efb4001e007800e20f50001e0032001e00780090
:10efc400e30f5000310032001e007800e10f5000c2
:10efd40003003200d222a8008cc0a9003a003700f6
:10efe400d6c2bf000080fb000000d1000004a200d4
:10eff4006140600061406000614060006140600009
:10f0040000414000612d200091407800d0cfb30032
:10f0140000c0600002407000d6e2b70060088000c3
:10f024000000d100600888000000eb0050648800f4
:10f0340025003700d6c2bf000080fb000000d100cd
:10f044000004a20061406000614060006140600013
:10f054006140600000414000612d20009140780033
:10f06400d0cfb30000c0600002407000d6e2b70009
:10f07400d6c2bf00624060000004e000120032000b
:10f0840010002000506488000f003700d6c2bf0073
:10f094000080fb000000d1000004a2006140600079
:10f0a40061406000614060006140600000414000d8
:10f0b400612d200091407800d0cfb30000c06000e3
:10f0c40002407000d6e2b70084c0a9000080fa00b4
:10f0d4003400f9004f0178004f00be0000400600e4
:10f0e4000200fa00000f780030002000506488000d
:10f0f4001e00e90060088800600880000000d1005c
:10f1040030088800d622a900d222a90011e1a80063
:10f1140084c0a9008cc0a8000080fa00000006008a
:10f124000000fa0020002000506488000080fa00eb
:10f13400000006000400fa00000f78001107980090
:10f14400406480000000e00007003a001e009000c8
:10f154000000e000040034001e00900030648800c9
:10f164001e007800deff07000080fa0000000600a1
:10f174003600f800809fbe00829fbe00849fbe00c0
:10f18400869fbe003400f80000002000a001880023
:10f194000000fa0084e0a900306480000000e00070
:10f1a40007003200306480000000e9003064880009
:10f1b400306480000000e00001003a00d8ff07003e
:10f1c400106580000000e00003003200106580003c
:10f1d4000000e90010658800206480000000e90058
:10f1e40020648800206480000000e0000a003d00e4
:10f1f400800c200020648800006580000000e0008e
:10f2040003003a0010002000006588000200370067
:10f214000000eb0000658800a06a80000000e000a8
:10f2240003003200a06a80000000e900a06a8800a0
:10f23400b06a80000000e00003003200b06a800081
:10f244000000e900b06a8800206580000000e0004a
:10f2540003003200206580000000e900206588007a
:10f26400e06480000000e00003003200e0648000fd
:10f274000000e900e0648800f06480000000e00021
:10f2840003003200f06480000000e900f0648800ac
:10f29400806a80000000e00003003200806a800081
:10f2a4000000e900806a8800906a80000000e000a5
:10f2b40003003200906a80000000e900906a880030
:10f2c400606480000000400060648800cec2bf001b
:10f2d400644060000004e00004003a0060648000c0
:10f2e4000000a000606488000400370060648000af
:10f2f400e1ff2f00010060006064880070648000fa
:10f304000000400070648800cfc2bf000044b20017
:10f314000004e00004003a00706480000000a000d3
:10f32400706488000400370070648000e1ff2f00df
:10f334000100600070648800806480000000e000c8
:10f344000b003a0060648000e10f400011003a00b5
:10f354001000200080648800401f2000c0648800e2
:10f36400306580000000e80030658800090037003f
:10f37400606480000000e00006003a000000eb003a
:10f38400806488000000eb00c06488000000eb008b
:10f39400a0648800906480000000e0000b003a0044
:10f3a40070648000e10f400011003a00100020005a
:10f3b40090648800401f2000d0648800306580007d
:10f3c4000000e9003065880009003700706480009f
:10f3d4000000e00006003a000000eb0090648800a2
:10f3e4000000eb00d06488000000eb00b0648800eb
:10f3f400c06480000000e00008003200c0648000a7
:10f404000000e900c0648800c06480000000e000df
:10f4140002003a0000052000a0648800d064800047
:10f424000000e00008003200d06480000000e90021
:10f43400d0648800d06480000000e00002003a003c
:10f4440000052000b0648800a06480000000e00093
:10f454000b003200a06480000000e900a064880072
:10f46400a06480000000e00005003a0000052000d0
:10f47400a0648800306580000000e80030658800e2
:10f48400b06480000000e0000b003200b064800033
:10f494000000e900b0648800b06480000000e0006f
:10f4a40005003a0000052000b06488003065800043
:10f4b4000000e900306588000080fa003400f9009b
:10f4c4004f03be004f02be004f01be004f00be00fe
:10f4d4003600f900004006000600fa001007980004
:10f4e40021079800b0002000000f78000c003700be
:10f4f4001e007800c200dd00a07d2b0000804000cb
:10f504001000be000001be001e009000ae0090007e
:10f51400800f5100818f5900030039001e0fe9004c
:10f524001e00e000f2ff3c00b00020009e0f10001f
:10f5340002003a000000eb00000f78001e00780083
:10f544000080fa00000006000000fa00e222a80091
:10f554001b0507000080fa00000006000000fa0006
:10f56400e222a900160507000080fa000000060048
:10f574000000fa00e0cfb300ec040700e0cfb300d2
:10f58400ea040700905e8000e804070000ceb300a0
:10f59400e604070030c0b300e4040700d0cfb30092
:10f5a400e20407000080fa00000006000600fa00ea
:10f5b400204798002e409000e24f400007003a0098
:10f5c4000000eb00406788000000eb003067880013
:10f5d4000000eb00200798006e0037002e409000da
:10f5e400e34f400059003a00f0ccbf00eaecb7000a
:10f5f400f1ccbf00ebecb700f2ccbf00ececb700f1
:10f60400ecccbf000004e00003003200ecccbf00ef
:10f61400e34f50004a003a0030678000e70f500083
:10f624000300320030678000e80f500044003a00c5
:10f634006000b80020688800316888003067800066
:10f64400000fe90038003700246880003568800026
:10f65400a00020000023b8006020b9000701780052
:10f66400000141006a28b9000001410082037800ca
:10f6740026688800376888009e00780000cf200044
:10f6840000804000104078000080fb004400de0051
:10f694000081fb00030020002068800031688000a6
:10f6a4000200400083804800206888003168880098
:10f6b4002468800035688000a00020000023b80082
:10f6c4006020b90007017800000141006a28b900f0
:10f6d40000014100820378002668880037688800aa
:10f6e4009e00780000cf2000008040001040780089
:10f6f4000080fb00010020006f0160006000b80082
:10f7040003002000020070008380700022688000e3
:10f71400336880000000410081804900206888002f
:10f72400316888001e0fe900220020009e0f11009e
:10f73400c5ff3c001000200020079800150037008a
:10f7440092002000220798001200370030678000e2
:10f75400f20f50000d003c003167800000cf200004
:10f76400008040002e419000024878000100e8002b
:10f7740030678800406780000000e8004067880028
:10f784000000eb002007980002003700320620003a
:10f79400220798002e0090000080fa000000060066
:10f7a4000200fa000000eb00a06b88001100370093
:10f7b4008a040700004f78001e4078007bff070092
:10f7c400e10f50000b003a0020688000316880008f
:10f7d40041ff070070678800005c80000000e000c3
:10f7e40002003a0070678000105d8800100020005d
:10f7f400a06b8800690407000004e000ecff3a00f5
:10f804000080fa00000006000a00fa000000eb0085
:10f81400000f7800905e8000801f7800a0802b008d
:10f82400801f7800d2c20700e4875700b000370079
:10f834005a0407000080fb00300798003e00900047
:10f844000000e000340032006404070040479800e0
:10f854004e4090000000fb00100798009e009000ae
:10f86400f00f200000806000100798001e00900038
:10f87400801f7800a0822b00801f7800bcc2070084
:10f88400e48757009e009000d00f2000808f500026
:10f8940004003a0000832b00801f7800b4c20700e4
:10f8a4008f87e9004e40900040ff0700e10f5000b1
:10f8b40019003a00206880003168800006ff0700c4
:10f8c4007067880034678000eaccbf008082fb0048
:10f8d400ebccbf000081fb007367800020688000d0
:10f8e40031688000841f7800851f7800821f7800ab
:10f8f400831f7800809fbe0030832b00801f780018
:10f904009bc20700ee875700c0862b00801f78003b
:10f9140097c207008f87e900bd0107000004e000db
:10f9240073003200b4010700404798004e40900035
:10f934000000fb004007980080052000ce009000e6
:10f94400808f50001600320080052000ce00900009
:10f95400808f500009003c0010032000ce0090006e
:10f96400808f50003900320030032000ce00900018
:10f97400808f50001a0032005d00370060062000be
:10f98400ce009000808f50000c003200a0062000b2
:10f99400ce009000808f50004700320054003700a2
:10f9a400f08a2b00801f780071c207008f87e9005e
:10f9b40010002000000f78004d003700905e80009a
:10f9c4000080fb00801f7800c08c2b00801f780013
:10f9d40067c20700e4875700e5fe070044003700cc
:10f9e400608f2b00801f780061c207008f87e900b9
:10f9f400e0cfb300cd030700e0cfb300cb03070093
:10fa0400905e8000c903070000ceb300c70307005f
:10fa140050c0b300c50307000040eb00c303070058
:10fa240000c9b300c103070090c6b300bf030700b9
:10fa340030c0b300bd0307000040eb00bb03070068
:10fa4400d0cfb300b903070029003700e0912b00a1
:10fa5400801f780046c207008f87e900e0cfb3001b
:10fa6400b2030700e0cfb300b0030700905e80004c
:10fa7400ae03070000ceb300ac03070050c0b300d0
:10fa8400aa0307000040eb00a803070000c5b30069
:10fa9400a603070070c2b300a403070050c4b30058
:10faa400a203070010c0b300a0030700d0cfb30027
:10fab4009e0307000e00370080942b00801f7800ff
:10fac4002bc207008f87e900c0cfb300970307005c
:10fad400c0cfb30095030700c0cfb3009303070062
:10fae400c0cfb30091030700c0cfb3008f0307005a
:10faf4001e00e0004eff32000080fa000000060005
:10fb0400809fbe003400f80000002000a00188009f
:10fb14000200fa00e0108000004f7800d06a8000f4
:10fb24000000e800d06a880058cdbf000040e8001b
:10fb34008040780000c8bf0080cf50000800320029
:10fb440058cdbf008080fb00708020000080400002
:10fb54001e48780058cdbf000040e80058edb700bb
:10fb640018c2bf00624060000004e00001003200df
:10fb74001822a9008700a9000080fa003400f900c7
:10fb84004f00be0000400600801f78003400f800db
:10fb940000002000a00188000200fa00104080004c
:10fba400104f7800104080000000e80010408800ea
:10fbb400204080000000e900204088001e80fb00f7
:10fbc400d0108800e06a80000000e800e06a880045
:10fbd400204080000000e00003003a008f20a900cc
:10fbe4000040eb0006e8b7008720a9000080fa0077
:10fbf4003400f9004f007800004006000600fa00c7
:10fc040010079800210798002e0090000000e000e3
:10fc140023003400ae00900000102000808f5000bc
:10fc24001f003c001e0090000000e00001003a00ac
:10fc34001b0037001e009000104088002e0090002a
:10fc44002040880019c2bf00624060000004e00048
:10fc5400fcff3a0010408000104f780010408000f4
:10fc64000000e80010408800204080000000e90007
:10fc7400204088001e80fb00d0108800e06a8000cd
:10fc84000000e800e06a8800204080000000e000f6
:10fc94000300320010c0b30006e8b7008f20a800ac
:10fca4000080fa00000006000000fa0000e385006e
:10fcb400f01088000000eb00b01088000000eb009a
:10fcc400c01088008700a9008f00a80017e2a800d0
:10fcd40019e2a8001942a8000080fa0000000600fa
:10fce4000200fa00000f7800700020009e0f100040
:10fcf4000200340070002000000f78001e0078001d
:10fd040080004000a0c52b00008040001000780057
:10fd1400f01088000080fa00000006000200fa00db
:10fd2400004f780006c8bf00e14f5000fdff3200cd
:10fd340019c2bf00624060000004e000fcff3a000a
:10fd44009e00fb00f00f200000806000d0108800af
:10fd5400e06a80000000e800e06a88000080fa00a1
:10fd6400000006000200fa0081d5200091407800ce
:10fd740000c8bf0000c05000004fe9001e80fb0017
:10fd84000080fa00000006000000fa000040eb00ca
:10fd940000e8b70010c0b30058edb7000080fa00c7
:10fda400000006000000fa0000c8bf000040e800a0
:10fdb4008040780058cdbf0080cf5000faff320059
:10fdc40000c8bf000040e80000e8b70000c8bf005a
:10fdd4008080fb007080200000804000104078008c
:10fde4000080fb000080fa00000006000200fa0018
:10fdf400ecff0700004f78001e407800c7ff0700a3
:10fe04001e80fb000080fa00000006000200fa00d9
:10fe1400000f7800040037001e00780010407800be
:10fe2400beff07001e0fe8001e0078001040780097
:10fe34000004e000f8ff3a000080fa000000060029
:10fe44000600fa006000b800100798002107980027
:10fe5400d4ff0700804078000174a100014f7800ae
:10fe64001e407800adff0700f0c2b3009e4f1000a3
:10fe74001600340090c3b3009e4f100013003c00e2
:10fe84009e009000a0002000000ab8001e00900010
:10fe94006000b90005017800000141002e009000c7
:10fea4006a00b90000014100820278009e00fb0054
:10feb40000fd2f0000804000cf80de0004004000e1
:10fec400858048001007980021079800d0c0b3002f
:10fed4009e4f1000deff3a001e009000ae0090001e
:10fee4000080fa00000006000400fa00004f7800c9
:10fef40090c3b3009e4f100006003e001e407800e1
:10ff040001cdb300014040000000fb001007980041
:10ff14001400370060c4b3009e4f100006003e007a
:10ff24001e40780091ccb300014040000000fb006b
:10ff3400100798000b00370060c6b3009e4f1000f6
:10ff440006003e001e40780091cab3000140400004
:10ff54000000fb0010079800020037000000eb00cf
:10ff6400100798001e0090000080fa0000000600b0
:10ff74000400fa008bff0700004f78001e40780051
:10ff840066ff07001e407800d7ff0700104798005f
:10ff94001e4090002047980082ff0700004f780021
:10ffa4001e4078005dff07001e407800ceff07006a
:10ffb400104798002e4090000080fb004400dd00b4
:10ffc400804078001e40900000c040002047980008
:10ffd4002e4090000080fb000080fa000000060024
:10ffe4000200fa00004f78001e4078004bff070023
:10fff4000080fa00000006000200fa0069ff070012
:020000040001f9
:10000400004f78001e80fb000080fa00000006000c
:100014000200fa0053ff0700000f78001e0078006a
:100024000080fa00000006000400fa0084ff0700c4
:10003400008fbe001e00be000080fa000000060013
:100044000200fa00caff0700004f78001e80fb0080
:080054000080fa000000060024
:020000040000fa
:020000040001f9
:10005c00280d00001e00000002000000000000003f
:10006c00000000000000000000b6030000000000cb
:10007c00000700000000000000000000000000006d
:10008c0000960000fe0a00008a000000000000003c
:10009c006a0d000004000000020000006300630011
:1000ac00000000006e0d00000200000000000000c7
:1000bc00500d0000080000000200000000000000cd
:1000cc000000000000000000840c00003c00000058
:1000dc0000000000080d00002000000000000000df
:1000ec00000800000801000000000000580d00008e
:1000fc0006000000020000000100000000000000eb
:10010c000809000002010000000000005e0d000064
:10011c0006000000020000000100000000000000ca
:10012c00700d000002000000020000000000000042
:10013c00460d00000a00000000000000720d0000d7
:10014c000200000000000000880b00006c000000a2
:10015c0000000000740d000002000000020000000e
:10016c0000000000e60c000022000000000000006f
:10017c00640d0000060000000200000000000000fa
:10018c0000090000f40b00004c000000000000000f
:10019c00760d0000020000000200000000000000cc
:1001ac00400c00004400000000000000c00c0000e7
:1001bc0026000000020000004f76650072666c009d
:1001cc006f77200021003100323334003536370090
:1001dc0038393000205465007374000000000000b2
:1001ec000000000000000000000000000a0a0000ef
:1001fc00f400000000000000bc0e00000200000033
:10020c000200000001000000780d000088000000d2
:10021c0002000000d80db0000d880d000000000099
:10022c000000000000000000000208000202ae0006
:10023c000daf0d00ae0dae000dae0d00ae0d9e005f
:10024c000d00000000000000000000000000000095
:10025c000000000000000000000000000000020090
:10026c0008010100d60dd7000dd60d00d60dd60015
:10027c000dd60d00c60d00000000000000000000af
:10028c000000000000000000000000000000000062
:10029c00000000000100000000fe0d00ff0dfe003c
:1002ac000dfe0d00fe0dfe000dee0d000000000019
:1002bc000000000000000000000000000000000032
:1002cc000000000000000000000000009c0e000078
:1002dc0012000000020000000100020000040000f7
:1002ec000800100000000000202b2d00233000001f
:1002fc00ae0e00000800000002000000686a6c00ee
:10030c00747a4c0000000000b60e000006000000dd
:10031c00020000000400000000000000be0e0000ff
:10032c000200000000000000000e00004800000069
:10033c00020000000000000000000000244000004b
:10034c000000000000005900400000000000000008
:10035c0088c34000000000000084d70097410000d3
:10036c0080e0370079c3410043176e0005b5b50036
:10037c00b8934600f5f93f00e9034f00384d3200c1
:10038c001d30f900487782005a3cbf00737fdd00b6
:10039c004f157500480e00003200000002000000ee
:1003ac004e414e00006e61006e0049004e4600004a
:1003bc00696e660000303100323334003536370058
:1003cc0038396100626364006566000030313200c8
:1003dc003334350036373800394142004344450048
:1003ec00460000007a0e000022000000020000000f
:1003fc003031320033343500363738003961620021
:10040c0063646500660030003132330034353600e9
:10041c003738390041424300444546000000000093
:10042c00c00e0000020000000200000000000000ee
:10043c00c20e0000020000000200000030000000ac
:10044c00c40e0000020000000200000000000000ca
:10045c00c60e0000020000000000000000000000ba
:020000040000fa
:020000040001f9
:10046c001200fa00889fbe00600798006e00900092
:10047c00cf80de00d0cb0700200798003107980012
:10048c002e019000be0190002e009000be00900046
:10049c0093cb0700008fbe00ee009000d01e200012
:1004ac00808f500017003400d27b230063582b0040
:1004bc001e00be008acb07000004be0032ff2100e4
:1004cc0023e523002e009000be00900084cb070093
:1004dc000001be000800be0024cb070022852300cb
:1004ec00b324240021cb0700400798005107980043
:1004fc004e009000de00900070079800010f9800ed
:10050c0051003700ee00900040042000808f500016
:10051c001700340072712b0013852b001e00be00d7
:10052c006fcb07000004be00c2f5280023e82300af
:10053c002e009000be00900069cb07000001be00a9
:10054c000800be0009cb0700f2a72e00732124007f
:10055c0006cb070040079800510798004e0090000a
:10056c00de00900070079800010f980036003700ed
:10057c006e009000e70f500017003400c296200068
:10058c0093b72b001e00be0055cb07000004be0025
:10059c0072ce280083f323002e009000be00900042
:1005ac004fcb07000001be000800be00efca0700d9
:1005bc0042602500b31b2400ecca070040079800da
:1005cc00510798004e009000de00900070079800d4
:1005dc00010f98001c0037006e009000e30f5000d4
:1005ec000e0034002e009000be0090000001be00f2
:1005fc00deca07000200200003162400dbca070035
:10060c0040079800510798004e009000de009000c3
:10061c0070079800010f98000b003700a2cd2a003c
:10062c00a3f223002e009000be0090002ccb0700fc
:10063c0040079800510798004e009000de00900093
:10064c0070079800010f98007e0090008e089000b3
:10065c004f04be000080fa00000006001400fa00ef
:10066c00889fbe0050079800610798007207980099
:10067c00030f980002002000031a24005e00900073
:10068c00ee00900077cb07000000e0000100350081
:10069c00030037000000eb00100f98003300370008
:1006ac005e019000ee0190007e0090008e0890009c
:1006bc003fcb07000000e00001003d0003003700c5
:1006cc00f0702200100f9800280037005e01900097
:1006dc00ee0190007e0090008e08900072cb070017
:1006ec0020079800310798000200200003f823002f
:1006fc002e009000be0090009cca07000004be00b3
:10070c002e019000be0190000000200001f8230093
:10071c0095ca07000001be000800be0062cb0700ae
:10072c00008fbe00d2cc2c00732c24001e00be0007
:10073c001fcb07000000e00001003c000300370065
:10074c0030062000100f9800080037001e00be0075
:10075c000200200003122400e1ca070094cb07001a
:10076c00400798004e009000100f98001e08900053
:10077c004f04be000080fa00000006000e00fa00d4
:10078c0050079800610798005e019000ee01900000
:10079c005e009000ee009000d1ca07001007980090
:1007ac00210798001e009000ae009000c2af2900f7
:1007bc0043b22300caca07003007980041079800cb
:1007cc00105d8000ea0f500008003a00225e8000a5
:1007dc00335e80003e009000ce009000c0ca07003f
:1007ec00300798004107980007003700025e800030
:1007fc00135e80003e009000ce009000b8ca070047
:10080c0030079800410798003e009000ce00900001
:10081c0067cb0700000f78001e0078000080fa00fc
:10082c0000000600809fbe00821f78003400f80094
:10083c0000002000a00188000200fa009010800047
:10084c00004f7800006b80000000e800006b88000f
:10085c005ecdbf000040e8008040780008c9bf00b2
:10086c0080cf500008003200e2d520001241780001
:10087c008280fb0090902000008040001e48780091
:10088c000240e8005eedb7000ec2bf00624060009f
:10089c000004e000010032000e22a9008520a9000e
:1008ac000080fa003400f9004f0178004f00be00c0
:1008bc00004006000000fa0080e38500a0108800cc
:1008cc000000eb00601088000000eb007010880046
:1008dc008520a9008d20a8000de2a8000f42a800d9
:1008ec000080fa00000006000200fa00000f7800f9
:1008fc00700020009e0f10000200340070002000d9
:10090c00000f78001e00780080004000a0c62b006d
:10091c000080400010007800a01088000080fa00d1
:10092c00000006000200fa00004f78000fc2bf0062
:10093c00624060000004e000fcff3a009e00fb00f7
:10094c00f00f20000080600080108800106b800089
:10095c000000e800106b88000080fa000000060020
:10096c000200fa00000f7800040037001e00780027
:10097c0010407800ebff07001e0fe8001e00780007
:10098c00104078000004e000f8ff3a000080fa0004
:10099c00000006000000fa00e1d52000914078002c
:1009ac0008c9bf0000c050000040e9000080fb00f7
:1009bc000080fa00000006000000fa000040eb0086
:1009cc0008e9b70010c0b3005eedb7000080fa0074
:1009dc00000006000000fa0008c9bf000040e80053
:1009ec00804078005ecdbf0080cf5000faff32000f
:1009fc0008c9bf000040e80008e9b70008c9bf00fb
:100a0c008080fb0090902000008040001040780017
:100a1c000080fb000080fa00000006000200fa00d3
:100a2c00ecff0700004f78001e407800bdff070068
:100a3c001e80fb000080fa00000006000600fa0091
:100a4c006000b8001007980021079800e1ff07002c
:100a5c00804078000174a100014f78001e4078009e
:100a6c00b0ff0700f0c2b3009e4f10001600340018
:100a7c0090c3b3009e4f100013003c009e009000ea
:100a8c00a0002000000ab8001e0090006000b90011
:100a9c0005017800000141002e0090006a00b900a9
:100aac0000014100820278009e00fb0000fd2f0037
:100abc0000804000cf80de000400400085804800ac
:100acc001007980021079800d0c0b3009e4f10006b
:100adc00deff3a001e009000ae0090000080fa008d
:100aec00000006000400fa00004f780090c3b30029
:100afc009e4f100006003e001e40780001cdb30052
:100b0c00014040000000fb00100798001400370063
:100b1c0060c4b3009e4f100006003e001e407800db
:100b2c0091ccb300014040000000fb00100798007e
:100b3c000b00370060c6b3009e4f100006003e004d
:100b4c001e40780091cab300014040000000fb0039
:100b5c0010079800020037000000eb001007980007
:100b6c001e0090000080fa00000006000400fa004d
:100b7c0098ff0700004f78001e40780069ff0700bf
:100b8c001e407800d7ff0700104798001e409000c9
:100b9c00204798008fff0700004f78001e40780018
:100bac0060ff07001e407800ceff0700104798003a
:100bbc002e4090000080fb004400dd008040780057
:100bcc001e40900000c04000204798002e4090002e
:100bdc000080fb000080fa00000006000200fa0012
:100bec00004f7800c6eb0700c0962b0077ed07008e
:100bfc001e40780048ed0700ffff37003600f80074
:100c0c00809fbe00829fbe00849fbe00869fbe0058
:100c1c000200fa0030032000a01088000000eb0056
:100c2c00000f780002003700000000001e0fe800e3
:100c3c00f0cf27009e0f1000fbff3400a0972b0075
:100c4c00801f7800c8bd07008f87e900103a80002c
:100c5c00801f780040992b00801f7800c2bd0700d0
:100c6c00e4875700f0c4b300dcff0700ffff370038
:100c7c003600f800809fbe00829fbe00849fbe009d
:100c8c00869fbe000000fa0040688800516888000a
:100c9c00626888007368880084688800956888009a
:100cac00a6688800b7688800c8688800d96888007a
:100cbc00ea688800fb6888000c6988001d69880058
:100ccc002e6988003f698800209a2b00801f7800cd
:100cdc00a5bd07008f87e90040688000801f780061
:100cec00a09b2b00801f78009fbd0700e487570056
:100cfc0050688000801f7800409c2b00801f78007b
:100d0c0099bd0700e487570060688000801f780059
:100d1c00e09c2b00801f780093bd0700e4875700f0
:100d2c0070688000801f7800809d2b00801f7800e9
:100d3c008dbd0700e487570080688000801f780015
:100d4c00209e2b00801f780087bd0700e48757008a
:100d5c0090688000801f7800c09e2b00801f780058
:100d6c0081bd0700e4875700a0688000801f7800d1
:100d7c00609f2b00801f78007bbd0700e487570025
:100d8c00b0688000801f780000a02b00801f7800c6
:100d9c0075bd0700e4875700c0688000801f78008d
:100dac00a0a02b00801f78006fbd0700e4875700c0
:100dbc00d0688000801f780040a12b00801f780035
:100dcc0069bd0700e4875700e0688000801f780049
:100ddc00e0a12b00801f780063bd0700e48757005b
:100dec00f0688000801f780090a22b00801f780094
:100dfc005dbd0700e487570000698000801f780004
:100e0c0040a32b00801f780057bd0700e4875700d4
:100e1c0010698000801f7800f0a32b00801f7800e1
:100e2c0051bd0700e487570020698000801f7800bf
:100e3c00a0a42b00801f78004bbd0700e48757004f
:100e4c0030698000801f780050a52b00801f78002f
:100e5c0045bd0700e487570010c4b3005fff0700cf
:100e6c00ffff37003600f800809fbe00829fbe0057
:100e7c00849fbe00869fbe000000fa003f69880078
:100e8c000f90200000a62b00801f780036bd0700b5
:100e9c008f87e90030698000801f780050a52b00f7
:100eac00801f780030bd0700e487570030c5b300c1
:100ebc004aff0700ffff37003600f800809fbe0096
:100ecc00829fbe00849fbe00869fbe000000fa0079
:100edc0060a72b00801f780023bd07008f87e900d7
:100eec00a0c5b3003dff0700ffff37003600f80038
:100efc00809fbe00829fbe00849fbe00869fbe0066
:100f0c000000fa0090a0a9009120a900b0a82b0025
:100f1c00801f780014bd07008f87e90090c4b300d0
:100f2c002eff0700ffff37000000fa000040eb0027
:100f3c0072edb700cb02a800cae2a800cac2a80092
:100f4c000080fa00000006000400fa00004f780050
:100f5c0072cdbf009e4f10004c0032001e40780036
:100f6c0072edb7001e00fb00100798001e009000e9
:100f7c00e30f50002a0032001e009000e30f5000d7
:100f8c000a003c001e009000e10f500018003200d7
:100f9c001e009000e10f50001b003c001e00900052
:100fac000000e0000e003200380037001e009000f8
:100fbc00e50f5000260032001e009000e50f500097
:100fcc001d0035001e009000e60f50002600320078
:100fdc001e009000e70f5000290032002b00370054
:100fec00cb02a800cae2a800cac2a800270037009a
:100ffc00cae2a800cac2a800a00020009003070003
:10100c00cb02a90021003700cb02a800cac2a8005d
:10101c00a00020008a030700cae2a9001b003700c9
:10102c00cac2a800a000200085030700cb02a900bb
:10103c00cae2a90015003700cb02a800cae2a8003a
:10104c00a00020007e030700cac2a9000f003700d1
:10105c00cae2a800a000200079030700cac2a900b8
:10106c00cb02a90009003700cb02a800a000200089
:10107c0073030700cae2a900cac2a9000300370023
:10108c00cb02a900cae2a900cac2a9000080fa00da
:10109c00000006000600fa00000f78001e00780021
:1010ac006101b9000080eb008080eb000201400080
:1010bc0083814800120798002307980090002000b5
:1010cc00010020001e019000ae019000800f510025
:1010dc00818f590055003e001e009000ae0090001c
:1010ec0000600100090037001100370019003700bb
:1010fc00210037002900370031003700300037005d
:10110c0038003700370037003f003700e9a2a8004d
:10111c00e982a900e9c2a900c4e2a900c4c2a900dd
:10112c00e802a900e822a900e842a900470037001c
:10113c00e9a2a900e982a800e9c2a900c4e2a900b9
:10114c00c4c2a900e802a900e822a900e842a9004b
:10115c003e003700e9a2a900e982a900e9c2a80073
:10116c00c4e2a900c4c2a900e802a900e822a900af
:10117c00e842a90035003700e9a2a900e982a900dc
:10118c00e9c2a900c4e2a800c4c2a900e802a900ef
:10119c00e822a900e842a9002c003700e9a2a90026
:1011ac00e982a900e9c2a900c4e2a900c4c2a8004e
:1011bc00e802a900e822a900e842a90023003700b0
:1011cc00e9a2a900e982a900e9c2a900c4e2a90028
:1011dc00c4c2a900e802a800e822a900e842a900bc
:1011ec001a003700e9a2a900e982a900e9c2a90006
:1011fc00c4e2a900c4c2a900e802a900e822a80020
:10120c00e842a90011003700e9a2a900e982a9006f
:10121c00e9c2a900c4e2a900c4c2a900e802a9005d
:10122c00e822a900e842a80008003700e9a2a900ba
:10123c00e982a900e9c2a900c4e2a900c4c2a900bc
:10124c00e802a900e822a900e842a9000080fa00ff
:10125c00000006000600fa0010079800210798000d
:10126c00b0002000000f78000c0037001e00780042
:10127c00c200dd0000be2b00008040001000be004c
:10128c000001be001e009000ae009000800f5100c7
:10129c00818f5900030039001e0fe9001e00e00089
:1012ac00f2ff3c00b00020009e0f100002003a003c
:1012bc000000eb00000f78001e0078000080fa00a0
:1012cc00000006000000fa0090c4b30095fd070072
:1012dc0060c4b30093fd0700b0c3b30091fd0700d9
:1012ec000080fa00000006000a00fa006000b80056
:1012fc001007980021079800a1c4200091407800a5
:10130c0000c3b30080cf500005003a00b1c42000e8
:10131c009140780000c3b30080cf5000050032002c
:10132c001e009000ae009000300798004107980016
:10133c002900370040002000000f78001f00370004
:10134c009e009000a0002000000ab8001e00900033
:10135c006000b90005017800000141002e009000ea
:10136c006a00b9000001410082027800140798005d
:10137c00250798009e00780080c420000080400063
:10138c00104078000080fb00010020006f0160001d
:10139c006000b80003002000020070008380700021
:1013ac001e019000ae0190000200400083804800b6
:1013bc0010079800210798001e0fe800c1002000bc
:1013cc009e8f1000deff34001e009000ae009000d7
:1013dc0030079800410798003e009000ce00900026
:1013ec000080fa00000006000200fa000000eb008a
:1013fc00000f780081c420009140780090c4b300a5
:10140c0080cf50000e003a0049ccbf008080fb001a
:10141c0060042000808f500001003200060037006d
:10142c00b1ff0700106288002162880010002000c4
:10143c00000f7800020037000000eb00000f78006e
:10144c001e0078000080fa00000006000600fa007a
:10145c00204798000000eb00000f7800ae40900091
:10146c00b0c3b30080cf50000a003a000062800085
:10147c00e10f500002003400dbff0700000f780082
:10148c000000eb00006288001e0078002007980026
:10149c000d0037000162800090032000808f500007
:1014ac0007003c000162800080c4200000804000e6
:1014bc002e419000024878000100e800006288008c
:1014cc001e007800200798002e0090000080fa0083
:1014dc00000006000400fa000000eb00000f78008a
:1014ec00160037003bfd0700204798002e40900067
:1014fc00ff4f5000110034002e409000d3ff070026
:10150c00000f7800100020009e0f10000b003a0016
:10151c0010628000216280004eff0700306288005c
:10152c00005c80000000e00002003a0030628000a5
:10153c00105d880010002000b06b880015fd0700be
:10154c000004e000e7ff3a000080fa00000006000b
:10155c000000fa00d0c3b300f2fc070020c4b300b3
:10156c00f0fc0700105d8000eb0f500003003a0008
:10157c0000c3b300ebfc070004003700105d8000d3
:10158c006f4060000043b000e6fc0700a0c0b30051
:10159c00e4fc0700d0c0b300e2fc07000080fa00b6
:1015ac00000006000000fa00f0c3b300ddfc0700e9
:1015bc0020c4b300dbfc0700a0c0b300d9fc0700bb
:1015cc00d0c0b300d7fc07000080fa000000060072
:1015dc000200fa000000eb00000f78000600370054
:1015ec009e00780060d42000808040000040eb001a
:1015fc00804878001e0fe800700020009e0f10003d
:10160c00f7ff34000000eb00706a88000080fa00dd
:10161c00000006000400fa00004f78001e04e000f1
:10162c000c003200a0c0b3009e4f10000900320025
:10163c0000c2b3009e4f100006003200c0c2b300bf
:10164c009e4f100003003200e0c2b3009e4f10000a
:10165c0003003a0010002000100798000200370029
:10166c000000eb00100798001e0090000080fa00ac
:10167c00000006000800fa00c6fc07000080fb0012
:10168c00200798002e0090000000e0004d00320072
:10169c00d0fc0700204798002e409000ddff07008b
:1016ac000000e00047003a00ae409000d0c3b30009
:1016bc0080cf500004003200ae409000f0c3b30065
:1016cc0080cf500001003a00c1ff07002e4090006f
:1016dc00ed4f500030003a0046cdbf000000fb003b
:1016ec0030079800d0032000be009000808f50007f
:1016fc000d003200f0032000be009000808f5000df
:10170c00010032002200370071d420009140780093
:10171c0020c4b30080cf500001003a008cff0700ba
:10172c00abff07002700370071d4200091407800f0
:10173c0020c4b30080cf500013003a0048cdbf0046
:10174c000000fb006f0f6000900020009e0f100047
:10175c000d003c00b3cbbf00e14f50000a003a0033
:10176c00a4cbbf00e14f500007003a00005c8000a2
:10177c000000e00002003a009e007800115d880035
:10178c0010002000806b880091ff07000d003700cf
:10179c008fff07000b003700716a800060d42000b7
:1017ac0000804000ae40900001487800706a8000d4
:1017bc00e60f500003003c00706a80000000e80057
:1017cc00706a88000080fa00000006000000fa0031
:1017dc00e202a900ca42a900f053200010118800af
:1017ec0000002800001188008500a9000080fa0084
:1017fc00000006000200fa00000f7800506b800019
:10180c009e0f10000d0032008500a90020118000f1
:10181c00706b88001e007800201188001e00780074
:10182c00506b880085c0bf00614060000004e00080
:10183c00fcff3200ca42a800ca42a9000080fa008c
:10184c00000006000200fa00000f7800606b8000b8
:10185c009e0f10000d0032008500a90020118000a1
:10186c00706b88001e007800201188001e00780024
:10187c00606b880085c0bf00614060000004e00020
:10188c00fcff3200e202a800e202a9000080fa008c
:10189c00000006000200fa00000f7800506b800078
:1018ac009e0f10000d0032001e007800506b880057
:1018bc00e00020009e0f100002003600e000200027
:1018cc00000f78001e00780080004000c0c32b0081
:1018dc000080400010007800c6ff07000080fa006e
:1018ec00000006000200fa00000f7800606b800018
:1018fc009e0f10000d0032001e007800606b8800f7
:10190c00e00020009e0f100002003600e0002000d6
:10191c00000f78001e00780080004000c0c32b0030
:10192c000080400010007800c6ff07000080fa001d
:10193c00000006000000fa0071e8070060b32b00fd
:10194c0022ea070000c4b30063e80700cfc2bf005f
:10195c000044b2000004e00006003a0030b42b0052
:10196c001aea0700cfc2bf000044b2000004e00036
:10197c00fcff3200cec2bf00624060000004e000f9
:10198c0006003a0030b52b0010ea0700cec2bf00ab
:10199c00624060000004e000fcff3200cec2bf00d9
:1019ac00644060000004e00006003a00c0b52b0063
:1019bc0006ea0700cec2bf00644060000004e000ed
:1019cc00fcff3200cec2bf00684060000004e000a3
:1019dc0006003a00a0b62b00fce90700cec2bf00ff
:1019ec00684060000004e000fcff3200c3c2bf008e
:1019fc000042b2000004e00006003a0030b72b00b1
:101a0c00f2e90700c3c2bf000042b2000004e000cc
:101a1c00fcff3200c3c2bf000044b2000004e0006f
:101a2c0006003a0010b82b00e8e90700c3c2bf005b
:101a3c000044b2000004e000fcff3200c3c2bf004f
:101a4c0001c8b300014060000004e00007003a0048
:101a5c00a0b82b00dde90700c3c2bf0001c8b3006a
:101a6c00014060000004e000fbff32000bf50700b2
:101a7c0023e807000080fa00000006003200f8009e
:101a8c00900188006118e100040032007018e10038
:101a9c0002003200f0ff2f00030037003119ba00aa
:101aac008301e900fdff3a003200f9000000060056
:101abc00849fbe004220a900440424006110e10070
:101acc000a003200540424007010e10007003200b8
:101adc0064042400f5ff2f000510e1000300320020
:101aec00f0ff2f004f02be00000006003200f8008d
:101afc00203b8800113b8800043b88000500fc005b
:101b0c0050052000303b8800a00a2000303b8800a4
:101b1c0061e7a800000000000000000061e7af00d2
:101b2c00feff37000000eb003200f9004f02be0050
:101b3c0000000600841f78004220a9004400240005
:101b4c006118e10006003200540024007018e10016
